:020000040800F2
:1000000000200010690803088108020839C30108AC
:100010007D0802087908020875080208000000003F
:10002000000000000000000000000000710802084D
:100030006D080208000000006908020879B501088F
:10004000D1080308D1080308D1080308D108030820
:10005000D1080308D108030815D0010855D10108BB
:1000600015D10108D5D0010895D0010849600008D4
:10007000396000082960000819600008096000085C
:10008000F55F0008E15F0008D1080308D108030804
:1000900069430208D1080308D108030855D00108B4
:1000A000D1080308D1080308D1080308D1080308C0
:1000B00079A20108BDA1010801A10108D108030826
:1000C000D1080308D1080308D1080308D1080308A0
:1000D000D1080308D1080308D1080308B9B50108FD
:1000E000D5CF0108D1080308F5FD0208D10803089F
:1000F000719F0108D108030839A00108D10803083D
:10010000000000000000000000000000D10803080B
:10011000D1080308D1080308D1080308D10803084F
:10012000CD5F0008B95F0008A55F0008915F000877
:100130007D5F0008D10803080000000000000000F7
:10014000D1080308D1080308D10803080000000003
:10015000000000000000000000000000000000009F
:100160000000000000000000D1080308D1080308C7
:10017000D10803080000000000000000000000009B
:0801800000000000D108030893
:1001880090ED057A90ED004AD0ED066AD0ED014A6F
:10019800D0ED047A90ED035AD0ED025AA4EE007A1D
:1001A800B0EE406AB0EE470AB0EE667AA4EE867A00
:1001B80067EEC07AA5EE407AE5EE867A80ED057A9C
:1001C800C0ED067A704700BFD0ED057A90ED013A90
:1001D800D0ED003AD0ED064A90ED024A90ED077A4C
:1001E80090ED035A90ED086AD0ED045AC0ED067AF6
:1001F800F0EE406A27EE830AC0ED056AA3EEA60A70
:1002080080ED087AA4EE240AA5EE470AA5EEC60AF0
:1002180080ED070A704700BFD0ED007A90ED017AB3
:1002280030EE670AE7EE007AB0EE670AC0ED007AB2
:10023800704700BF704700BF0028F0B403DA2D23D1
:100248000B7040420131092804464FF0010307DDD5
:1002580003EB83035B00B0FBF3F2092AF8D883B100
:100268000F48A0FB0326B4FBF3F2092A02F1570C4E
:1002780002F1300709DD03FB1244F30801F801CB52
:10028800EFD100230B70F0BC704703FB1244F30856
:1002980001F8017BE5D100230B70F0BC704700BF6B
:1002A800CDCCCCCC884270B44FF0010442D301FBD2
:1002B80004F4B0FBF4F58D42F9D2ECB142BB092D40
:1002C80004FB150005F1570605F130020EDDB4FBFD
:1002D800F1F403F8016B7CB1B0FBF4F5092D04FBD4
:1002E800150005F1570605F13002F0DCB4FBF1F416
:1002F80003F8012B002CEFD100221A7070BC704754
:1003080003F8016BB4FBF1F4002CF5D0B0FBF4F565
:10031800092D04FB150005F1370605F13002EFDC65
:10032800B4FBF1F403F8012B002CEFD100221A7072
:1003380070BC70470546002AEAD1C0E72DE9F047AE
:1003480014461D4606464FF47A7200232046294675
:1003580030F0BAF84D4BDFF848814D4A4D4F034411
:1003680088FB03101844D91782FB032CC1EB6010DB
:1003780088FB002887FB03279C44474AC1EBEC2CE9
:10038800C0EB001E82FB0C29A3EB8E0E1F44434AD0
:1003980086F806E0C1EB27474FEAEC7E08EB000A37
:1003A800CEEBA90E82FB07824FEAE0780EEB4E0EE9
:1003B800C8EB6A18ACEBCE0CC8EB0818DFF8E4E021
:1003C80086F804C0A0EB880070718EFB0303F81751
:1003D800C0EBE21240F2B55000FB1272C1EBE353DE
:1003E800B2F5896F4FEA83073CDA40F2DA239A4282
:1003F80042DCB2F5B77FB4BF4FF0000E4FF0010EEC
:100408004FEA4E09DFF8A08009EB0E0308EBC3039F
:100418001FFA8EFCD88A09EB0E0108EBC1011631D0
:100428000B2301E031F8020D904218DD013BF9D1B0
:10043800CE44012338F83E00B37007F5FA6701325D
:10044800121ABC44F270A6F800C0204629464FF4A0
:100458007A72002330F038F83281BDE8F087013332
:10046800DBB2E9E74FF0030CE64640F29650DFF8BE
:1004780038804FF00609CEE74FF0020CDFF82880ED
:10048800E64640F229404FF00409C4E780BC92C711
:10049800C5B3A29107452EC2ABAAAA2A73B06D169E
:1004A80089888888792D0311BC0D030803685A1CB4
:1004B80002601970704700BF2DE9F047089C257845
:1004C800002B804689460CBF4FF0200A4FF0300AB7
:1004D800661C25B3002A26DD334601E0024698B1A2
:1004E80013F8011B501E0029F8D1971E60B13D4634
:1004F800013D51464046C8476B1C002BF8DC257867
:1005080027EAE770013045B1041B29464046C84731
:10051800301916F8015B002DF7D1BDE8F087002AE5
:1005280003DC2846F9E70020EEE7571EDFE700BFA7
:10053800034600F11001FF221A705A7002338B42F1
:10054800FAD10271427170470123212100224170C2
:10055800C27003708370704730B4152216231725B4
:100568002D242E21027043702F22FF2385704471A1
:100578008171C27143738373C370037103724372D1
:1005880030BC704730B409222C23022518241921C5
:10059800027043721A22002385728473C172027337
:1005A800437330BC704700BF30B4022300250124D8
:1005B80014213D2205708470C17082714370C3712B
:1005C80030BC7047002306214FF47A720170C0E9ED
:1005D80001230373704700BFCB794A7930B48D7912
:1005E8000C7BDB09520202F4606243EA45031343C1
:1005F80022071DD40380CB790A7A5B0103F47E635A
:1006080043EAD20343808B7A0A7A4C7ADB09520296
:1006180043EA440302F46062134383808B7ACA7A04
:100628005B0103F47E6343EAD203C38030BC7047A6
:100638000381CB790A7A5B0103F47E6343EAD20330
:1006480043818B7A0A7A4C7ADB09520243EA4403E3
:1006580002F46062134383818B7ACA7A5B0103F4E4
:100668007E6343EAD203C38130BC704701207047E0
:10067800CB79002B5ED1F0B58D7A4E7B91F809C00D
:10068800CF7A0A7CCB7C91F811E02C0204F47064D8
:100698004CEA04042D094FEA062C45EA07150CF428
:1006A800706791F80CC04CEA070C8F7B85B036094F
:1006B80046EA07161702ADF8025007F47065CF7BBB
:1006C800ADF804C02F4391F814C08D7CADF80660D6
:1006D8001902120901F470611B0942EA0E1229433A
:1006E80043EA0C1304ADADF80870ADF80A20ADF874
:1006F8000040114EADF80C10ADF80E300DF10202AD
:10070800C5F10E0CC5F11E0701E032F8024BC4F327
:100718000A0303F2CA4321054FEA4303A6FB031366
:100728004CBFB9180CEB02015B08AA424352ECD14A
:1007380005B0F0BD704700BFABAAAAAAF0B4174C29
:100748002378591C01F03F01E5184B1C21447E26F3
:1007580003F03F021B232E7122700B71C61D7D27EB
:1007680004E0A518B042DAB2297113D010F8011BC1
:10077800A1F17D05531C012D03F03F03F1D822445C
:10078800E51881F020010133B042177103F03F02F0
:100798002971EBD12270F0BC704700BFF80F002020
:1007A800F0B58F7A8D79CC7ACE790A7CDFED5F3A15
:1007B8004B7C4FEA072E0EF4706E45EA0E053F019A
:1007C80007F4706C04EE105A4FEA042E0D7A2401D7
:1007D80004F470670EF4706E46EA0C0404EE904A56
:1007E80045EA0E0405EE104A4C7AF8EEE44A3C431A
:1007F80005EE904A16020C7B120102F4706506F4AD
:1008080070664A7BB8EEC55A64EEA34A34432A435D
:1008180006EE104AF8EEE55A25EE235AFCEEE44AB5
:1008280006EE902A1D028A7B1B0185B003F47064D2
:1008380005F47065CB7BB8EEC66A14EE901A65EEC7
:10084800A35ABCEEC55A2A4307EE102AB8EEC44A8A
:10085800F8EEE66A26EE236AFCEEE55AADF80210D9
:1008680015EE101A234307EE903AB8EEC77A24EE35
:10087800234A66EEA36ABCEEC66AADF8041015EE0C
:10088800901AF8EEE77A27EE237ABCEEC44AFCEE1B
:10089800E66AADF8061016EE101A67EEA37A14EEA3
:1008A800103ABCEEC77AADF8081016EE901A9BB253
:1008B800FCEEE77AADF80A1017EE101A1A46ADF8F2
:1008C8000C10A2F5487217EE901A0DF10204B2F559
:1008D800AF6FADF80E10ADF80030214604AD08D862
:1008E800A9420CD031F8022BA2F54872B2F5AF6FCD
:1008F800F6D90F4B1B78122B0CD005B0F0BD821E19
:100908000E3001E034F8023B22F8023F9042F9D160
:1009180005B0F0BD074A0849B2F8443001339BB22C
:10092800A2F844300B8005B0F0BD00BFABAA2A3F47
:1009380004270020F80F002008270020054A92F815
:1009480046303F2B05D8D118013381F8480082F88A
:1009580046307047F80F0020014BD3F8883018470D
:10096800F80F00200206144A1449127800EBC0035D
:100978004FEA131346BF523B1BB24133032AA1F877
:100988008C3000D0704770B40D4D0E4E28780E4C48
:1009980036F81020DB009BB29A1A26F8103023682C
:1009A800411C13440948236001F00F011A092970FA
:1009B800028070BC704700BFB2380020F80F0020DA
:1009C800B3380020B4380020D4380020D8380020AC
:1009D80038B590F90E30002B01DB002038BD0378C4
:1009E800812BFAD1104D427995F98E30B3EBD20FA5
:1009F800F3D149B195F8912043789A42EDD195F811
:100A0800922083789A42E8D10446407BFFF7AAFFF8
:100A1800E37A227B9B0003F01C0343EA921385F8D8
:100A2800CC30012038BD00BFF80F002040F0800115
:100A380001481CF05DBC00BF544000204FF4006327
:100A4800038370470B460246FF2101481CF098BCFF
:100A58005440002010B50446FB20FFF7E7FF00F0E4
:100A68007F000E2801D8002010BD20460F21FFF777
:100A7800E9FF012010BD00BF012380F85030704706
:100A880038B5144C94F8C83063B1F020FFF7CEFFA6
:100A98000546F120FFF7CAFF802D01D0002038BDA0
:100AA8000328FBD10C4B987B1BF032F8C4F8D0001C
:100AB8000028F3D0392200218271C1711BF07EFA1F
:100AC800064B1A781AB903221A70012038BD012082
:100AD80038BD00BFF80F002044400020B238002085
:100AE80070B4D0E90041057B02690223AB40636022
:100AF8000B684FF6FE7003400B60EFF31183502133
:100B080081F31288D66B3168C9071CD4706870B934
:100B1800D2E909418C4213D095690D44F56017D884
:100B28001469611A71609062002182F85810326865
:100B380042F00102DBB2326083F3118870BC704767
:100B4800012182F85810DBB283F3118870BC70471A
:100B5800611A71609462E7E770B40468037B2268E5
:100B6800022101FA03F31A4216D002691148124908
:100B7800642505FB02020D785068016875B915698E
:100B8800528928684FF6FE7630402860C868D243FC
:100B980092B20240CA60636070BC70470069026824
:100BA8004FF6FE752A400260CA684FF6FF600240A1
:100BB800CA60F0E7445300204053002010B501F00C
:100BC800010428B1C94301F0010101381CF0E2F920
:100BD80014B9024B024ADA6010BD00BF00ED00E014
:100BE8000400FA05014B18681AF0D4BD402600200D
:100BF80010B50368017B1A6802238B401342044630
:100C080011D0114AD2F8D4300133202BC2F8D43095
:100C18000AD1182200210D4830F079F8217B22688A
:100C280002238B40536010BD222BF7D10023C2F85A
:100C3800D430074A13704268136823F001031B0479
:100C48001B0C1360EAE700BFF80F0020343B0020BC
:100C5800693300201CF0D4BC30B4012200231025D5
:100C680011244FF6FF7145704471027202700271CF
:100C780043818381C3810182817430BC704700BF86
:100C880010B500210446012019F094FB207010BD16
:100C980038B52C22002130F03AF8034640F2DC51F6
:100CA800642040F21A4240F26C7540F20224187433
:100CB8005982132040F275319A8240F64302DD8250
:100CC8001C830E2502249876D9830A2019211A84B8
:100CD800012283F82B001973197783F8225083F8BF
:100CE8002A409A7383F8252083F829201946024858
:100CF800BDE8384029F0C2BE9453030810B50C462D
:100D080029F00AFBFFF7BCFE08230A4823700A4AA9
:100D18000A4B01781268C3F8D82013294FF0000253
:100D280083F8DC2008BF064B4FF0010008BF1A808B
:100D380010BD00BF0427002098450020F80F0020B0
:100D48000827002008B5302011F034FA4FF47A70E3
:100D58001AF09CFA8E2104481CF0CAFAA0F1C400CB
:100D6800B0FA80F0400908BD5440002010B51A4C74
:100D7800362011F01FFA94F98E3003EB4303234415
:100D8800232093F8E01011F00DFA94F98E3003EB5C
:100D980043032344242093F8E11011F003FA94F953
:100DA8008E3003EB43032344252093F8E21011F01F
:100DB800F9F994F88E1001EB41014900103101F066
:100DC800FE010A2011F0EEF93A2011F0F3F934206F
:100DD800BDE8104011F0EEB9F80F0020094890F86E
:100DE800CC1090F98E300B44DAB2931C5BB21D2BF9
:100DF800C4BFA2F11D035BB2002BF4DB80F88E3078
:100E0800B4E700BFF80F002010B50D4B0D4A0E4C8B
:100E18001B781268C4F84021132B4FF0C00284F8E5
:100E2800442103D1094B4FF6C072DA80C0210C204F
:100E380011F0B8F90F2384F88E30BDE8104095E71B
:100E48000427002098450020F80F002008270020DC
:100E580010B5264C94F8453194F846211844C0B290
:100E6800904284F8450105D3801AC0B29042FBD263
:100E780084F84501362011F09DF994F84531234452
:100E8800232093F8943003EB4303234493F8481149
:100E980011F088F994F845312344242093F89430CC
:100EA80003EB4303234493F8491111F07BF994F8B9
:100EB80045312344252093F8943003EB430323441E
:100EC80093F84A1111F06EF994F8453123440A2039
:100ED80093F8941011F066F994F84534082B00D073
:100EE80010BD3A20BDE8104011F064B9F80F002099
:100EF80070B505460E4629F00FFAFFF7C1FD2B78AD
:100F0800334C092B84F845342DD00F2B2BD0082BCC
:100F180012D0304B1A780AB903221A702E4A126876
:100F2800C4F85C2400233222C4F8543484F86034B2
:100F3800C4F85824012070BD284A33701368284A21
:100F48002849C4F888205A05C4F84814E1D5264B26
:100F58001A7892BB254A2649116002221A70012389
:100F680084F84C34D5E710202249234A3070092BE5
:100F7800C4F84814C4F8882013D00F2B06D12322B4
:100F88004FF4AF6384F84D24A4F84E34134B1B6818
:100F98005B05BED5194D2B788BB1002384F85034EE
:100FA800B7E74FF4C873A4F84E340C4B1B682022E3
:100FB8005B0584F84D24ACD5ECE70023D0E7104B53
:100FC800104A1A6021F02AFC02232B700123E5E75E
:100FD800F80F0020B238002098450020344E002039
:100FE800A907000841220008FA320020AC27002097
:100FF80045090008CD1B000879060008C832002002
:10100800402D00204507000838B50F4C054694F8D8
:1010180093100C2011F0C6F80821182011F0C2F81E
:1010280085B994F89110092011F0BCF80D2107201A
:1010380011F0B8F81621192011F0B4F8BDE83840BD
:101048002AF082BC0321EEE7F80F0020024BD3F808
:10105800D0001BF0B1BF00BFF80F0020F8B5D94E83
:1010680005461AF0C1F896F8DC3004460E2B00F25B
:10107800E580DFE813F00F00F1000C01E300E30066
:10108800E300E300E300E300E30049015701B50191
:10109800D801E500CC4BD6F8D8201B689B1A0A2B40
:1010A80040F2CC80002529F01BF9A6F86254FFF71E
:1010B80049FE0121022011F075F80721032011F0E3
:1010C80071F8D321042011F06DF89121052011F059
:1010D80069F80D21062011F065F80421072011F0A8
:1010E80061F80C21082011F05DF82921092011F080
:1010F80059F806210B2011F055F896F89310B34CC7
:101108000C2011F04FF85C210D2011F04BF84E2106
:101118000E2011F047F8C4210F2011F043F87C216C
:10112800102011F03FF84321112011F03BF8032162
:10113800122011F037F82321132011F033F83B2146
:10114800142011F02FF84421152011F02BF80F214D
:10115800172011F027F80821182011F023F81D2175
:10116800192011F01FF86C211A2011F01BF8032127
:101178001B2011F017F840211C2011F013F89121C1
:101188001D2011F00FF85621212011F00BF8102125
:10119800222011F007F8A921232011F003F80A21D1
:1011A800242010F0FFFF2946252010F0FBFF112115
:1011B800262010F0F7FF5921292010F0F3FF88218D
:1011C8002C2010F0EFFF31212D2010F0EBFF0B2128
:1011D8002E2010F0E7FFFF213E2010F0E3FF04F17E
:1011E8005A071025362010F0E5FF29460A2010F08E
:1011F800D9FF332010F0DEFF4FF461701AF046F883
:101208002320FFF713FC20702420FFF70FFC6070E9
:101218002520FFF70BFC033404F8010C0635BC420B
:10122800EDB2DFD16A4B1A780A23132A86F8DC302C
:1012380004D1684AB6F86214518013800020F8BDC2
:1012480019F0FAFA624B1A780023132A86F8DC3070
:1012580000F084810120F8BDFFF7F8FE002840F077
:10126800BC81D6F86434E41A002C40F31B814FF497
:10127800FA7029F00FF8FFF7B1FDD6F8643403F5DA
:10128800F42303F59073C6F864340020F8BDFFF723
:10129800DDFE002840F08081D6F86434E21A002A86
:1012A80040F3008196F8702403F5D4531033032AD1
:1012B800C6F8643400F0DE80454B1978132900F035
:1012C8004481002A40F0D680D6F86C340133642B70
:1012D800C6F86C3440F2CE800123132986F8DC303E
:1012E80001D13C4A1380FFF779FD3B4B1B78032B58
:1012F80002D13A4B00221A8004F5F42404F59074C4
:10130800C6F864440020F8BD012028F09FFF00289B
:1013180040F0B7802E4B1A780123132A86F8DC3068
:10132800E1D1DEE796F944317D2B07DD284B1B78A8
:101338008222132B86F8442100F00281224CD6F831
:10134800402123689B1ADC2B00F20C81FFF77EFEFC
:1013580000283FF473AF2846FFF77CFB00283FF4D2
:101368006DAF00212846FFF733FB002800F0BE8050
:10137800AB7B03F07F03282B40F2B880144F6B78C7
:101388003A7886F89130132A08BF124A96F9443100
:10139800A97886F868344FF0340008BF938086F83F
:1013A800921010F007FF3A782368C6F84031132AE4
:1013B8004FF00C0386F8DC307FF440AF054A00207C
:1013C8001380F8BDF80F002098450020D8100020A1
:1013D8000427002008270020B2380020D838002031
:1013E800A34C642028F056FF2368D6F840219B1AA6
:1013F800B3F55C7F03D896F968747A2F64DD2368A7
:1014080096F84411C6F840310C2010F0CBFE342079
:1014180010F0D0FE974B1A780D23132A86F8DC308B
:101428007FF40CAFCAE7924F642028F033FF3B6883
:10143800D6F8402196F944419B1AB3F55C7F02D84F
:1014480014F17A0F57DA96F968341A1B022A1ADD52
:10145800884A2344117803EBD3735B100E221329B7
:1014680086F8933086F8DC207FF4E8AE824B0020C3
:101478001A80F8BD002486F87044FFF7AFFC2046B8
:10148800F8BD28F03BFFFFF7BFFC7A4B1B780B2217
:10149800132B86F8DC207FF4D1AE774B0B221A8011
:1014A8000020F8BD002028F0D1FE00283FF4C6AE89
:1014B800704B1B780022132B86F8DC207FF4BEAE1D
:1014C8006D4B00201880F8BDFFF7C0FD00283FF4E1
:1014D800B5AE2846FFF7BEFA00283FF4AFAE28465F
:1014E8000121FFF775FA002840F0B180342010F090
:1014F80061FE0020F8BDFFF7A9FD00283FF49EAE6D
:101508002846FFF7A7FA00283FF498AE284601219D
:10151800FFF75EFA0028E9D0564A3B681278C6F809
:101528004031132AA4F10403D9B208BF524A4BB27E
:1015380086F8443108BFD3800C2010F033FED5E77D
:101548004D4B4FF68272DA80F8E6B6F862344A48B4
:1015580001339BB2A6F862344380B2E6464A0120C2
:101568001380F8BD434A96F8441112782368C6F8E8
:101578004031132A01F11001C9B208BF3E4A4BB2EB
:101588004FF00C0086F8443108BFD38010F00AFEF3
:10159800342010F00FFED9E62846FFF75BFA002842
:1015A8003FF47AAE01212846FFF712FA00289DD0B1
:1015B8002B7B0022C6F86C241A0739D596F87024BC
:1015C80004F5FA7442F00202C6F8644486F87024FE
:1015D8005B073FF533AE0220F8BD2846FFF73AFA1D
:1015E80000283FF43EAE01212846FFF7F1F9002814
:1015F8003FF47CAF2B7B19077FF578AF0023C6F843
:101608006C3428F07BFE1B4B1A78132A08BF1A4A41
:101618004FF002034FF0030104F5FA7486F87014D2
:1016280086F8DC3008BF1380C6F864440020F8BD93
:1016380004F6AC543420C6F8644410F0BBFD96F8A8
:1016480070242B7B42F0010286F87024C0E7094A17
:1016580023681278C6F84031391DC9B24BB2132A33
:1016680086F868347FF468AF034A938064E700BF64
:101678009845002004270020082700202DE9F04184
:10168800B64E96F860340446052B00F2CC80DFE8AD
:1016980003F01722318BBE0396F89030002B00F030
:1016A8001F82502428F012FE2AF0B8F8631E13F0A7
:1016B800FF04F7D1062386F860340120BDE8F081E5
:1016C800A74BD6F85C241B689B1A0A2B00F24C81A6
:1016D8000020BDE8F081012028F0B8FD002840F086
:1016E800A88096F89000002840F0A380062386F88A
:1016F8006034EEE796F97834994AD6F874147D2B5D
:10170800C4BF822386F8783413685B1A322B00F240
:101718001681FFF79BFC0028DAD0FB20FFF786F93B
:1017280010F07F05D4D0294625442046FFF78AF9D2
:1017380015F8013C1A06CBD5A578012DC8D103F0C0
:101748007F03322BC4D996F8783486F89330362044
:1017580010F030FD96F84811232010F023FD96F87C
:101768004911242010F01EFD96F84A11252010F08A
:1017780019FD00210A2010F015FD3A2010F01AFD7D
:10178800142019F083FD342010F014FD00240523E3
:10179800284686F8793486F84641FFF735FC032356
:1017A800204686F8603494E7FFF750FC00288FD075
:1017B800FB20FFF73BF910F07F0589D02946254427
:1017C8002046FFF73FF915F9013C002B80DAA37892
:1017D800012B7FF47DAF607900287FF479AFE27840
:1017E800237986F891206FF0040186F89230091B5E
:1017F800621D04F10A058B18034412F8010F3344E3
:10180800AA4283F8940000F093806079F3E796F891
:101818007954782D47D9362010F0CCFC052386F86A
:101828006034002055E7D6F848344E49BDE8F04109
:10183800184728F063FD1421192010F0B3FC484A1A
:1018480082231946126886F878340C20C6F8742466
:1018580010F0A8FC0C21072010F0A4FC0821182087
:1018680010F0A0FC362010F0A5FC96F848112320B3
:1018780010F098FC96F84911242010F093FC96F883
:101888004A11252010F08EFC00210A2010F08AFC55
:101898003A2010F08FFC342010F08CFC022386F8DC
:1018A8006034002015E7FFF7D1FB00283FF410AFA4
:1018B800FB20FFF7BBF810F07F073FF409AF39466C
:1018C80027442046FFF7BEF817F9013C002BBFF666
:1018D800FFAEA378012B7FF4FBAEE27896F8913047
:1018E8009A427FF4F5AE227996F892309A427FF4C4
:1018F800EFAE6279AA427FF4EBAE04F1050E002345
:101908001EF801CF17F8038CF018E045D9B210443F
:1019180003F1010302D0BCF1000F02D12C2D00F21B
:101928003481052B80F894C000F033816279E7E7B1
:10193800237B86F8C630042386F86034C8E696F818
:1019480078341268C6F874240533DBB219460C20C3
:1019580086F8783410F026FCDBE600BFF80F00208C
:101968009845002058140020FFF7ECF901210220C7
:1019780010F018FC1821084610F014FC0421072068
:1019880010F010FCFF213E2010F00CFC00210C2070
:1019980010F008FC5C210D2010F004FC232113201A
:1019A80010F000FC7A21142010F0FCFB16211920FD
:1019B80010F0F8FB6C211A2010F0F4FB03211B2017
:1019C80010F0F0FB40211C2010F0ECFB91211D20B1
:1019D80010F0E8FB5621212010F0E4FB1021222012
:1019E80010F0E0FBA921232010F0DCFB0A212420C1
:1019F80010F0D8FB0021252010F0D4FB112126205F
:101A080010F0D0FB5921292010F0CCFB88212C2084
:101A180010F0C8FB31212D2010F0C4FB0B212E2023
:101A280010F0C0FB0721032010F0BCFB00210920A7
:101A380010F0B8FB96F84544092C7DD00F2C52D0F5
:101A4800082C27D10C21172010F0ACFB76210E2092
:101A580010F0A8FB27210F2010F0A4FB1921062065
:101A680010F0A0FB0521204610F09CFB21460B201E
:101A780010F098FBAA21102010F094FB39211120B6
:101A880010F090FB1121122010F08CFB4221152040
:101A980010F088FB414C0025362010F08BFBE9B292
:101AA8000A2010F07FFB332010F084FB4FF46170A4
:101AB80019F0ECFB2320FEF7B9FF20702420FEF775
:101AC800B5FF60702520FEF7B1FF0135FF2DA0702E
:101AD80004F10304E0D1012386F860340020F8E51E
:101AE80018F0AAFEE6E50E21172010F05BFB802116
:101AF8000E2010F057FB2046002110F053FB232145
:101B0800062010F04FFB0121082010F04BFB0821A4
:101B18000B2010F047FB7B21102010F043FBF8212D
:101B2800112010F03FFB0321122010F03BFB532142
:101B3800152010F037FBADE70C21172010F032FB11
:101B480076210E2010F02EFB27210F2010F02AFB03
:101B58001E21062010F026FB0121082010F022FB90
:101B68000A210B2010F01EFB7B21102010F01AFB1D
:101B78006121112010F016FB1321122010F012FB26
:101B88005121152010F00EFB84E70A4486F84621FF
:101B980041E6053586F8795400209AE54011002081
:101BA80038B50D4604463B2010F004FB2A46214672
:101BB80003482AF041FF3520BDE8384010F0FABA52
:101BC800544000202DE9F04F0B78063B83B00D46BA
:101BD8000746042B20D8DFE803F0A2230340700057
:101BE800BA4CFFF733FA20B194F88064002E00F065
:101BF800118194F88834002B40F0B78019F0F4FA7A
:101C0800D4F87C34D4F8581442F22832C01A02FBB3
:101C180001F28242C0F29680002003B0BDE8F08F46
:101C280019F0E2FAA94C00260822C4F87C0441F213
:101C3800B4432A703046C4F8843484F8806428F0A9
:101C480005FB0028CDD03223C4F87C64C4F8546462
:101C58002E703046C4F85834DFE79C4C19F0C4FAAB
:101C6800B4F84E24D4F88414D4F87C340A44C01A46
:101C78008242D1DC362010F09DFA2AF032FF3A2059
:101C880010F098FA1E2019F001FB362010F092FA95
:101C980094F8B4140131C9B204F2B440FFF780FFDC
:101CA80094F85034002B40F0FC8094F880340A22D9
:101CB8002A70002BB0D00220AFE7844E19F094FAB6
:101CC800D6F88424D6F87C3402F67462C01A8242AC
:101CD800A2DA19F089FA7E4FC6F87C0441F2B443BF
:101CE8007878C6F88434002486F88044FFF7B0F882
:101CF800342010F05FFAD6F85434642B00F2C68012
:101D0800744A1278122A08BF734A03F1010308BF04
:101D18005380C6F8543408232B7000207DE76B4BA2
:101D28002F22002083F84621FFF76EF907232B7036
:101D38000120FFF78DF8342010F03CFA002003B0A2
:101D4800BDE8F08F28F0C2FA644B1B78032B02D150
:101D5800634B00221A800120FFF77AF8342010F034
:101D680029FA07232B70002057E719F03DFAD4F819
:101D78007C34D4F88424C01A8242BFF63FAF0923CA
:101D88002B7094F8913084F8B53494F8922084F844
:101D9800B6240E2384F8B43494F8C814FB7884F875
:101DA800B734002940F0328194F8C720012A00F0A6
:101DB800DC81C0F0D181022A0CBF3222002284F8D3
:101DC800B8247A7D81F0010184F8C814110740F124
:101DD8008F808821002284F8B91484F8C9244148E6
:101DE800DFF808C100F10906002101E010F8013F01
:101DF80083EA11220CEB42028642B2F8603083EA91
:101E080001231BB299B2F1D1090A84F8C11484F8EC
:101E1800C234F3E6FB20FEF709FE94F84D8400F087
:101E28007F0080453FF6E5AE41463846FEF70AFE9C
:101E3800A8F1070313F0FF0307F1030200F0B281D2
:101E48000333DFF8A8C0F91812F8013B83EA162318
:101E58000CEB43038A42B3F8603083EA0626B6B235
:101E6800F2D1330A07EB080212F8041C994200F079
:101E7800D480184AD4F8F03412780133122AC4F8FE
:101E8800F0347FF4B6AE144A9380B2E632230122CE
:101E9800C6F85834072386F8884420463A702B70D1
:101EA800BBE6114AD4F8E8341268D31A0020182B7C
:101EB8008DF8070067D902AF012307F8013DC4F880
:101EC800E8243946002220F08DF8EEE6F80F0020CD
:101ED800000000200427002008270020B238002036
:101EE800D8380020AF14002098450020BC0D030806
:101EF800C2F3011112F0400240F03F81481C94F8EF
:101F0800C91400F0030081423FF469AF94F8A86453
:101F180094F8E43494F800E0BD4806F0F00661F364
:101F2800010684F8B96473455FFA82FC04EB030781
:101F380003F1010602F1010200F036813B7900F855
:101F4800013B052A06F03F03EDD184F8E4349446BA
:101F5800B04884F8BAC4074601EB41064A1C710030
:101F680057F812CD40F801C0564206F0030608445F
:101F780002F00302BF8894F8B734878058BF7242D2
:101F880084F8C9242BE794F8B094DFF8A88209F103
:101F9800010909F003094FEAC90A83460DF1070749
:101FA800AAEB0906264496F89234002B89D000281B
:101FB80087D196F88C2494F8EC34934202D313E03A
:101FC8000028EDD1F2183946002392F88D044246D4
:101FD80020F034FD94F8EC3496F88C240133DBB20D
:101FE800934284F8EC34EBD39A42D9D1AAEB090A8C
:101FF800A24409F1010384F8B09403F003098AF8B4
:1020080092B484F8ECB44FEAC90AC9E794F88C2072
:1020180062F07F0284F8B824D3E612F8033CF6B2E3
:10202800B3427FF426AF3B78A8F1030843457FF419
:1020380020AF7A7894F891309A427FF41AAFBA7840
:1020480094F892309A427FF414AF94F8C62022B1E3
:10205800BB7913B19A427FF40CAF00230122C4F874
:102068005434C4F88434C4F8582428F047F96A4A28
:102078001378A3B17B79387994F846119B00DBB2C9
:102088008842537006D301F13F068642C0F2B280FF
:10209800013353700121002384F88814137094F8D5
:1020A8004D343B443E4613F8020CFEF75BFC787D4A
:1020B8005A4956F8163F94F8A9C400F00300C0EB3B
:1020C800C0028B5011440CF10103B6888E80224463
:1020D80003F003030121DEB282F89214B0424FF0FC
:1020E800000284F8A8240DD03246C2EBC201214474
:1020F80002F1010E91F89214002958D00EF0030253
:102108009042F2D1C3EBC3022244002192F89224F8
:10211800C4F8AC1482B1B44503D10DE08C450BD0A2
:102128000E46013303F00303C3EBC3022244D9B2C2
:1021380092F89224002AF1D194F8A83484F8A9647A
:1021480066F3051384F8A83419F04EF80123C4F88F
:102158007C0484F880344CE5314A324812880532D0
:10216800A0FB0202C2F3C60229E62F482F4A007BD1
:1021780032F81020C2F3461221E62D4E94F8A82416
:1021880001EB410706F1120000EB470002F0F002F4
:1021980007688088C4F8BA7461F30102B08084F8D3
:1021A800B9241CE61E465DE684F8E434D0E694F8CB
:1021B800A8E4D4F8AC0462F3051E5FFA8EF242F08C
:1021C8004002013084F8A8245206C4F8AC0499D51A
:1021D8000428B9D9032384F8921484F8991484F84C
:1021E800A01484F8A714C4F8AC1484F8B03484F8A4
:1021F800A934A9E701F17F06B04202DC023353702B
:1022080048E7BF318842DCBF0333537042E700BF61
:10221800B3140020C41400200000002084140020FF
:10222800C02C0020CDCCCCCCDC46002004470020BC
:10223800B2140020750600082DE9F0410C4682B062
:10224800054618F0D1FF2378063B0746032B49D8EB
:10225800DFE803F04D2A023EB94EFEF7F7FE0028EC
:1022680059D10025D6F85814D6F8F43442F2283259
:1022780002FB01F2FF1ABA4249DA01296DD1D6F8F8
:102288005434642B03F1010200F29E800120C6F849
:102298005424FEF7DDFD34200FF08CFF0723284679
:1022A800237002B0BDE8F081A54E082323700020FA
:1022B800C6F8F47427F0CAFF0028CED000253223D0
:1022C800C6F8F454C6F854542570C6F858341EE0BD
:1022D8009B4D18F089FFD5F8F834C01A40F26353C3
:1022E800984258DC0025284602B0BDE8F081944B9E
:1022F8002F22002083F84621FEF786FE072323704D
:102308000120FEF7A5FD34200FF054FF00252846D4
:1023180002B0BDE8F081FB20FEF788FB00F07F00EB
:1023280013289ED914212846FEF78CFB95F9133003
:10233800002B96DA2B7800220120112BC6F85424A2
:10234800C6F858044CD0D6F8F42442F22833BF1A01
:102358009F42C7DD0122002598E727F0B7FF794B98
:102368001B78032B13D1784F784E3A78784836F893
:1023780012C00368511C01F00F0139700021A3EB52
:102388000C0326F81210734A03601B0913800D20F2
:10239800FEF75EFD7FE736200FF00CFF2AF0A1FB69
:1023A8003A200FF007FF36200FF004FF95F80015CC
:1023B800013105F5A060C9B2FFF7F2FB0823C5F8A3
:1023C800F47423700225A2E75E4B1B783221032B9D
:1023D800C6F858147FF45AAF5E4B0021198055E7B0
:1023E8006A7896F891309A42ADD1AA7896F89230E8
:1023F8009A42A8D1019027F081FF0198FEF728FDA5
:10240800A87CFEF7AFFAEB7803F00303022B08D0A1
:1024180034200FF0CFFE07232370C6F8F47402258A
:1024280020E718F0E1FE96F8C730C6F8F804012B4B
:102438002ED05FD3022B4849484A0CBF642300239F
:10244800497C287932F8111096F84C2496F8915066
:1024580086F80335090986F804154FF0110C96F82B
:102468009210B6F88C3086F8FC0486F800C586F819
:10247800015586F8021586F805358AB9134686F897
:10248800063596F8FC2486F8072509232370C4E747
:102498003149324A0B7B32F81330C3F30713CFE7C5
:1024A80096F8143596F84620834230D096F81535BC
:1024B80086F8163596F8161596F84600284D002227
:1024C80005E09EF848308CF808300A2A1BD001F144
:1024D8000108884206EB010E05EB020CD3B208F0A6
:1024E8003F0102F10102ECD1002286F8160586F8B8
:1024F8004620C4E71B4B18491B88184A0520B3FB24
:10250800F0F3DBB29CE786F816151346B7E70133FC
:1025180003F01F0396F8161586F8143586F8151576
:10252800002AC7D186F8162518F05EFE0E4B0F4A12
:102538001B68C31A9342BDDD20F0F6FABAE700BF64
:10254800F80F0020B2380020B3380020B43800203B
:10255800D4380020D8380020DC460020044700206A
:10256800F8140020C02C0020E032002047E80100C9
:10257800F0B5836983B0064613B11A689B88138542
:102588007069DFF8A0C08389C3244FF47A730627E3
:102598006D464FF6FF710CF1010C03E0013B9BB255
:1025A8008B421CD002899207F8D504734FF47A73D2
:1025B80002E0A3B28B4212D00289D20703F1FF34A2
:1025C800F7D5027BD2B20DB12A7001354FB1013F68
:1025D800FF24BCF1000FE5D09CF80040DBE71AF0BF
:1025E8006BFEB36913B11A689B8893619DF8050067
:1025F8009DF801509DF802109DF803409DF80420B5
:102608009DF8063041EA052143EA002342EA042204
:102618000120A6F85010A6F85220A6F8543003B0AE
:10262800F0BD00BF1C100308037B022B01D0002063
:102638007047F0B5436983B013B11A689B88138556
:102648000446006940F2E933828901E0002B5ED03C
:102658000289013B12F0020F9BB2F7D0BB23037330
:1026680040F2E93301E0002B51D00289013B12F01E
:10267800010F9BB2F7D0037B2069838903899907EF
:102688004FF005076E464FF47A724FF0FF0C4FF685
:10269800FF7506D4531E9BB2D2B11A460389990717
:1026A800F8D580F80CC04FF47A7302E08BB2AB42D5
:1026B8000ED00289D20703F1FF31F7D5027BD2B2DF
:1026C8000EB1327001367A1E27B117461A46E5E771
:1026D8001AF0F2FD636913B11A689B8893619DF83B
:1026E80004009DF800609DF801109DF802509DF8C7
:1026F80003209DF8053041EA062143EA002342EA17
:10270800052201206183A283E38303B0F0BD1AF0A0
:10271800D3FDB1E72DE9F04F87B00346029040683A
:102728009A68038823F040031B041B0C038003886A
:102738009BB223F0380343F038030380038843F047
:102748004003038012B1136892881A85838940F286
:10275800E93302E0002B00F082810289013B12F08C
:10276800020F9BB2F6D06B23037340F2E93302E009
:10277800002B00F074810289013B12F0010F9BB21B
:10278800F6D0037B029B586840F2E933828902E065
:10279800002B00F061810289013B12F0020F9BB20D
:1027A800F6D08023037340F2E93302E0002B00F0F7
:1027B80053810289013B12F0010F9BB2F6D0037BD3
:1027C800029B9B6813B11A689B8893610623A54CEA
:1027D800DFF89C82DFF89CA2A34DA44E04939623B5
:1027E800DFF894C201934FF0100EDAF80430C3F307
:1027F8000803002B40F0B480EFF31183002B40F066
:10280800AF802068AA6823689842FAD133689A4250
:10281800F7D8D8F800704FF47A7101FB07F39B1AC8
:10282800B3FBF7F301FB00304FF47A774FF001095F
:10283800DAF80430C3F30803002B72D1EFF31183E5
:10284800002B6ED12368A96822689342FAD13268B6
:102858009142F7D8D8F8002007FB02FBABEB010147
:10286800B1FBF2F107FB03131B1AB3F57A7FDFD331
:10287800019B013B0193B8D1029B9B6813B11A6875
:102888009B881385029B586840F2E933828902E0ED
:10289800002B00F087800289013B12F0020F9BB2E7
:1028A800F6D0F523037340F2E93301E0002B79D029
:1028B8000289013B12F0010F9BB2F7D0037B029B08
:1028C8005868838940F2E93301E0002B67D0028918
:1028D800013B12F0020F9BB2F7D0FF23037340F2C3
:1028E800E93301E0002B5AD00289013B12F0010FB5
:1028F8009BB2F7D0037BDBB20393029B9A6812B1B9
:10290800136891889961039B682B4ED0049B013B07
:1029180013F0FF0304937FF462AF184607B0BDE8D5
:10292800F08FEFF311818EF31288D5F808B02B6879
:10293800DB0344BFCCF80090D5F808B02368DCF876
:102948000020C9B281F31188D8F80010134407FB9E
:1029580001F2A2EB0B02B2FBF1F207FB032383E7C0
:10296800EFF311838EF31288AF682A68D20303D578
:102978000122CCF80020AF682068DCF80090DBB2B8
:1029880083F31188D8F800104FF47A72484402FB98
:1029980001F3DB1BB3FBF1F302FB003044E71AF051
:1029A8008BFCAAE71AF088FC89E712B113689288B1
:1029B8001A85029B586840F2E933828901E0002BAE
:1029C80047D00289013B12F0020F9BB2F7D08C234B
:1029D800037340F2E93301E0002B3AD00289013B4E
:1029E80012F0010F9BB2F7D0037B029B58688389D2
:1029F80040F2E9330289013B12F0020F9BB215D174
:102A0800002BF7D11AF058FC029B9B6813B11A6887
:102A18009B889361059B142B04D3182B17D9543B1F
:102A2800062B14D9002007B0BDE8F08FFF230373ED
:102A380040F2E93301E0002BE4D00289013B12F0B7
:102A4800010F9BB2F7D0037BDBB20593DCE70320D1
:102A580064E71AF031FCC8E71AF02EFCB0E61AF069
:102A68002BFC8FE69845002010E000E0A8450020E8
:102A7800A445002000ED00E0A04500202DE9F04F1E
:102A880090F8613087B00646002B40F05384D6E9B1
:102A98000502038823F040031B041B0C03800388F2
:102AA8009BB223F0380343F038030380038843F0D4
:102AB8004003038012B1136892881A85838940F213
:102AC800E93302E0002B00F02E860289013B12F068
:102AD800020F9BB2F6D06B23037340F2E93302E096
:102AE800002B00F020860289013B12F0010F9BB2F7
:102AF800F6D0037B706940F2E933828902E0002B4B
:102B080000F0FD860289013B12F0020F9BB2F6D05D
:102B18008023037340F2E93302E0002B00F0EF86D4
:102B28000289013B12F0010F9BB2F6D0037BB36917
:102B380013B11A689B8893619623AA4CAA4FDFF8B1
:102B4800B092AA4DDFF8AC820093019618F04CFBC6
:102B58004FF0100C4FF47A714FF0010ED9F8043091
:102B6800C3F30803002B40F0C383EFF31183002B5A
:102B780040F0BE832368AE6822689342FAD1D8F841
:102B880000209642F6D8D7F800A001FB0AF2921B63
:102B9800B2FBFAF201FB03231B1AB3F57A7FDDD3EC
:102BA800009B013B0093D1D1019EB36913B11A6810
:102BB8009B881385706940F2E933828902E0002B13
:102BC80000F099860289013B12F0020F9BB2F6D001
:102BD8006823037340F2E93302E0002B00F08B8690
:102BE8000289013B12F0010F9BB2F6D0037B70699A
:102BF80040F2E933828902E0002B00F078860289EE
:102C0800013B12F0020F9BB2F6D00323037340F28C
:102C1800E93302E0002B00F06A860289013B12F0DA
:102C2800010F9BB2F6D0037BB36913B11A689B8876
:102C380093619623DFF8B8916C4DDFF8B881009363
:102C4800019618F0D1FA4FF0100C4FF47A714FF04A
:102C5800010ED9F80430C3F30803002B40F0288391
:102C6800EFF31183002B40F023832368AE682268BA
:102C78009342FAD1D8F800209642F6D8D7F800A0A7
:102C880001FB0AF2921BB2FBFAF201FB03231B1AA7
:102C9800B3F57A7FDDD3009B013B0093D1D1019E30
:102CA800B36913B11A689B881385706940F2E933D8
:102CB800828902E0002B00F016860289013B12F09F
:102CC800020F9BB2F6D06B23037340F2E93302E0A4
:102CD800002B00F008860289013B12F0010F9BB21D
:102CE800F6D0037B706940F2E933828902E0002B59
:102CF80000F0F5850289013B12F0020F9BB2F6D075
:102D08000323037340F2E93302E0002B00F0E78568
:102D18000289013B12F0010F9BB2F6D0037BB36925
:102D280013B11A689B88936118F05EFA054618F08B
:102D38005BFA401B0E28FAD9B36913B11A689B884D
:102D48001385706940F2E933828902E0002B00F0B4
:102D5800C2850289013B12F0020F9BB2F6D06A23AA
:102D6800037340F2E93302E0002B00F0B4850289D6
:102D7800013B12F0010F9BB2F6D0037B706940F261
:102D8800E933828902E0002B00F0A1850289013B2A
:102D980012F0020F9BB2F6D01023037340F2E9330E
:102DA80002E0002B00F093850289013B12F0010F2D
:102DB8009BB2F6D0037BB36913B11A689B88936101
:102DC80018F012FA054618F00FFA401B0E28FAD927
:102DD800B36913B11A689B881385706940F2E933A7
:102DE80082890CE098450020A445002010E000E00E
:102DF80000ED00E0A8450020002B00F06485028962
:102E0800013B12F0020F9BB2F6D06C23037340F221
:102E1800E93302E0002B00F056850289013B12F0ED
:102E2800010F9BB2F6D0037B706940F2E9338289C7
:102E380002E0002B00F043850289013B12F0020FEB
:102E48009BB2F6D00023037340F2E93302E0002B73
:102E580000F035850289013B12F0010F9BB2F6D0D4
:102E6800037BB36913B11A689B88936118F0BCF9A6
:102E7800054618F0B9F9401B0E28FAD9B36996F837
:102E8800605013B11A689B881385706940F2E93362
:102E9800828902E0002B00F00E850289013B12F0C6
:102EA800020F9BB2F6D01923037340F2E93302E014
:102EB800002B00F000850289013B12F0010F9BB244
:102EC800F6D0037B706940F2E933828902E0002B77
:102ED80000F0ED840289013B12F0020F9BB2F6D09C
:102EE800057340F2E93302E0002B00F0E084028928
:102EF800013B12F0010F9BB2F6D0037BB36913B10B
:102F08001A689B88936118F06FF9054618F06CF9F8
:102F1800401B0E28FAD9B36913B11A689B88138528
:102F2800706940F2E933828902E0002B00F0BB842B
:102F38000289013B12F0020F9BB2F6D01B230373E8
:102F480040F2E93302E0002B00F0AD840289013B36
:102F580012F0010F9BB2F6D0037B706940F2E9339F
:102F6800828902E0002B00F09A840289013B12F06A
:102F7800020F9BB2F6D01823037340F2E93302E044
:102F8800002B00F08C840289013B12F0010F9BB2E8
:102F9800F6D0037BB36913B11A689B88936118F064
:102FA80023F9054618F020F9401B0E28FAD9B36911
:102FB80013B11A689B881385706940F2E9338289D6
:102FC80002E0002B00F067840289013B12F0020F37
:102FD8009BB2F6D01C23037340F2E93302E0002BC6
:102FE80000F059840289013B12F0010F9BB2F6D020
:102FF800037B706940F2E933828902E0002B00F01C
:1030080046840289013B12F0020F9BB2F6D01823C6
:10301800037340F2E93302E0002B00F038840289A0
:10302800013B12F0010F9BB2F6D0037BB36913B1D9
:103038001A689B88936118F0D7F8054618F0D4F8F9
:10304800401B0E28FAD9B36913B11A689B881385F7
:10305800706940F2E933828902E0002B00F01384A2
:103068000289013B12F0020F9BB2F6D0372303739B
:1030780040F2E93302E0002B00F005840289013BAD
:1030880012F0010F9BB2F6D0037B706940F2E9336E
:10309800828902E0002B00F0F3830289013B12F0E1
:1030A800020F9BB2F6D01023037340F2E93302E01B
:1030B800002B00F0E5830289013B12F0010F9BB25F
:1030C800F6D0037BB36913B11A689B88936118F033
:1030D8008BF8054618F088F8401B0E28FAD9B36912
:1030E80013B11A689B881385706940F2E9338289A5
:1030F80002E0002B00F0C1830289013B12F0020FAD
:103108009BB2F6D03823037340F2E93302E0002B78
:1031180000F0B3830289013B12F0010F9BB2F6D095
:10312800037B706940F2E933828902E0002B00F0EA
:10313800A1830289013B12F0020F9BB2F6D0012352
:10314800037340F2E93302E0002B00F09383028915
:10315800013B12F0010F9BB2F6D0037BB36913B1A8
:103168001A689B88936118F03FF8054618F03CF8F8
:10317800401B0E28FAD97269138823F040031B04F8
:103188001B0C1380138823F038031B041B0C1380BB
:10319800138843F04003138018F026F8054618F00A
:1031A80023F88542FBD07069038823F040031B0491
:1031B8001B0C038003889BB223F0380343F03803C9
:1031C8000380038843F04003038096F85B30032BA9
:1031D80000F2AE8096F85E50A5F10105B5FA85F5C6
:1031E8006D09B36913B11A689B881385838940F206
:1031F800E93302E0002B00F03A830289013B12F028
:10320800020F9BB2F6D01A23037340F2E93302E0AF
:10321800002B00F02C830289013B12F0010F9BB2B6
:10322800F6D0037B706940F2E933828902E0002B13
:1032380000F01A830289013B12F0020F9BB2F6D00C
:10324800057340F2E93302E0002B00F00D83028998
:10325800013B12F0010F9BB2F6D0037BB36913B1A7
:103268001A689B88936117F0BFFF054617F0BCFFEB
:103278008542FBD07069038823F040031B041B0CB4
:103288000380038823F038031B041B0C0380038886
:1032980043F040030380337C022B00F0D781B6F95A
:1032A80052305BB2013300F0178107B0BDE8F08FF0
:1032B800EFF311828CF31288D5F808A02B68DE038F
:1032C80004D5794BC3F800E0D5F808A0764E2368FA
:1032D800D6F800B0D2B282F311883E685B4401FB95
:1032E80006F2A2EB0A02B2FBF6F201FB0323CEE4DC
:1032F800EFF311828CF31288D5F808A02B68DB0352
:1033080004D5694BC3F800E0D5F808A0664E2368D9
:10331800D6F800B0D2B282F311883E685B4401FB54
:1033280006F2A2EB0A02B2FBF6F201FB032333E436
:10333800002556E71C09013C052C03F00F0300F299
:103348008F825A4A32F8140040FA03F2D50740F146
:1033580087824FF0010808FA03F3013B18402DF06B
:1033680003F9534BDFF864A113F8049081441AEB76
:10337800C90400F07582B4F804C04E4BBCFA8CF155
:103388002022C1F11F01A271481C4FF00002E27116
:10339800F3603FF47CAB5AF83900474A474DDFF8F1
:1033A80030E100F138439B0A6F18D25C97F86872D5
:1033B80002F01F03520906F10C0B022A08FA03F364
:1033C8004EF821B000F04782032A00F03F824245C0
:1033D80003D13B494A6913434B6104A94FF00008E4
:1033E800CDE904C81DF0DCFBA3885AF83910DFF8D2
:1033F800E4C0B3FA83F3C3F11F03D8B200F0FC02B0
:1034080002F1804202F5803200F0030080004FF0A4
:103418000F0E0EFA00F9D2F808E02EEA090EC2F8EB
:1034280008E0D2F80890C1F38721814041EA0901F8
:10343800916003F01F0E23F01F014FF0010909FAF4
:103448000EFE41F80CE0082204A804938DF815201C
:103458008DF814808DF8169028F00CFE194BDA5D63
:10346800F02A10D93D44F02195F878228DF80C20E7
:1034780003A803228DF80E808DF80F90D9558DF88A
:103488000D2028F0C5FCA388B3FA83F3C3F11F030A
:103498005A1C3FF4FCAA0C490122086802FA03F3FB
:1034A80003430B60FFF7F3BAA0450020844D0308DF
:1034B800BC4C0308810A00080C1C0308BC0D030857
:1034C800001002402425002000040140AC450020E3
:1034D800E42400201404014096F9503001337FF4AD
:1034E800E4AE0A23DFF8D0A2B04DB14E019328F024
:1034F800C7FF4FF4FA73DFF8CCE200934FF01008DF
:10350800DAF80430C3F30803002B40F07E81EFF3B0
:103518001183002B40F079812068AA6823689842BB
:10352800FAD133689A42F7D8D7F800C04FF47A71C5
:1035380001FB0CF39B1AB3FBFCF301FB00304FF4C7
:103548007A7C4FF00109DAF80430C3F30803002B42
:1035580040F00E81EFF31183002B40F009812368BE
:10356800A96822689342FAD132689142F7D83A683A
:103578000CFB02FBABEB0101B1FBF2F10CFB0313FB
:103588001B1AB3F57A7FDED3009B013B0093B7D1BA
:10359800072028F0E1FD4FF47A73DFF828E2009362
:1035A8004FF01008DAF80430C3F30803002B40F09A
:1035B8000B81EFF31183002B40F006812068AA6885
:1035C80023689842FAD133689A42F7D8D7F800C0EE
:1035D8004FF47A7101FB0CF39B1AB3FBFCF301FB6C
:1035E80000304FF47A7C4FF00109DAF80430C3F365
:1035F8000803002B40F09E80EFF31183002B40F06E
:1036080099802368A96822689342FAD13268914266
:10361800F7D83A680CFB02FBABEB0101B1FBF2F106
:103628000CFB03131B1AB3F57A7FDED3009B013B17
:103638000093B7D1019B013B01937FF458AF5D49DB
:103648005D4B5E485E4A0860DA602EE6B36913B1E6
:103658001A689B881385838940F2E93301E0002BBF
:1036680065D00289013B12F0020F9BB2F7D0C32349
:10367800037340F2E93301E0002B58D00289013B83
:1036880012F0010F9BB2F7D0037B7069838903891D
:103698009B074FF0050504AA4FF47A714FF0FF0E0F
:1036A8004FF6FF7C06D44B1E9BB2D9B1194603894D
:1036B8009B07F8D580F80CE04FF47A7302E08BB2E0
:1036C80063450FD0B0F8088018F0010F03F1FF31FF
:1036D800F5D0017BC9B20AB11170013225B1013DA3
:1036E8001946E4E719F0E8FDB36913B11A689B8835
:1036F80093619DF810209DF811109DF812509DF8C7
:1037080013309DF8140041EA02219DF81520A6F80F
:10371800501043EA05231BB242EA0022A6F85230B1
:10372800A6F85420BDE519F0C7FDFFF7E3B919F075
:10373800C3FDAAE7EFF3118188F31288D5F808B022
:103748002B68DB0344BFCEF80090D5F808B0236897
:10375800DEF80020C9B281F31188396813440CFBE4
:1037680001F2A2EB0B02B2FBF1F20CFB032359E7C7
:10377800EFF3118188F31288D5F808B02B68DB03C2
:1037880044BFCEF80090D5F808B02368DEF80020D2
:10379800C9B281F31188396813440CFB01F2A2EB1A
:1037A8000B02B2FBF1F20CFB0323E9E610E000E0A8
:1037B800A8450020FC9F002000ED00E0EFBEADDE34
:1037C8000400FA05A0450020EFF3118388F312885E
:1037D800D5F808C02A68D20304D50122CEF8002003
:1037E800D5F808C02068DEF80090DBB283F31188B2
:1037F80039684FF47A72484402FB01F3A3EB0C03D7
:10380800B3FBF1F302FB0030EBE6EFF3118388F32F
:103818001288D5F808C02A68D20304D50122CEF848
:103828000020D5F808C02068DEF80090DBB283F3EA
:10383800118839684FF47A72484402FB01F3A3EB0C
:103848000C03B3FBF1F302FB003078E62E4AD16992
:103858000B43D361C1E52C498A6913438B61BCE5ED
:103868002A4BF360002316E619F026FDF6E419F05A
:1038780023FDD7E419F020FD70E419F01DFD50E494
:1038880019F01AFD1EE419F017FDFFF7FEBB19F039
:1038980013FDFFF7CBBB19F00FFDFFF7AABB19F01B
:1038A8000BFDFFF777BB19F007FDFFF756BB19F0C3
:1038B80003FDFFF723BB19F0FFFCFFF703BB19F06B
:1038C800FBFCFFF7CEBA19F0F7FCFFF7ADBA19F019
:1038D800F3FCFFF770BA19F0EFFCFFF74FBA19F0D5
:1038E800EBFCFFF71CBA19F0E7FCFFF7FBB919F07E
:1038F800E3FCFFF799B919F0DFFCFFF778B919F085
:10390800DBFCFFF714B900BF00100240810A000871
:10391800F8B5304E304D32782B789A424FD12F4B34
:1039280093F800C0BCF1000F48D02D4A2D4B1078F9
:10393800002140F20D3E11E05C681F89676027682E
:1039480047F001072760A2F848E0D468013144F441
:1039580080748C45D46003F59A730FDD1A680028CB
:10396800EAD15062B3F83041D76801313C438C4505
:10397800D46003F59A7323F8040CEFDC31782B78C4
:1039880099421BD003EB83029200174FB858BE1818
:10399800A0B9327A92B9727A82B9013303F003037B
:1039A800D8B28142287009D003EB83039C003B19ED
:1039B8001A7217F019FC736803443B51F8BD0FF0F5
:1039C8005FFB0028FAD0054B93F800C0BCF1000F4C
:1039D800ABD1D3E75C1B00205D1B002064560020A0
:1039E8004053002068560020601B002020B100785A
:1039F800B0FA80F0400970470120704708B52021CF
:103A08002DF09CF90346184623B10278202A03F1C9
:103A18000103F8D008BD037903F01803082B0AD076
:103A280002D82BB100207047102B16D0182BF9D1D3
:103A3800B0F80B007047124BB0F80B0093F9003048
:103A4800591C06BF0F4B1B78DBB2C3EB0312C3EB49
:103A5800820300EB430080B270470B4BB0F80B00B9
:103A680093F900305A1C06BF064B5B78DBB203EBB8
:103A7800430203EB820300EB430080B2704700BFB0
:103A880031060020A463002030060020F0B5067936
:103A980006F06003402B09D144794FF0FF3500232D
:103AA800012006F00706A3420BD1F0BD602B08BF2A
:103AB80045794FF001040CBF04FA05F54FF0FF35C6
:103AC800EDE7042E0CD8DFE806F0030D18242E00CD
:103AD80030B1C85CD75C784028420CBF0120002078
:103AE8000133E0E70028FBD0C856D756A0EB070CF7
:103AF800DCF1000040EB0C00F2E70028F0D031F8D0
:103B0800130032F81370784028420CBF01200020BF
:103B1800E6E70028E4D031F9130032F91370C71B27
:103B280078427841DCE70028DAD051F8230052F8CF
:103B38002370784028420CBF01200020D0E7024BB8
:103B48000146186819F05CBD2C25002038B5064DD3
:103B5800441E14F8011F286819B9BDE8384019F047
:103B6800D5BC19F04DFDF4E72C2500200048EDE701
:103B78000F52030808B5FFF7E9FFBDE80840F5E76D
:103B880038B5074C074DAC4203D3074B00221A70D7
:103B980038BD6288D4E901012DF095F81434F2E7B4
:103BA800489A0308A89E03081C24002038B5074C2F
:103BB800074DAC4203D3074B01221A7038BD628807
:103BC800D4E901102DF07FF81434F2E7489A03087D
:103BD800A89E03081C240020024A136823EA000058
:103BE80010607047344E00202DE9F3410569064600
:103BF8000F467DBBD0F80080C8F30A0323B3002327
:103C0800D6F80080019328F070FF042819D1224CBF
:103C1800236943F001032361BBB2A8F8003028F000
:103C280064FF04282ED108F102030193019B3F0C85
:103C38001F8028F05AFF2369042823F00103236119
:103C480025D06FF0010505E028F04FFF042805D0C6
:103C58004FF0FF35284602B0BDE8F0810E4C2369CD
:103C680043F002032361C4F81480236943F040033E
:103C7800236128F03AFF2369042823F00203236113
:103C8800BDD0E5E7236923F001032361D9E7336851
:103C980004333360DEE700BF00200240F8B5044675
:103CA8000D468E180027B54201D12069F8BDE3689A
:103CB800591CE160234415F8012B1A720429F2D12A
:103CC800A1682046FFF790FFC4E90370EBE700BF47
:103CD80030B402681146531C036011F8024B0160AE
:103CE800D31C517803609378151D05601B0443EAC3
:103CF8000123D078234343EA006030BC704700BFFB
:103D08000368591C1A46016012F8021B02605878B1
:103D180041EA0020704700BF03685A1C0260187807
:103D2800704700BF38B50446006815462CF0CBFF35
:103D380022682A44226038BD03685A1C026010B405
:103D4800197003680A0A5C1C04601A7003680A0C7C
:103D58005C1C04601A700368090E5A1C0260197012
:103D68005DF8044B704700BF03685A1C0260197065
:103D78000368090A5A1C02601970704707EE901A06
:103D8800F8EE677A9FED837A27EE800A20EE070A1D
:103D9800FDEEC07A17EE903A2033402B00F2818076
:103DA800DFED7D7AB4EEE70AF1EE10FA40F3E68033
:103DB800B0EE407A9FED796ADFED796A01E0B0EE06
:103DC800677AB4EEE67AF1EE10FA77EE467AF6DC28
:103DD8009FED747AF4EEC77AF1EE10FA40F1D180D3
:103DE8009FED6E6ADFED706A01E0F0EE477AF4EE5F
:103DF800E67AF1EE10FA37EE867AF6D4DFED6B7AD2
:103E0800B4EEE77AF1EE10FA40F3A780DFED627ABC
:103E180037EEC77A27EE076ADFED655ADFED657A78
:103E2800DFED656A9FED655AE6EE257A67EE065A7C
:103E3800E6EE276AF7EE007AA5EEA67AF0EE675A64
:103E4800E7EE055AE7EE457A87EEA55ADFED577A91
:103E580030EE277AFDEEC76A16EE903A2033402BF3
:103E680024D99FED577AF6EE006AB7EE006AF7EEAE
:103E7800004AC4EEA57A0023836143610362C361EB
:103E880080ED045A67EEA66A27EE866A27EE877ADF
:103E9800C0ED006AC0ED026A80ED016A80ED037A28
:103EA8007047B7EE005AF0EE455ACFE7B4EEE70A8E
:103EB800F1EE10FA6BDD9FED396ADFED396A01E04A
:103EC800B0EE677AB4EEE67AF1EE10FA77EE467A5B
:103ED800F6DC9FED347AF4EEC77AF1EE10FA53D59A
:103EE8009FED2E6ADFED306A01E0F0EE477AF4EEDE
:103EF800E67AF1EE10FA37EE867AF6D4DFED2B7A11
:103F0800B4EEE77AF1EE10FA33DCDFED2E7AB4EE98
:103F1800E77AF1EE10FA44BFDFED227A37EEC77A7E
:103F280027EE076ADFED224ADFED226ADFED227A0B
:103F3800E6EE246A67EE064AE6EE267AB7EE006AEF
:103F4800A4EEA77AF6EE006A36EE476AF8EE007A33
:103F580027EE277A66EE266A89E7DFED1A7AB4EE4D
:103F6800E77AF1EE10FA44BFDFED0E7A37EEC77A42
:103F780050E7DFED097A37EEC77AD1E7F0EE407AFD
:103F880026E7B0EE677A39E7B0EE677AB6E7F0EE83
:103F9800477A9EE727D4D236DB0F4940DB0FC9406A
:103FA800E4CB1641DB0F49C0E4CB16C1DB0FC93F98
:103FB80092E741B99730083C15A82ABEF304353F6B
:103FC80000000000DB0FC9BFDFED2E7AB4EEE70A70
:103FD800F1EE10FA4ADDDFED2C6A9FED2C7A01E054
:103FE800B0EE670AB4EEC70AF1EE10FA70EE667A20
:103FF800F6DC9FED277AF4EEC77AF1EE10FA3ED59B
:10400800DFED216A9FED237A01E0F0EE407AF4EECD
:10401800C77AF1EE10FA37EEA60AF6D4DFED1E7A6B
:10402800B4EEE70AF1EE10FA14DDDFED167A37EE9A
:10403800C00A60EE006A9FED196A9FED197ADFEDFC
:10404800197AA6EE867A20EE266AE6EE877AA6EE3A
:10405800270A7047DFED147AB4EEE70AF1EE10FA9A
:1040680044BFDFED0B7A37EEC00AE2E79FED087A2E
:10407800F0EE407AF4EEC77AF1EE10FAC0D4B0EE62
:10408800670ACBE7DB0F4940DB0FC940E4CB164199
:10409800DB0F49C0E4CB16C1DB0FC93F92E741B93A
:1040A8009730083C15A82ABEDB0FC9BF02B370B40D
:1040B8008E1803E0121B14D1B14215D010F8012B51
:1040C800A2F14103192B11F8013BA3F1410598BF57
:1040D8002032192D03F12004ECD9D21A01D1002B7A
:1040E800EAD1104670BC70470022104670BC704779
:1040F8001046704770B5044608460D462BF028FF59
:10410800064602E014F8013F43B1324629462046EC
:10411800FFF7CCFF0028F5D1204670BD1C4620468D
:1041280070BD00BF4FF0FF32FFF7C0BFA0F16103C1
:10413800192B98BF20387047A0F14103192B98BF5D
:1041480020307047202805D0093804288CBF00206B
:104158000120704701207047613819288CBF002062
:1041680001207047413819288CBF00200120704772
:10417800303809288CBF002001207047A0F1300397
:10418800092B07D920F02000413819288CBF0020BE
:10419800012070470120704701212BF02FBE70B518
:1041A8000D461446FFF72AFC0646A0B1FFF7F4FFB8
:1041B80040F634039842A8BF1846B0F5617FB8BFEF
:1041C8004FF461701923A0F5617090FBF3F028702B
:1041D8002378013323703046FFF710FC0646A0B160
:1041E800FFF7DAFF40F634039842A8BF1846B0F547
:1041F800617FB8BF4FF461701923A0F5617090FB1F
:10420800F3F06870237801332370304670BD00BF27
:104218000378202B024600F10100F9D0092BF7D0D2
:104228002D2B00F0A4802B2B03BF5378B7EE000A88
:104238000246B7EE000AA3F13001C8B209289FED83
:10424800577A10D8F2EE046A07EE901AF8EEE77A79
:1042580012F8013FE7EE267AA3F13001C8B2092827
:10426800B0EE677AF0D92E2B63D003F0DF03452B2D
:1042780002D020EE070A704710B451782D294FD08C
:104288002B2979D0A1F13003092B02F101027AD848
:104298000024002303EB830301EB430312F8011FFF
:1042A800A1F130000928A3F13003F3D9B3F59A7FBF
:1042B8001A4628BF4FF49A72072B6CD9DFED386A7B
:1042C8001346F7EE007A083B072B67EEA67AFAD872
:1042D80002F00702DAB1F2EE046A012A67EEA67A62
:1042E80015D0022A67EEA67A11D0032A67EEA67ABD
:1042F8000DD0042A67EEA67A09D0052A67EEA67AB9
:1043080005D067EEA67A062A18BF67EEA67A002CB3
:104318003BD087EE277A5DF8044B20EE070A7047FA
:104328009178A1F13003092B02F1020230D801245F
:10433800AFE75378A3F13001C8B2092802F10102AE
:1043480093D8F2EE046AF0EE665A07EE901AF8EE89
:10435800E77A12F8013F87EEA66AA3F13001C8B2E6
:10436800092866EEA56A37EE067AEED97DE7537816
:10437800BFEE000A02465EE79178A1F13003092BEF
:1043880002F1020284D9F7EE007A27EE277AC2E713
:10439800F7EE007ABDE7F7EE007A9BE70000000031
:1043A80020BCBE4CF8B5064615460846B6FBF2F4E6
:1043B80034B905FB14640C4B1B5D00F8013BF8BDD8
:1043C800B4FBF2F75FB905FB1747074B05FB14640D
:1043D800DA5D00F8012B1B5D00F8013BF8BD38469B
:1043E800FFF7E0FFEFE700BFA0530308B5EEC00AF0
:1043F800DFED677A674AF1EE10FACCBF30EE270A94
:1044080030EE670ADFED647A20EE270A2DE9F047DF
:10441800FDEEC07A88B017EE904A84EAE47600236D
:10442800A6EBE476CDE902330493A2FB06325FEAF9
:10443800D208054641D105AF58483946554BA3FB2C
:104448000623DB0803EB8303A6EB4303002CC35CC2
:104458000B704FF00002ACBF20232D234A70384662
:104468008DF808302BF074FD0128394639D0022820
:1044780042D0032805BF302302A802A88DF80930CE
:104488002CF04DFC02A82BF063FD0338C4B2224681
:1044980002A928462CF079FC00232B5528462BF03E
:1044A80057FD2E22431C02A92A542144E8182CF057
:1044B80052FC284608B0BDE8F087394BA3FB062319
:1044C8005B0922D105AF35483946324AA2FB08328A
:1044D800D20802EB8202A8EB4202835C01F8013B9E
:1044E800ACE7302302A88DF809308DF80A308DF832
:1044F8000B302CF014FCC5E7302302A88DF80930E6
:104508008DF80A302CF00BFCBCE7264AA2FB0612F9
:104518005FEA92190ED105AF204839461D4AA2FB21
:1045280003C2D20802EB8202A3EB4203C35C01F888
:10453800013BCAE71C4AA2FB06125FEA523A0ED1B7
:1045480005AF16483946134AA2FB09C2D20802EB46
:104558008202A9EB4202825C01F8012BDEE71348D4
:10456800B6FBF0F058B905AF39460A20BAFBF0F2AD
:1045780000FB12A20948825C01F8012BE3E705AFB2
:1045880039460A220193FFF70DFF019B0146ECE72C
:104598006F12033ACDCCCCCC00007A44A053030868
:1045A8001F85EB51D34D62105917B7D1A086010072
:1045B8000F4B2DE93048D3E9004554EA05020AD1EA
:1045C800034640F2011200201880988098715A80A2
:1045D8001881BDE83088074B1A6814EB020B45F1C7
:1045E800000C5A466346FBF7A9FE0120BDE8308857
:1045F80038210020984500200A44914215D010B473
:104608000139541E11F8012F0823504010F0800F73
:104618004FEA400018BF80F0D500013BC0B2F5D189
:10462800A142EFD15DF8044B70477047484008231A
:1046380010F0800F4FEA400018BF80F0D500013B12
:10464800C0B2F5D1704700BF0A44914215D030B4CA
:104658000139551E41F2210211F8014F082380EA61
:10466800042004044CBF82EA40004000013B80B2B1
:10467800F7D18D42F0D130BC7047704770B5022237
:104688001349144C144E4FF6FF70FFF7DDFF2288D4
:104698004AB1A518B54218D2052A16D92146FFF7FE
:1046A800D3FF2C46F3E721460222FFF7CDFF022273
:1046B800A118FFF7C9FF094BE41A094B1C8041F602
:1046C8000F53C31A5842584170BD0020FCE700BF81
:1046D80000F0030802F0030800000408FAEF0308DA
:1046E8001E2400202DE9F043002489B006460D461B
:1046F8001F46A04605E025290CD030460134A847BE
:10470800039A531C039311780029F4D1204609B069
:10471800BDE8F083931CCDE903385078302842D0A7
:10472800A0F13003DBB2092B4FF0000945D96C2802
:104738002AD0642873D019D9732858D063D975281A
:1047480040F0828007F1040C386805AB00220A218A
:104758006746FBF7A7FD05AB049A009329464B462D
:104768003046FBF7A9FE039A0444CAE725283CD043
:1047780051D958286BD06328C2D139783046A84718
:1047880004370134039ABCE7039B5A1C03921B7835
:10479800642B52D016D8252B27D064D9582B18D083
:1047A800632BEAD0ADE7D31C03939078A0F13003D4
:1047B800DBB2092B4FF00109B9D804AA03A929F0E3
:1047C800ABFDB4E7732B12D051D9752B2DD0782BB4
:1047D80097D1A3F15802B2FA82F23868520905ABB0
:1047E80010210437FBF75EFDB5E7252185E73B6817
:1047F800049A0093294600233046FBF75DFE0437F0
:104808000444039A7DE76E287FF47AAF039A3B68E5
:1048180004371C6075E700283FF478AF70E7386804
:1048280005A9FBF709FD043795E7386805AB0022B1
:104838000A21FBF737FD04378DE73B1D386805A9CA
:104848001F46FBF7F9FC86E778287FF459AFA0F1FB
:104858005802B2FA82F23868520905AB1021FBF708
:1048680021FD043777E7002B3FF450AF49E76E2B63
:10487800CDD046E710B5064C0B46024605492068E0
:10488800FFF730FF2068BDE8104018F03FBE00BFBA
:104898002C2500205D0C000838B504460D46084854
:1048A800FFF754F929462046FFF7E4FF0548FFF7CC
:1048B8004DF9054B1B7813B1044B01221A7038BD12
:1048C800505103085B51030834250020352500208A
:1048D8000FB407B504A951F8040B0191FFF7DCFFE9
:1048E800FFF744F903B05DF804EB04B070470148E2
:1048F800EEE700BF5F5103080FB407B504A951F8EC
:10490800040B0191FFF7C8FF03B05DF804EB04B096
:1049180070470FB407B504A951F8040B0191FFF7CC
:10492800A9FFFFF723F903B05DF804EB04B0704763
:10493800F7B50646FFF75AF8054658B1002401A90D
:1049480020462AF053FB0134FFF7F2FF122CF6D170
:1049580003B0F0BD3046FFF71FFCC4B2112C5ED87F
:10496800701CFFF74BF8314D0746C0B9304B13F8B0
:1049780014108A1E514251412D4B13F81420AA5C81
:10498800002947D003EB440319205B7840F2EE215D
:1049980000FB031321462748FFF7BBFFD8E7017840
:1049A80028462CF0CBF960B1234B032C8CBF032293
:1049B8000022401B134453FA80F090F87F62032EC4
:1049C80002D1FFF794FFC3E73846FFF717F8F0B1B5
:1049D800022EF6D1FFF7E0FB40F6CA0280B2904201
:1049E800134BA8BF104640F2EE22904203EB44035B
:1049F800B8BF1046A0F2EE20192290FBF2F05870D2
:104A0800B31E594259410A4B03F81460B4E7022E09
:104A1800F6D1D6E721460948FFF77BFF98E711232F
:104A28002A4607490748FFF753FF91E7DC1E0308AA
:104A3800AC4000206B510308BC0D03087B510308F0
:104A480088510308905103080FB407B504A951F819
:104A5800040B0191FFF70EFF03B05DF804EB04B0FF
:104A680070472DE9F04F87B00346FEF7BFFF0646B3
:104A780020B1FFF73CFF07B0BDE8F08F05AA8249D7
:104A8800DFF84CB218462CF079F8B0468246344626
:104A9800B14635464FF0FF37BAF1000F27D17B48B2
:104AA8003946FFF7D1FF7A4B93F9062078B2824254
:104AB80000F0C78093F90E20824200F0C180002DDB
:104AC80014BFA8464FF46148002C08BF03240023F4
:104AD800E4B20293CDE900841A46194612F08CFA22
:104AE800074600283CD16B48FFF744F8C3E7B8F104
:104AF800030F07D8DFE808F0020F14245046FFF729
:104B08004BFB074605AA604900202CF037F808F14E
:104B180001088246C0E75046FFF73EFB0546F1E72D
:104B28005D495046FFF7E6FA08B144F001045946DA
:104B38005046FFF7DFFA0028E4D044F00204E1E72A
:104B480050462BF005FA554902465046FFF7AEFA93
:104B580020B15046FFF720FB8146D3E70126D1E775
:104B6800414675B94E48FFF76FFF4E48FFF702F808
:104B78004D4B186803681B6A33B13A464B4998474E
:104B880002E04B48FFF760FF4A4B4B494B48464C05
:104B9800002E18BF1946FFF7BCFE16B9B9F1000F71
:104BA80006D020680368DB6913B14A464449984730
:104BB8002468204612F006FA384612F003FA00215B
:104BC800084617F09BFB0021012017F097FB2046B1
:104BD80016F07AFDA0B10121002017F08FFB2046C6
:104BE80016F06AFD0546384616F06AFD0028FAD028
:104BF8002946384616F0CEFD0021084617F07EFB00
:104C0800384616F061FD0028E1D00121002017F098
:104C180075FB384616F050FD0546204616F050FD47
:104C28000028FAD02946204616F0B4FD002108468F
:104C380017F064FBCBE7B9682248FFF705FF0EE0E1
:104C480008331F68002F3FF43AAF002DF3D02946F0
:104C58001D48FFF7F9FE2946384613F077FA5CB18C
:104C68003979A14208D019482246FFF7EDFE3B6882
:104C7800E1B29B6938469847FB6A0BB10023FB6297
:104C8800002D81D171E700BF4B5C0308C2510308B6
:104C980094600020CB510308B6510308BC510308A7
:104CA800E05103086E5203083025002055810108A1
:104CB800FD510308A9510308115203089152030832
:104CC800C50B000835520308125203085052030856
:104CD800B95103082DE9F843037903F06002202A4B
:104CE80028D002D84AB1BDE8F883402A46D0602AC5
:104CF800F9D12548BDE8F8430BE603F00703022B7A
:104D080002D0042B08D06BB9B0F80720B0F8051012
:104D18001E48BDE8F843FCE5D0F805101C48BDE87E
:104D2800F843F6E5B0F90720B0F905101748BDE8D3
:104D3800F843EEE54579174E1748FEF707FF06EBEF
:104D4800C502002492F804800123A04503D8BDE8D9
:104D5800F843FEF70BBF56F8357057F824204FEA92
:104D680084094AB113B90D48FEF7F0FE57F8091047
:104D78000B48FFF769FE00230134E6E7417909484B
:104D8800BDE8F843C5E500BF06530308CA52030847
:104D9800B4520308741D0308E1520308F2520308D1
:104DA800A25F0308F55203082DE9F041174602797E
:104DB80002F06003402B05460C462BD10026524FCB
:104DC800DFF8648115E02B7903F00703022B15D077
:104DD800032B19D0012B14BFA15DA1573846FFF74B
:104DE80033FE6B79013BB34202DD4046FEF7AEFE6F
:104DF80001366B79B342E6DCBDE8F08134F8161071
:104E08003846FFF721FEECE734F916103846FFF76D
:104E18001BFEE6E702F00702042A67D8DFE802F083
:104E2800031E27292C002478202B3CD0602B49D046
:104E3800002BE1D1B5F80560B5F807803248214666
:104E4800FFF702FEA64249DCA04547DB002FD3D07E
:104E5800424631462D48BDE8F041F5E594F9004059
:104E6800202B20D0602B2DD0002BC5D146E02488E4
:104E7800DAE7B4F90040F3E72668202B344612D06D
:104E8800602B1FD0002BB7D131462148FFF7DCFD3E
:104E9800D5F805108E4221D8002FADD01D48BDE8A9
:104EA800F041D1E500246A791B4B03EBC201097973
:104EB800A14213DD53F8323053F82400BDE8F04125
:104EC800FEF744BE6A791441E30703D51348BDE8E9
:104ED800F041B9E51248BDE8F041B5E5FEF746FEF8
:104EE800224629680F48BDE8F04105E5202BD9D0B6
:104EF800602BEFD0002B7FF47FAF1C46B5F905601F
:104F0800B5F907809AE700BFDE5203082653030865
:104F1800C752030820530308741D03081B530308D2
:104F28002D530308315303081E5303080CB407B567
:104F380010F020000BD079B92320FEF700FE05A958
:104F480004980191FFF796FCFEF710FE012003B0CC
:104F58005DF804EB02B070470020F8E70CB4C30614
:104F680007B500D561B905A904980191FFF782FC3E
:104F7800FEF7FCFD012003B05DF804EB02B07047BA
:104F88000020F8E72DE9F04F89B002F11003DFF8AF
:104F9800BCA02D4EDFF8B8B00793814690460D4669
:104FA800144695F902309AF906209A4203D09AF9E4
:104FB8000E209A423CD1B8F1000F42D00822214677
:104FC80028462BF071FE627994F9023056F82220B7
:104FD8000492A27956F822200392227956F82220C8
:104FE8000292E27856F822200192B0FA80F72288DD
:104FF80000927F095A4639464846FFF797FF6A7973
:1050080095F9023056F822200492AA7956F82220FF
:1050180003922A7956F822200292EA7856F822203A
:1050280001922A88009239465A464846FFF796FF69
:10503800079B0834A34205F10805B2D109B0BDE8C1
:10504800F08F4746DBE700BF603803089460002014
:105058004B5303082DE9F04188B00346FEF7C6FC20
:10506800044630B146490022012008B0BDE8F041AD
:1050780088E7CDE9060018465E1C414DFFF78CF81D
:1050880095F9023040B2834276D095F90A308342CE
:1050980071D025463046FEF7B1FC074628B1FFF728
:1050A8007BF80134ADF81800E4B2DFF8D8800026A8
:1050B8003846FEF7A3FC074600B3FFF76DF8002259
:1050C80058F822108842D3B203D00132102AF7D1FF
:1050D800002358F82320904210D1022E1AD0032E14
:1050E8001DD05A1E012ED2B20FD00B2A03D88DF82C
:1050F8001B300134E4B20136042ED9D1052C14D862
:1051080008B0BDE8F041FFF7F2BB042AF3D88DF8E8
:105118001C30EEE7052BEED88DF81E30E9E79A1E15
:105128000D2AE8D88DF81D30E3E706AB03CB154A06
:1051380069609DF81D10286052F8211004919DF8AF
:105148001E109DF91A3052F8211003919DF81C1079
:1051580052F8211002919DF81B1052F8212001925B
:105168000021BDF8182000920846074AFFF7F6FE0E
:1051780008B0BDE8F08108358DF81A00012489E7E8
:10518800A4600020603803084B5303082DE9F04F52
:10519800DFF8DCA087B0814690460D46144600260D
:1051A800B8F1000F61D00622214628462BF07CFD7D
:1051B800B0FA80F720780EF0F9FE834660797F090F
:1051C8000EF0F4FEBBF1000F1DD09BF80810A2787A
:1051D80094F803B094F801C04FF4617E192313FBCF
:1051E80002E213FB0BE394F804E000B1007ACDE986
:1051F8000223CDE904E0CDE9001C33465246394686
:105208004846FFF793FE28780EF0D0FE834668796B
:105218000EF0CCFEBBF1000F1DD09BF80810AA7849
:1052280095F803B095F801C04FF4617E192313FB7C
:1052380002E213FB0BE395F804E000B1007ACDE934
:105248000223CDE904E0CDE9001C33465246394635
:105258004846FFF783FE0136142E05F1060504F1D2
:1052680006049DD107B0BDE8F08F4746CBE700BFE5
:10527800685303082DE9F04186B00746FEF7B6FBF0
:10528800044638B1002253490120FFF77FFF06B0DA
:10529800BDE8F0813846FEF77FFF1328054600F386
:1052A800918006264643781C8DF81740FEF7A6FB2A
:1052B800484C074660B1FEF76FFFC0B20EF05AFEC9
:1052C80030B10378A3559DF8173001338DF81730A6
:1052D8003846FEF793FB074660B1FEF75DFF0D28E1
:1052E80008D8062303FB054358709DF8173001338F
:1052F8008DF81730B11C0DF1170221443846FEF71E
:105308004EFFFEF77BFB074660B1FEF745FF01281D
:1053180008D8062303FB054318719DF8173001339D
:105328008DF817303846FEF769FB78B1FEF734FF81
:10533800C0B20EF01FFE48B1062303FB05430278F6
:105348005A719DF8173001338DF817309DF81720E2
:10535800042A4FF0060327D103FB054300221A71E4
:105368005A7104F0DFFE06236B43E618E05C0EF08A
:105378001DFEF278B778192380464FF4617470796E
:1053880013FB074713FB02440EF010FE017A7378F3
:1053980098F80820039131790F480097CDE9014129
:1053A8002946FFF7B6FA72E7052A04D103FB05433D
:1053B80000225A71D5E7062AD3D0A2190023A35197
:1053C8009380CEE71323224604490548FFF780FA65
:1053D8005DE700BF603F002068530308815303085E
:1053E800905103080EB400B584B005AB019053F892
:1053F800042B0649039301A8FFF774F9019B0022C7
:105408001A7004B05DF804EB03B07047B5040008E7
:105418002DE9F04F1E468DB007460B889246002AAC
:105428005ED115461446B3F5FA6F39D391F8028068
:1054380008F1FF320B2A33D891F803C00CF1FF3280
:105448001E2A2DD891F804E0BEF1170F28D891F83C
:105458000590B9F13B0F23D888793B2820D80A89D1
:10546800B2F57A7F1CD21A4643464FF001085EBB5C
:1054780009890491002CB4BF2D212B21002CB8BF21
:105488006442CDE90290CDE905140795CDE900CE37
:1054980038464449FFF7A6FF40460DB0BDE8F08FF7
:1054A80000234149ADF828304FF0010C18468DF81B
:1054B8002A30ADF82C3099469E461A4698460991EE
:1054C800634609A9002ED3D0CDE90290CDE900CEDC
:1054D80038463649FFF786FF40460DB0BDE8F08FE5
:1054E800A3F5FA638D7891F80380DFF8CC9091F8F2
:1054F80004E02F4C487991F806C003F0030202EB50
:105508004202013D05EB82059A0839F81590294DAC
:1055180008F1FF3340F2B55808FB02334B4403EB64
:1055280043030EEBC30384FB0A24C3EB03134FEAC4
:10553800EA7200EB830354446544C2EB6414C3EB82
:10554800031305EB8303B1F80880C4EB04154FF48B
:105558007A7BAAEB85054FF00009CBFB03892DB2B6
:10556800002D4FF47A724FF0000340464946B8BF09
:105578006D422AF0A9FF3C230AFB030A4FF47A7212
:105588000023404649462AF09FFF002392B2CBFBF6
:105598000A2309A8FAF7D2FE24B209A9BDF82430D3
:1055A80041E700BFE853030800000101C85303089E
:1055B8008988888880436D38BC0D030810B44C096D
:1055C800012250F8243001F01F0102FA01F123EA08
:1055D800010340F824305DF8044B704710B44C09BF
:1055E800012250F8243001F01F0102FA01F10B43A7
:1055F80040F824305DF8044B704700BF4B0901F0B8
:105608001F0150F82320012303FA01F1114214BFAE
:1056180018460020704700BF70B544880546C4F39B
:105628000B042246084600212BF071FB2969094A20
:105638009142034602D3084A914204D341B1184625
:10564800BDE8704008472246BDE870402BF03BBBE0
:1056580070BD00BFA89E0308F89F030838B5064C24
:10566800064DAC4206D2616820461434FFF7D4FFD9
:10567800AC42F8D338BD00BF489A0308A89E030877
:10568800084B09498B4203D309E014338B4206D2F5
:105698001A88C2F30B029042F7D1184670470023CC
:1056A80018467047489A0308A89E03082DE9F74F43
:1056B800DFF8C0B081468A460025D8462A4B0D241B
:1056C80018686C4317F022FF04EB0B031B7903F0F7
:1056D80018034B4504D0B9F1000F3ED1182B3CD12B
:1056E8000D2303FB05820093B2F80900FFF7C8FFFA
:1056F800444407462046FEF78EF9D7E901210646BD
:10570800024401442046FEF7C1F91AF0100F024680
:10571800009B00D008BB03FB05831AF0200F1B6811
:105728000FD072B91946114800930192FFF78CF90E
:105738007968019A31442046FFF736FBFEF716FADE
:10574800009B0B481946FFF77FF9B96800223144DE
:105758002046FFF729FBFEF709FA0135B5F5BB7FAF
:10576800ACD103B0BDE8F08F2C2500208753030887
:10577800885303089021030870B50546B0F809005E
:10578800FFF77EFF064B1E7804462846FEF743F9CE
:1057980016B1A368184470BD63681844FBE700BFDE
:1057A8001C24002038B505460C46FFF7E5FF2A798A
:1057B80002F0070302F06002602A28D1022B0ED003
:1057C800042B18D03BB96A7901239340DBB20278E5
:1057D80014B11343037038BD22EA0303FAE76A7968
:1057E800012393409BB2028814B113430380F2E76C
:1057F80022EA0303FAE76A79012303FA02F203684B
:1058080014B113430360E6E723EA0203FAE7042B23
:10581800E1D8DFE803F00303050507000470DAE7C1
:105828000480D8E70460D6E738B50D460446FFF78C
:10583800A3FF2A4601462046BDE83840FFF7B4BA20
:1058480008B5838940F2E93300E09BB10289013B46
:1058580012F0020F9BB2F8D0017340F2E93300E076
:1058680043B10289013B12F0010F9BB2F8D0007BD3
:10587800C0B208BD17F020FDC0B208BD38B5054C50
:105888000D4601466068FFF7DBFF29466068BDE802
:105898003840D5E794510020F8B584894FF6FF7653
:1058A8004FF47A742BB311B30F78013101E0B4428D
:1058B80017D00589013CAD07A4B2F8D507734FF49A
:1058C8007A7402E0BCB2B4420BD00589ED0704F14A
:1058D800FF37F7D5057BEDB20AB115700132013BF0
:1058E800E0E717F0E9FC003018BF0120F8BDFF27FA
:1058F800DFE70120F8BD00BF038823F04003B1F5BE
:10590800807F4FEA0343A8BF4FF480711B0C0380CC
:1059180002290388B8BF022191FAA1F20029B2FA3C
:1059280082F29BB208BF4FF0FF32013A23F03803EE
:1059380043EAC2039BB20380038843F04003038019
:10594800704700BF2DE9F843DFF8D080DFF8D0902A
:105958002E4E0421404617F089FCD8F8080016F0AE
:10596800B9FC00210520FFF789FF00210620FFF779
:1059780085FF99F80010042041F00101FFF77EFF30
:1059880033888BB1224F234D3C4615F8011FFF2960
:1059980008BF20210720FFF771FF2B7804F8013B8F
:1059A8003288E31B9A42F0DCFF210720FFF766FFED
:1059B80099F800100420FFF761FF3388DBB1164F18
:1059C800002403E033880134A34214DD17F8015B97
:1059D800FF2DF7D1C4F307210520FFF74FFFE1B2F0
:1059E8000620FFF74BFF29460720FFF747FF3388BC
:1059F8000134A342EADCD8F8080016F071FCD8F8A4
:105A080004000221BDE8F84376E700BFBC07002088
:105A1800CC2A0020C3280020C4280020945100204C
:105A2800F42F002070B5114BC1F1030141EA800049
:105A38009A78C5B2AA4218D00D4E9D7030460421FE
:105A480017F014FCB06816F045FC1024E0B22946A3
:105A58000134FFF713FF202CF8D1B06816F040FC92
:105A680070680221BDE8704046E770BD0000002064
:105A780094510020F8B5364C0421204617F0F6FB67
:105A8800A06816F027FC334B1B78012B56D045D362
:105A9800022B37D1304F08233B704FF4C3732F4E7E
:105AA8002F4D33800221FF230020AB70FFF7BAFF90
:105AB8000421274817F0DAFBA06816F00BFC3978A8
:105AC8000020FFF7DBFE274B02201978FFF7D6FEF0
:105AD800254B03201978FFF7D1FE244B19780420B1
:105AE8000143FFF7CBFEA06816F0FAFB60680221BD
:105AF800FFF702FF32881E4800212BF008F9EB78E7
:105B08003BB9F8BD144F3B785B06C6D54FF4F0732C
:105B1800C5E7FFF717FF0023EB70F8BD0021A020B1
:105B2800FFF7ACFE00F00603022B0B4F03D000F08A
:105B38000500012808D008233B70AEE7064F48232C
:105B48003B704FF4F073AAE748233B70DEE700BFD1
:105B580094510020D0510020C8070020BC07002025
:105B680000000020D7510020D8510020F42F002039
:105B7800CC2A00202DE9F047404C414D414E0421EC
:105B8800204617F073FBA06816F0A4FB00218020C4
:105B9800FFF774FE0746A06816F0A2FB60680221B2
:105BA800FFF7AAFE2B78D6F80080BB420DD1364B02
:105BB8001F7847B9DFF8D890D9F81835A8EB030350
:105BC800B3F57A7F04D8BDE8F087BDE8F04751E720
:105BD8000421204617F04AFBA068DFF8B8A016F0A9
:105BE80079FB3946A020FFF749FE0746A06816F062
:105BF80077FB60680221FFF77FFE9AF80030192BC7
:105C08000CD12B78214A03F04003002B07F0070141
:105C18000CBF0D20102013805180D080790706D545
:105C28000023C9F81C35C9F81885BDE8F08707F0C6
:105C38000507012F1AD0002FF5D12B785B06F2D576
:105C4800D9F81C35B3B13268D31A642BEBD9FFF7F6
:105C580011FF9AF80030192BE5D1B9F820350B4A15
:105C680001339BB2A9F820359380DCE72B785A06DC
:105C7800E6D5D8E73368C9F81C35D4E79451002035
:105C8800C807002098450020D05100200827002090
:105C9800F80F002004270020074A0023516881429A
:105CA80002F11C0204D001330C2BF7D100207047FD
:105CB800581CC0B2704700BF3406002000F1FF3CFA
:105CC8004FEACC002DE9F043A0EB0C04A400374FB9
:105CD800DFF8FCE03E59364DDEF81490DFF8F4802A
:105CE8003C44AE420CBF01260226656846EA090616
:105CF8004545CEF8146083B0A16023613ED02D4B9A
:105D08009D423DD014339D423CD014339D4232D045
:105D180014339D4239D014339D4239D014339D42F7
:105D280039D003F562739D423AD014339D4239D07D
:105D380014339D4232D014339D4235D01E491F4B37
:105D48008D420CBF1D460025A0EB0C0007EB800020
:105D58009209447B85610021012301A88DF8044044
:105D68008DF805208DF806108DF8073026F050F8CC
:105D780003B0BDE8F0834FF40055E5E70225E3E7FB
:105D88002025E1E74FF40075DEE74FF40035DBE747
:105D98004FF40015D8E74FF00075D5E7084DD3E765
:105DA800084DD1E7084DCFE7084DCDE73406002070
:105DB800000002401C00024058040240000002108B
:105DC8000002001002000010200000100020001047
:105DD80000100240080002400138C0EBC000094B27
:105DE8008000F0B4084D1C58084F6E691844BC4236
:105DF8000CBF0123022333436B6101754275F0BC6C
:105E0800704700BF34060020001002400000024026
:105E18002DE9F04F544C54F8204083B0002C5FD04B
:105E2800E56DA1601F469046504B6A686265236025
:105E380004F1620204F1E2036261A36180224FF47B
:105E48008073C4E903238146287E25F013FEE868A1
:105E580060B1FFF721FF09F10102D2B20C21FFF76F
:105E6800BBFF636DEA68A26324332365A86898B111
:105E7800FFF712FF09F101020646D2B20B21FFF724
:105E8800ABFF2346EA7E3A493046FFF717FF636DBA
:105E9800AA68E2632833E36494F8610015F038FED9
:105EA800064694F8600015F033FE3A07824695F8E6
:105EB80019B019D5C6B117F0110F4FF00B0309F13E
:105EC8000100F07114BF4E213E21B3715A4630468D
:105ED80015F0E4FEFB0743D5A36B6BB3E36B5BB331
:105EE800204603B0BDE8F08F17F0010F0CBF2E2736
:105EF8004E2718F0020F0AD04EB10B2209F1010308
:105F0800B271F37130465A46394615F0C7FE18F09B
:105F1800010FE1D0BAF1000FDED00C2309F1010026
:105F28008AF807008AF806305A463946504615F06E
:105F3800B5FEA36B002BD1D12B7FAA7E8DF8042050
:105F48009B090021012201A88DF805308DF8061063
:105F58008DF8072025F05CFF204603B0BDE8F08FE0
:105F6800304616F0B7F9B7E7942300204410030829
:105F7800E90A00080348D0F83C3113B100F59A70DB
:105F880018477047340600200348D0F8203113B171
:105F980000F58C7018477047340600200348D0F885
:105FA80004310BB1FC301847704700BF340600209D
:105FB8000348D0F8E8300BB1E0301847704700BF0D
:105FC800340600200348D0F8CC300BB1C430184751
:105FD800704700BF340600200348D0F8B0300BB13A
:105FE800A8301847704700BF340600200348D0F88F
:105FF80094300BB18C301847704700BF340600202E
:106008000248836F0BB17030184770473406002080
:106018000248C36D0BB1543018477047340600204E
:106028000248036C0BB1383018477047340600201B
:106038000248436A0BB11C301847704734060020E9
:106048000248836803B11847704700BF3406002030
:106058002DE9F8430501744C63596119002B00F0D0
:106068009A80724A6719934204BF01230B7306464C
:10607800387A25F0FFFC3B7A03F01F015B09012207
:10608800022B02FA01F200F0A880032B00F0A08096
:10609800012B03D1664B996A0A439A626319013648
:1060A800187915F035FDF6B2074610B11223C671FE
:1060B80083716319587915F02BFD10B11323C6713C
:1060C80083716319987915F023FD10B11423C671F3
:1060D800837166190E21F279384615F0DFFD707963
:1060E80015F016FDF2790E2115F0D8FDB07915F0EE
:1060F8000FFDF2790E2115F0D1FD63594D4A9342F7
:1061080070D04A4A934200F083804B4A934274D03D
:106118002C44227B002A40D000252E469988474AE5
:1061280021F480510904090C958156819980B3F8AE
:1061380004E0D788B2F808C0B2F80E90B2F8108020
:10614800508A94884EF4805EB7F5827FA3F804E005
:1061580026D0998821F470610904090C4CEA0101E0
:1061680099802743198849EA070448EA040401F496
:10617800415120430843304345EA00011980998B77
:10618800908A21F400621204120C9A8318821A88E9
:1061980042F040021A80BDE8F88301250226BDE7D7
:1061A80044EA0904198844F4827448EA040404435C
:1061B80001F44150044346EA0400284318809988B2
:1061C80021F470610904090C4CEA01019980D6E7B1
:1061D800174B19690A431A6160E7154BD9680A43D6
:1061E800DA605BE702F56042D16841F48051D16022
:1061F800D16821F48051D1608AE702F5EA32116949
:1062080041F400411161116921F4004111617FE7F6
:1062180002F5EC32116941F480411161116921F4F0
:106228008041116174E700BFA05100200038004090
:106238000010024000300140003C004000000020F7
:106248001749184B184A194810B4D1F8884044F433
:106258007004C1F888401C6844F001041C605C6844
:1062680022405A601A6822F0847222F480321A603E
:106278001A6822F480221A605A6822F4FE025A60D0
:10628800DA6A22F00F02DA621A6B002410404FF02B
:10629800006218639C608A605DF8044B704700BF19
:1062A80000ED00E0001002400CC07FF8CCFC00FFBD
:1062B80030B4134B1B78012B18D040F22E414FF409
:1062C800F07201234182028083700E4B0E494361B4
:1062D80040F22625012426220E2305824471C0F8A7
:1062E8000710C0F80B20037630BC70474FF47A745F
:1062F8004FF47A5104220371448201808270E4E7EA
:10630800A8150020D007E80328291312AD4AB2F9CE
:106318000030002BB8BF5B42B3F5E17F07DAB2F972
:106328000230002BB8BF5B42B3F5E17F01DB0020F0
:106338007047A54B93ED096AD3ED076AD3ED057A4B
:1063480093ED037A76EE866A37EE277A76EEA66ABA
:10635800F7EE007A37EEE66A37EE077AB0EEC66AED
:10636800F0EEC75AB4EEE56AF1EE10FAB4BFB0EE3B
:10637800655AB0EE465AB5EE405AF1EE10FA00F002
:10638800B280B4EEE56AF1EE10FA8CBFB0EE654A61
:10639800B0EE464AC4EE054A9FED8C2A9FED8C5A12
:1063A800DFED8C1ADFED8C2A9FED8C3ADFED8C3A0D
:1063B8009FED8C4AA4EE825AE4EEE12AE4EE857A57
:1063C800A4EEA23AB0EE675AF0EE637AE4EE837A6E
:1063D800A4EEA74AC4EE057AB4EEE56AF1EE10FA27
:1063E80044BF9FED816A76EE677AB7EE006AF4EEF5
:1063F800C66AF1EE10FAC8BFDFED7C6AB5EEC07A66
:10640800C8BF76EEE77AF1EE10FA48BFF1EE677A88
:10641800BEEE007A67EE877A9FED737A77EE876A29
:10642800BDEEE66A16EE102A2032402A61D9DFED69
:10643800706AC3ED0A6AFDEEE76A9FED6D7A16EEA3
:10644800902A2032402A83ED0B7A83ED0C7A4DD8BE
:106458009FED667AF4EEC77AF1EE10FA40F3A88061
:106468009FED646ADFED646A01E0F0EE477AF4EECE
:10647800E67AF1EE10FA37EEC67AF6DCDFED5F7AEF
:10648800B4EEE77AF1EE10FA40F18F809FED596A89
:10649800DFED5B6A01E0B0EE677AB4EEE67AF1EE22
:1064A80010FA77EE067AF6D49FED4F7AF4EEC77AB3
:1064B800F1EE10FA68DD9FED4D7A77EE677A27EEF8
:1064C800A76ADFED505ADFED506A9FED507AE6EE8D
:1064D800256A67EE865AA6EE267AE5EE877A0120C7
:1064E800C3ED0D7A7047DFED3F7A75E7F0EE477A36
:1064F800F5E7F4EEC77AF1EE10FA5FDDDFED3D5A0D
:106508009FED3D6A01E0F0EE476AF4EEC66AF1EEEF
:1065180010FA36EEE57AF6DCDFED386AB4EEE67AA4
:10652800F1EE10FA47D5DFED335A9FED356A01E0F9
:10653800B0EE667AB4EEC67AF1EE10FA77EE256A16
:10654800F6D49FED297AF4EEC76AF1EE10FA27DC4B
:106558009FED2F7AF4EEC76AF1EE10FA44BF9FED73
:10656800277A77EE666A66EEA65A9FED265A9FED61
:10657800266A9FED267AA5EE856A26EEA55AA5EE2F
:10658800867AE5EE076A54E79FED217AF4EEC77A3A
:10659800F1EE10FA44BF9FED197A77EE677A8EE72D
:1065A8009FED127A77EE666ADDE7F0EE477A7BE7D1
:1065B800B0EE677A62E7F0EE476AC2E7B0EE667A55
:1065C800AAE700BFB02800202C00002099FB243F38
:1065D80069A2163E39094E3DE3B59E3E88FA163E3D
:1065E80045FE7F3FA7DFA834DB0FC93FDB0F4940DB
:1065F80000000000DB0FC940E4CB1641DB0F49C0A7
:10660800E4CB16C192E741B99730083C15A82ABED9
:10661800DB0FC9BF10B40A784C78A24215D20430F7
:10662800104B33F9101040F633039942A8BF1946AE
:10663800B1F5617F4FF0190340F28330B8BF4FF4D2
:10664800617113FB02028A4203DB00205DF8044BF0
:10665800704713FB04008842B4BF002001205DF896
:10666800044B7047243300202C4B1B681844837953
:106678009BB107EE903ADFED2A6AF8EEE77A20EE52
:10668800A07A67EEA67A27EE207AF7EE006AD7EEB0
:10669800877A77EEA67A20EE270AC378DFED206A9C
:1066A80007EE903AF8EEE77AB0EE007A67EEA67A4F
:1066B800F4EEC77AF1EE10FA05DD37EEC77ADFEDB2
:1066C800196AE7EE267A437A9FED177A20EE070AD1
:1066D80020EE270A03B3DFED127A9FED147A06EE57
:1066E800903A60EEA77AF8EEE60A60EEA70AF4EEB2
:1066F800C70AF1EE10FA04DDDFED0D7A20EE270A65
:106708007047F5EEC00AF1EE10FA05D4F7EE007AFC
:1067180077EEE00A80EE200A704700BFC4320020FE
:106728000AD7233CD7A3684100004843A4707D3FA3
:106738000000C842174B9FED185A1B681844BFEE5B
:10674800007A437A06EE103AC378A0EE007A07EE94
:10675800903A8379B8EE466A05EE903A60EE850A7B
:10676800F7EE006AF2EE044AB0EE664A20EE240A1A
:10677800A6EE204A27EE057AF8EEE55AF8EEE77A13
:10678800E5EE876A67EE807A24EE270A20EE260A6D
:10679800704700BFC43200200AD7233C084AD37A86
:1067A800022B09D00748084B9188B0F91220D980EC
:1067B8001A805A809A8070474FF4006012F08ABDA0
:1067C800A8150020646100202433002010B50B4C6C
:1067D800012202234FF48060E27084F8203012F026
:1067E80079FD074A074B1168587A2388642212FBFF
:1067F800001201336261238010BD00BFE02C00202D
:1068080098450020A8150020F0B45D4E5D48327B05
:106818005D4B5E4DDC6B2D780132A0FB02700009E8
:1068280000EB8000A2EB80001A683073914201EB04
:1068380004005C6811D293F84520002A4ED000F578
:106848008030B0FBF5F084420BD2041B4FF4803249
:1068580092FBF5F2A21A9A600AE0B0FBF5F08442C6
:1068680044D34FF4803292FBF5F2121B02449A6033
:1068780040F68C240025A242C3E9001083F8455055
:1068880017D993F8402093F942108A4256B241D062
:10689800002093F9411083F843008A4247D0012130
:1068A800002283F8426083F8441083F84020F0BC4B
:1068B800704793F844100029F9D0A2F2EF2040F273
:1068C800DA5188421AD893F840100B2916D803EBEE
:1068D80081000131C26083F84010E8E7B0FBF5F0B1
:1068E8008442BED2041BA21A9A60C1E793F84520DD
:1068F800002AAAD1041BA21A9A60B9E7244A0021E7
:1069080002F1300083F8441042F8041F8242FBD1A0
:10691800F0BC7047111F0829BAD893F843101829FA
:1069280026D8013183F8431093F94110B5E793F85D
:1069380044100029B3D0FAB11649154C0FFA82FC5D
:10694800084601EB4C0754F8045F20F8025BB84294
:10695800F9D10B2A07DC104801EB4C02002122F880
:10696800021B9042FBD10D490A7801320A7096E762
:1069780083F84160314690E794460649EBE700BF4B
:10698800A8150020CDCCCCCC0C520020F20F002052
:106998001452002060390020783900205039002036
:1069A80030B40E4D0E4B2A7B0E4C0132A3FB020372
:1069B8001B09E06B03EB8303A2EB83034FF6FF7223
:1069C800914200F101002B73084408BF0123E063E2
:1069D80008BF84F8453030BC704700BFA8150020B8
:1069E800CDCCCCCC0C5200202DE9F04FC84BC94C73
:1069F8001B68C94A2DED0E8B1D7EC84BD4ED049A39
:106A08001B8812788BB0002DB7EE009A40F603056C
:106A18000390019108BFB0EE699A03F40060C3F3D4
:106A2800C0212B40009200F0A381A369002B40F005
:106A3800C884019BA36101230293B94A237F21756E
:106A48001178002B00F09D81B64B2C29D3ED008ADC
:106A580000F0F584DFF80893D4ED0A6AD9ED007ADE
:106A6800B7EE007AF4EEC76AF1EE10FA68EEA78A7C
:106A780017DDD4ED0B7A9FEDAC6A77EE677A67EE97
:106A8800A67AF4EEC77AF1EE10FA88BFF0EE477AEC
:106A9800F4EEC67AF1EE10FAB8BFF0EE467A68EE78
:106AA800A78ADFF8C0B2DFF8C0A20BF170080BF1BB
:106AB800E00707AE00250BEB0500D4F89C30BAECD4
:106AC800010A984708EB0500D4F80C319847781963
:106AD800D4F87C31984724356C2DA6EC010AEAD10C
:106AE80094F88031002B00F0BE84904ADFED906A64
:106AF800D9ED007ADFF83C82D2ED015AD8ED0B4A85
:106B080098ED067A92ED026A98ED015A92ED034AE1
:106B180067EEA67AF0EE646A67EEA55A27EE866AF3
:106B2800E7EE656AA4EEA57AF0EE455AE6EE665AF7
:106B380067EE847AE5EE066AB0EE656AA7EE876AC4
:106B4800A7EEE57AC8ED0B6A88ED016A88ED067A4A
:106B58000026DFF81892774D9FED77AADFED77CA08
:106B68009FED71CA9FED76BADFED76AADDF800A039
:106B780000923746744B3344D3ED007A734BF5EEED
:106B8800407A03EB060BF1EE10FADBED00DA17D0D2
:106B98001833334493ED007A7DEEC76AB0EEE66AA7
:106BA800F4EEC67AF1EE10FA08D5F5EEC06AF1EE09
:106BB80010FACCBF77EE87DA77EE67DAC3ED00DA42
:106BC800029B002B3ED0022F00F05986039A604B9F
:106BD80092F82D20334407EE902A93ED007A534221
:106BE800F8EEE76A07EE903A26EE877AF8EEE77A4B
:106BF800B4EEE77AF1EE10FA0AD407EE902AF8EE2E
:106C0800677AF4EEC77AF1EE10FA88BFF0EE477AA9
:106C1800504A424B5049188831F9173002EB470265
:106C2800B2F90A209B1A07EE103A40F60103B8EEB3
:106C3800C77A0342E7EE6C7A00F0B682D4ED79DACF
:106C480067EEADDABAF1010F00F02C82009A94F8E1
:106C58000932324492ED01DA3DEECD8AB0EE48EACF
:106C6800002B00F0B480D4F80C320199D4F810222B
:106C7800CB1A934240F36682039A92F84E20022A76
:106C880000F05F85022FD4F8140240F0FA82D4EDA8
:106C9800867AB1EE678AB4EEC8EAF1EE10FA08D443
:106CA800B4EEE7EAF1EE10FA8CBFB0EE678AB0EE08
:106CB8004E8A834285ED01CA40F30583274B1B6842
:106CC800980740F1F8842449224AB1F90030B2F912
:106CD8000AC0D4F82002A3EB0C03002BB8BF5B4218
:106CE800834280F2FA82B1F90230B2F90C209B1A81
:106CF800002BB8BF5B42984240F3EF82002318464E
:106D080084F8093216F01CF9D5ED016AE7E200BFF4
:106D1800C4320020A8150020C0300020482D0020D3
:106D280004270020C0070020000000009C47002026
:106D380035FA8E3CC43E002000004843CDCCCC3D03
:106D4800AE47813F0000C842681700205C1700204A
:106D580080170020C8300020B0280020C430002050
:106D680094610020D8150020A04700202C1700208F
:106D7800A3610293DC4A237F21751178002B7FF4ED
:106D880063AE637F002B3FF45FAED4ED086AA38C3B
:106D9800DFEDD67AD648B0EEE67AA3F57A7327EE19
:106DA800277A07EE903AF8EEE77AF7EE008AE7EEF0
:106DB800878A2C29C0ED008A7FF44CAE9FEDCD0A5E
:106DC800CD4D26EE800A29F023FF688038E3D5ED03
:106DD800016A99ED000ABAF1010F69EE00BA40F0B4
:106DE8008B8268EE2BBA022FC5ED00BAB0EE48EAE6
:106DF80000F09584D4ED957A94ED967A27EE888AFA
:106E0800F1EE477AE8EE286AF4EEE76AF1EE10FA56
:106E180008D4F4EEC76AF1EE10FA8CBFF0EE477AA8
:106E2800F0EE667AB54BC5ED017A9A19B44B92ED3E
:106E3800008A1B78C2ED00DABB423DEEC88A00F03A
:106E48002381B04A12789AB3AF4A1278012A00F027
:106E58009B81022A29D1AD4906EBC6020A4492ED6C
:106E6800027AD2ED067A92ED056AD2ED014AD2EDA8
:106E7800076A92ED035AD2ED045A82ED066A67EE6C
:106E8800277A92ED007A82ED058AE4EE867A92ED11
:106E9800086AC2ED086AE5EE667AE5EEC67AE8EEBB
:106EA800077AB0EE678AC2ED077ABB4200F06081CC
:106EB80099ED02DA07ABB5EEC0DA3344F1EE10FA19
:106EC800D3ED00EA40F38D80BAF1010F00F0C880DD
:106ED8008F4BA26901988F49D4ED9A6A334493ED98
:106EE800007A821A37EE6E7A8A4267EE26DA00F363
:106EF800B883894A128889498819D0ED006AF5EE65
:106F0800C06AF1EE10FA00F3D582F7EE00BA6DEE22
:106F1800A97AC3ED00EA67EE8D7A67EEABBAC5EDE4
:106F280002BA002A40F0A681D9ED036AF5EEC06ADC
:106F3800F1EE10FA40F3F584D4EDC57AF5EEC07A97
:106F4800F1EE10FA00F3EE80F7EE007A94ED9A7AFB
:106F580026EE877A27EE088A95ED027A28EE278AA8
:106F680085ED038AD5ED006AD5ED017A76EEA77A2C
:106F7800013777EE877A032F37EE888A09F11009EF
:106F880085ED048A06F1040605F114057FF4F2ADD7
:106F980094F81833002B40F052830023C8F80030CF
:106FA800C8F80430C8F80830C8F80C30C8F81030F1
:106FB800C8F81430C8F81830C8F81C30C8F82030A1
:106FC800C8F82430C8F82830C8F82C30C8F8303051
:106FD800C8F83430C8F838300BB0BDEC0E8BBDE8BB
:106FE800F08F4D4B4A4A1B8885ED02CA3244C2EDE8
:106FF80000EA002B3ED1BAF1010F95D185ED03CA05
:1070080094F80832D8ED0B7A022B00F02181F5EEC6
:10701800C07AF1EE10FA00F12A81B0EE4C7AB4EEA3
:10702800E77AF1EE10FA98BFF0EE477A012BC8ED37
:107038000B7A10D1D8ED067A88ED00CAF5EEC07A41
:10704800F1EE10FAB8BFF0EE4C7A88ED01CA88ED7F
:107058000ACAC8ED067A95ED038A95ED027A81E7AA
:107068002D4B2B4A1B8885ED02CA3244C2ED00EA3B
:10707800002BC3D0BAF1010F85ED03CAC0D0B0EE22
:107088004C8A95ED027A6DE7174A1278292A7FF41F
:10709800D8AE28EE2A0A049329F0BAFD164A049BB2
:1070A8005080CEE6012F00F0778294F80832012B49
:1070B80000F0C1821A4B3344D3ED00DAF6EE007AC1
:1070C800F4EEE7DAF1EE10FA88BFF0EE67DAFEEEDA
:1070D800007AF4EEE7DAF1EE10FAB8BFF0EE67DA0C
:1070E8006DEE8ADAB2E500BF042700200AD7233CF8
:1070F800C007002000007A4408270020003F002035
:10710800916100209361002092610020B06100200D
:107118000418002040420F00482D002024180020A9
:1071280080170020D24B334493ED007A67EE877ABC
:10713800B7EE007AF4EEC77AF1EE10FA88BFF0EEF7
:10714800477A03E799ED000AD5ED016ABAF1010F14
:1071580069EE00BA3FF445AEB0EE48EA6EEE2BBADF
:10716800022FC5ED00BA00F0DA82D9ED017A43E6C4
:10717800C04B1B78292B7FF49BAE28EE2A0A29F0F6
:1071880047FDBD4B988093E6BC4A02EBC702D2ED9F
:10719800007A92ED017A38EE678AE7EE087AB0EE67
:1071A800678AC2ED007A80E694ED7A7AD4ED7B6A3C
:1071B800B1F90030B1F9021094F8F82194ED7D5A34
:1071C800F4EEC76AF1EE10FAB4BFB0EE476AB0EE5B
:1071D800666A002BB8BF5B420029B8BF49428B42A0
:1071E800B8BF0B4607EE103AB8EEC77A27EE2C7AEE
:1071F800002A00F0EE80B5EEC05AF1EE10FA40F326
:107208002881D4ED7F4AF5EEC04AF1EE10FA40F33A
:10721800208134EEC77ADFED9A5AC7EE246A66EE0B
:10722800255AB7EE007A85EE856AF4EEC76AF1EE64
:1072380010FA88BFF0EE476AF5EEC06AF1EE10FA70
:1072480036EE077AB8BFF0EE4C6A26EE877AE2E0AF
:107258009FED8C7AF4EEC77AF1EE10FA40F1EC80EB
:1072680088ED0B7A95ED038A95ED027A7AE6F0EED1
:107278004C7ADBE685ED03CAB0EE4C8AB0EE6B7A49
:1072880070E6814A1268920740F110827F4A80496D
:10729800D4ED79DA31F917E085ED01CA02EB470C34
:1072A8006DEEACDABCF90AC0ACEB0E0C07EE90CA76
:1072B800F8EEE77A834267EEADDA3DEECDEAB0EE5E
:1072C8004E8A3FF702AD94ED0B7AF7EE007AB4EEF2
:1072D800E77AF1EE10FA00F10082F0EE4C6A99EDCF
:1072E800000ABAF1010F69EE00BA3FF47AAD94F8DA
:1072F8000932002B7FF430AF664B94F83C2203EB45
:10730800C703D3ED007A93ED016A3DEEE77AE6EE26
:10731800077AC3ED007A002A3FF420AF022F04D188
:10732800022A02D0042A7FF419AF3DEEE70A94ED51
:10733800906AB0EEC00A80EE067AF7EE00EA7EEEBA
:10734800C7EAF5EEC0EAF1EE10FAF5EEC06AB8BF8A
:10735800F0EE4CEAF1EE10FA05DDB5EEC08AF1EE7A
:1073680010FA00F10382F5EEC06AF1EE10FA00F1AE
:10737800F78194F84432012B00F01882002B00F0BA
:107388006A829FED458A002F7FF4E8AE394B1B785F
:10739800272B7FF4E3AECDED056A29F039FC364B97
:1073A80004932EEEAA0A188029F032FC049BB0EE52
:1073B800480A588029F02CFC049BDDED056A98806A
:1073C800CCE618B1237D002B3FF433AB01230293A5
:1073D800D0E4D4ED805AF4EECB5AF1EE10FA0FD582
:1073E800F7EE004A34EEE54ADFED2C6ADFED2C4A71
:1073F80036EEC77A64EE244AE7EE245A25EE255A7B
:10740800B5EEC05AF1EE10FA23D9CAEE856AB7EE86
:10741800007AA6EE667AB7EE006AB4EEC67AF1EEA6
:1074280010FA88BFB0EE467AB5EEC07AF1EE10FADF
:10743800B8BFB0EE4C7A0EE09FED1A7AEFE50E4D2C
:107448009FED190A28EE800A29F0E2FB2880FFF751
:1074580001BB9FED117AD4ED816A67EEA67AE7EE5B
:1074680087DAFFF7EFBB114ADFF84480FFF770BBFC
:10747800901700200427002008270020986100208A
:107488000000C8C2000048C2C4300020C830002034
:10749800B0280020CC170020000000000000344372
:1074A800610BB63B0000484200007A449C4700202C
:1074B800C43E002001F10C0C06EBC6006044D0ED80
:1074C800004AD0ED057A94EDBE6A94EDBD0A90EDC0
:1074D800017A90ED065AD0ED045AEDEEA47A803187
:1074E80001EBC701B0EEC8EA2EEE06EAB0EEE76A95
:1074F80026EE000A91ED006AF7EE00BAB4EECE0A65
:10750800F1EE10FA76EEC64A7BEEE66AADEE875AE1
:10751800B4BFB0EE4E7AB0EE407AE6EE874AD1EDCF
:10752800016A90ED037AA6EEA46A65EEE75AF0EEDA
:10753800466AB0EE456AA7EEC76AD0ED027A80EDDA
:10754800056AB0EE656AADEEA76AF4EEEB6AF1EE95
:1075580010FA80ED066A98BFF0EE66BAC1ED006ACF
:10756800002F00F0B981012F7FF4D1ACCA49097806
:1075780031297FF4CCACDFEDC97A94ED670A20EEAF
:10758800270ACDE9043220EE2B0A29F041FBC44931
:10759800DDE90432C880BAE4C24B94F81A033344D4
:1075A800D3ED00DAF6EE007AF4EEE7DAF1EE10FA4F
:1075B80088BFF0EE67DAFEEE007AF4EEE7DAF1EE75
:1075C80010FAB8BFF0EE67DA6DEE8ADA00283FF4F9
:1075D8003DABF5EEC0DAF1EE10FA7FF737ABB24902
:1075E800B24AB1F90230B2F90C209B1A07EE903A70
:1075F80007EE100AF8EEE77AB8EEC77A67EEAC7ACB
:10760800F4EEC77AF1EE10FA15DA77EE677AB2EE91
:10761800047AF4EEC77AF1EE10FA3FF617ABB1EE42
:10762800047A7DEEC7DA67EEAC7AA7EEAD7AF0EEB3
:1076380047DAFFF70BBBDFED9EDAFFF707BB94F8DD
:107648006C32002B7FF4A9AC94F81933002B3FF46B
:10765800C3AC0023C8F80430C8F81830C8F82C3078
:10766800BAE4039A92F84E2022B9924A1288110578
:107678007FF541AC94F86C22002A7FF43AAC8E4A2C
:1076880094F80912127812F0010240F0968000294D
:107698003FF42FAC0493104684F8092215F050FCEF
:1076A800844B99ED02DA1A88049B24E4834285ED21
:1076B80001CA7FF708AE814B1A88002384F8093283
:1076C800002A69D17E4A7F4B1178186881F0010140
:1076D80014F00CFED5ED016A01E6009B94ED877A63
:1076E800D3ED017AF0EEE77AF4EEC77AF1EE10FA0C
:1076F8007FF5F3ADD3ED027AF0EEE77AB4EEE77AF0
:10770800F1EE10FA7FF7E9ADD3ED037AF0EEE77A00
:10771800B4EEE77AF1EE10FA3FF7D0AADDE5B0EE65
:107728006B0AD4F850326848CDED046A9847BAF12C
:10773800010F88ED0A0ADDED046A7FF416ADFFF744
:1077480059BB5E4A1288AAB95D4A5E4B117818681F
:1077580014F0CCFDD4F80C32019AD31AFFF792BA80
:10776800B5EEC08AF1EE10FA7FF703AE022A3FF6B3
:107778000AAEFEE555494A69002A3FF483AA5448EF
:10778800544A008892FBF0F00A684FF0010C106030
:1077980081F811C0FFF776BA4C494A694AB10A68BC
:1077A800F0EE4C6A13604B74FFF713BB28EE2E8A79
:1077B800E9E5F0EE4C6AFFF70CBB94ED0B7AF7EEB7
:1077C800007AB4EEE77AF1EE10FA5DDB00295ED1BB
:1077D800D4ED9C7AB0EEED7AB4EEE77AF1EE10FAD9
:1077E8007FF787ABD4ED9D7AB0EECE7AB4EEE77A28
:1077F800F1EE10FA7FF77DABDBED007A94ED9E7A1F
:10780800F0EEE77AF4EEC77AF1EE10FA7FF571AB95
:1078180001220198C4F80C0284F80922D4F8102235
:107828008A427FF766ABD4ED9D7AB0EECEEAB4EE2D
:10783800E7EAF1EE10FA0BD4DBED007A94ED9E7ACC
:10784800F0EEE77AF4EEC77AF1EE10FA7FF751AB73
:10785800049300221FE777EECD7AB0EEE77AB4EE14
:10786800C70AF1EE10FA3FF78CADF5EEC07AF1EEEB
:1078780010FAACBF37EEC08A30EE278A83E5BAF13A
:10788800010F7FF4E3A910E400293FF432ABD4F8E8
:107898000C12019A511AC1E7042700202FAF934612
:1078A8000827002080170020B0280020C8300020BA
:1078B80000000000482D0020B72800201C470020A9
:1078C8001E47002020470020F017002024470020F2
:1078D8003C47002020A107001649097831297FF488
:1078E80016AB20EE2A0ACDE9043229F091F9DFF827
:1078F8004CB02EEE2A0AABF8000029F089F9DFED2A
:107908000E7A94ED630AABF8020020EE270A20EE07
:107918002B0A29F07DF9DDE90432ABF80400FFF702
:10792800F6BA85ED03CAB0EE4C8A95ED027AFFF7F8
:1079380019BB00BF042700202FAF9346082700205B
:1079480070B50A4C7625064621462A4629F0BBF929
:107958002A462146701929F0B6F92A46214606F129
:10796800EC00BDE8704029F0AEB900BF7410030800
:107978002DE9F041057804460E460846294690460A
:107988001F46FDF73BFE78B12379012B15D00FB9BF
:10799800BDE8F08129463046FDF710FE21784046C3
:1079A800BDE8F041FDF71ABE29464046FDF726FE20
:1079B8000028EDD12379012BE9D129463046FDF77E
:1079C8000DFE002FE4D121784046BDE8F041FDF7D7
:1079D80005BE00BF38B50B4B1B78093B012B00D9FE
:1079E80038BD054645200C4620F0C2FC0D2020F08D
:1079F800BFFC284620F0BCFC2046BDE8384020F0FB
:107A08002DBE00BF3C3800200C4B014610B5044683
:107A1800186813F0BFFE0A4B1888082280EA042071
:107A280041F2210110F4004F4FEA400018BF4840CE
:107A3800013A80B2F6D1188010BD00BF203B00206B
:107A4800283B002010B5054C206813F03DFE0028A7
:107A5800FAD02068BDE8104013F02EBE203B00206D
:107A680010B5FFF7EFFF094A138883EA00239BB29A
:107A7800082141F2210413F4004F4FEA430318BFD1
:107A8800634001399BB2F6D1138010BD243B00201E
:107A9800F8B5E64C8388D4ED9A7AB6EE007A67EEAC
:107AA800877A2DED048BFCEEE77A064617EE905A9E
:107AB8009D4280F05982C288954200F23C83DC4B9B
:107AC800DC4FC4F89C30DC4B97ED005AB6F86220C6
:107AD800D3ED004A7388B8EE455A002A40F05B811E
:107AE800002B40F05781D24BC4F80C31B6F84C301B
:107AF80013B19D4280F06C82CD4BC4F87C31338841
:107B080013B19D4280F02783C94996F85030DFEDC4
:107B1800CB6A94F83C22C4F8501207EE103AB8EE3B
:107B2800477A0023C6EE877AC4F81C3377EEA47A26
:107B380084EEA77A84EDC87ABAB194F82423C4F8FD
:107B4800243207EE902AF8EE677AC4F82C3286EED3
:107B5800A77AC4F8343237EE247AC4EE877AC4EDB3
:107B68008A7AC4ED8C7AC4ED8E7ADFEDB57A9FED12
:107B7800B57ADFEDB53AB54B9FEDB52A9FEDB53A2D
:107B8800DFEDB50A9FEDB51ADFEDB51ADFEDB56A81
:107B980074EEA77A25EE075AC4EEA72A03F17402F9
:107BA80003F16C05FDEEC57A35EE230A17EE901A3F
:107BB800FDEEC07A203117EE900AB7EE004A203069
:107BC800402900F28380B4EEC25AF1EE10FA40F375
:107BD800B782B0EE457ADFEDAA5A9FEDA36A01E0BD
:107BE800B0EE677AB4EEC67AF1EE10FA77EE657AFF
:107BF800F6DCF4EEC37AF1EE10FA40F1A982DFED7B
:107C0800A05A9FEDA06A01E0F0EE477AF4EEC67A3A
:107C1800F1EE10FA37EEA57AF6D4B4EEE37AF1EE87
:107C280010FA40F3A38032EE477A67EE077AB0EE97
:107C3800418AA7EEA08A4028F0EE618AE7EE888A9A
:107C480067EE275A9FED906AA5EEA87AB0EE448AAF
:107C5800F0EE447AA7EE068AE7EE467AC7EE888AFF
:107C68003AD9B0EE667AB6EE006AF7EE005AC4EE7C
:107C7800087A2433083243ED058A27EE866A67EED0
:107C8800A55A27EE877A03ED096A03ED076A43EDE3
:107C9800085A03ED067A43ED036A43ED046A43ED9F
:107CA800016A43ED026A9D4242ED026A42ED012AF1
:107CB80086D1DFED6E7AC4EDCA6A74EEA77ABDECA0
:107CC800048B84EEA77A84EDCB7AF8BDF7EE008AB0
:107CD8004028B0EE688AC4D8B4EEE35AF1EE10FA40
:107CE80040F38982B0EE407ADFED655A9FED5E6A17
:107CF80001E0B0EE677AB4EEC67AF1EE10FA77EEEC
:107D0800657AF6DCF4EEC37AF1EE10FA40F170828F
:107D1800DFED5B5A9FED5B6A01E0F0EE477AF4EE27
:107D2800C67AF1EE10FA37EEA57AF6D4B4EEE37A15
:107D3800F1EE10FA24DD32EE477A67EE077AB0EEFC
:107D4800416AA7EEA06AF0EE619AE7EE869A67EEBE
:107D5800275AB8EE009AA5EEA97AB6EE006A74EE34
:107D6800475A27EE097A25EE866A80E7DFED407AE2
:107D7800B4EEE77AF1EE10FA48BF33EE477A54E7EB
:107D8800DFED3B7AB4EEE77AF1EE10FA48BF33EE56
:107D9800477AD2E71A4695427FF6A5AE96F826307E
:107DA800002B00F00882012B7FF49DAE07EE102A0D
:107DB800DFED307A9FED240A2F49C4F80C1165EEE7
:107DC800277AB8EE477AB0EE403A27EE277A2B4B5F
:107DD8009FED1F2ADFED1F2ADFED1F0A9FED1F1AF7
:107DE800DFED1F1A9FED1F6AFDEEC77A37EE000A16
:107DF80017EE901AFDEEC07A203117EE902A40292E
:107E080003F16C0002F12002F7EE003A00F2A780BD
:107E1800B4EEC27AF1EE10FA40F3DE82F0EE476A71
:107E28009FED174ADFED105A32E000BFA815002079
:107E38003D020008B86000209461002083F9223ECA
:107E48003661823C98C4033ADB0FC93F30180020E2
:107E5800DB0F4940DB0F49C092E741B99730083C36
:107E680015A82ABE00000000E4CB1641F2D62D3C2E
:107E7800DB0FC9BF27D4D236D1010008481600202D
:107E8800DB0FC940E4CB16C1F304353FF0EE676A57
:107E9800F4EEE56AF1EE10FA76EEC47AF6DCF4EE6A
:107EA800E27AF1EE10FA40F194821FED0B4A5FED91
:107EB8000B5A01E0F0EE667AF4EEE57AF1EE10FA8C
:107EC80077EE846AF6D4F4EEC36AF1EE10FA40F362
:107ED800638272EE666A66EEA67AB0EE418AA7EE13
:107EE800A08AF0EE618AE7EE888A26EEA74A5FED5F
:107EF8001A5AE4EE286AB0EE638AF0EE637AA6EEC8
:107F0800A58AE6EEE57AC7EE888A402A40F2C8815B
:107F1800F0EE467AF6EE006AF7EE005A83EE884AEB
:107F2800243343ED058A66EE846A65EE845A67EE6B
:107F3800847A43ED096A43ED076A43ED085A43ED35
:107F4800067A03ED036A03ED046A03ED016A03EDA3
:107F5800026A98423FF4CAAD40297FF659AFF7EE5E
:107F6800008AB0EE688AD0E7002B3FF4A8ADC2883B
:107F7800002A3FF4A4AD07EE902A07EE103AF8EE77
:107F8800677AB8EE478A27EEE77A68EE277AA8EE8E
:107F9800087AD44FD44B3968D448C4F89C30C7EE1B
:107FA800878AB0EE480AF0EE680A24F0B3FDF0EED6
:107FB800680A3968CE48B0EE480A24F0ABFDF0EE06
:107FC800680AB0EE480A3968CA4824F0A3FD7AE581
:107FD80096F86020002A00F0D180012A7FF48CAD49
:107FE80007EE903AB8EE677ADFEDC37A9FEDC30AE1
:107FF800BD4AC34BC4F87C2127EE277AF0EE400A2D
:1080080027EE057ADFEDBF2A9FEDBF3A9FEDBF1A35
:10801800DFEDBF1A9FEDBF2A9FEDBF6AFDEEC77A5D
:1080280037EE000A17EE901AFDEEC07A203117EEEF
:10803800902A402903F16C0002F12002F7EE003A81
:1080480074D8B4EEE27AF1EE10FA40F3C881F0EE9B
:10805800476A9FEDB24ADFEDB25A01E0F0EE676A77
:10806800F4EEE56AF1EE10FA76EEC47AF6DCF4EE98
:10807800C37AF1EE10FA40F1A9819FEDA84ADFED2D
:10808800A95A01E0F0EE667AF4EEE57AF1EE10FA1C
:1080980077EE846AF6D4F4EEE06AF1EE10FA40F373
:1080A800858172EEE66A66EEA67AB0EE618AA7EE80
:1080B800818AF0EE428AE7EE888A26EEA74ADFED4B
:1080C8009A5AE4EE286AB0EE638AF0EE637AA6EE76
:1080D800A58AE6EEE57AC7EE888A402A40F28E80C5
:1080E800F0EE467AF6EE006AF7EE005A83EE884A1A
:1080F800243343ED058A66EE846A65EE845A67EE9A
:10810800847A43ED096A43ED076A43ED085A43ED63
:10811800067A03ED036A03ED046A03ED016A03EDD1
:10812800026A83423FF4EBAC40298AD9F7EE008A11
:10813800B0EE688AD1E7ABB2002A3FF4C0AC1AE7C8
:10814800F0EE457AF4EEC37AF1EE10FA3FF557AD4A
:10815800B0EE677A61E507EE903ADFED746A74492C
:10816800F8EE677A002386EEA77AC4F8483277EEED
:10817800247A84EEA77A84ED937AC6E407EE903ADF
:10818800DFED6A6A6A4AC4F87C21F8EE677A002350
:1081980086EEA77AC4F81031C4F83431C4F85831DF
:1081A80037EE247AC4EE877AC4ED457AC4ED4E7A68
:1081B800C4ED577AA3E407EE902ADFED5C6A5C4AC7
:1081C800C4F80C21F8EE677A002386EEA77AC4F883
:1081D800A030C4F8C430C4F8E83037EE247AC4EECE
:1081E800877AC4ED297AC4ED327AC4ED3B7A7DE40E
:1081F800B0EE677A9AE5F0EE407A83E5B4EEE07A7D
:10820800F1EE10FA40F3F180F0EE407A9FED434A28
:10821800DFED435A01E0F0EE667AF4EEE57AF1EE2E
:1082280010FA77EEC46AF6DCF4EEC36AF1EE10FADF
:1082380040F1D8809FED394ADFED3A5A01E0F0EE7F
:10824800676AF4EEE56AF1EE10FA76EE847AF6D40F
:10825800F4EEE07AF1EE10FA00F3B580DFED356A5E
:10826800F4EEE67AF1EE10FA48BF73EE677A67EE3D
:10827800A76AF0EE615AE6EE815AB0EE429AA6EE8F
:10828800A59A67EEA66AB8EE004AE6EE897AF6EE97
:10829800006A73EEE75A67EE847A65EEA66A25E708
:1082A800B4EEC37AF1EE10FA40F3A580F0EE407A0E
:1082B8009FED1A4ADFED1A5A01E0F0EE667AF4EE05
:1082C800E57AF1EE10FA77EEC46AF6DCF4EEE26ACB
:1082D800F1EE10FA40F18C809FED104ADFED115A53
:1082E8002CE000BFB860002089010008D8150020E4
:1082F800FC1500202016002027D4D236DB0FC93FFA
:10830800B8160020DB0F4940DB0F49C092E741B99E
:108318009730083C15A82ABE00000000DB0FC940B2
:10832800E4CB1641E4CB16C1F304353F83F9223E72
:1083380021020008DB0FC9BFF0EE676AF4EEE56AB8
:10834800F1EE10FA76EE847AF6D4F4EEC37AF1EE12
:1083580010FA35DC5FED096AF4EEE67AF1EE10FA10
:1083680048BF72EEE77A67EEA76AF0EE415AE6EE8A
:10837800A05AB0EE619AA6EEA59A67EEA66AB8EE84
:10838800004AE6EE897AF6EE006A73EEE75A67EE7F
:10839800847A65EEA66AC1E55FED1A7AF4EEE76ABB
:1083A800F1EE10FA48BF72EEE66A94E55FED1F7AC7
:1083B800F4EEE76AF1EE10FA48BF73EE666A72E609
:1083C80072EE677ACFE772EEE77A50E7F0EE676A07
:1083D80061E6F0EE676A76E5F0EE477A5FE5F0EE83
:1083E800477A44E6F0EE667A32E7F0EE406A1BE739
:1083F800F0EE667AA9E7F0EE406A67E7022816D839
:10840800022914D8884212D010B4094BC0EB0014CA
:10841800C1EB0112C0EB8400C1EB820103EB400009
:1084280003EB410176225DF8044B28F04CBC704701
:10843800DC35002090F84730F0B5002B40F06F8114
:10844800DFEDE24A8389027ADFEDE17A857ADFEDB2
:10845800E11A9FEDE12ADFEDE12A9FEDE13AE14FD4
:108468009FEDE14A05EE103A05EE902A427ADF4B7D
:10847800B8EEC55A06EE902A428AC3EDC54A25EEE3
:10848800275A06EE102A028B83ED645A07EE102A4B
:10849800827B9FEDD75A03EE902AF8EEE33AB8EEC6
:1084A800C66A63EEA13AB8EEC77AC3ED653AC27BF5
:1084B80003EE902AF8EEE33A26EE276A63EE823A54
:1084C80027EE277AC3ED663A067C83ED686A07EEE5
:1084D800906AF8EEE77AB0EE041A67EEA27A06EE32
:1084E800105AC3ED677A027D04EE902AF8EEE44A4A
:1084F800F8EEC63A64EEA14AF8EEE55AC3ED694AC9
:10850800427D90F816C083ED6C7A07EE902A07EE4C
:1085180010CAF8EEE77AB8EEC77A67EE827A27EEE5
:10852800227A67EE817A83ED6B7AC3ED6A7A827E6E
:1085380007EE102AC27E07EE902A027FF8EEE66A5E
:1085480006EE102AB8EEC77AF8EEE77A65EEA15A79
:1085580066EE826A27EE037A67EE837AB8EE466A99
:1085680063EEA22A90F82F20C3ED615AC3ED626A28
:1085780083ED797AC3ED817A83ED7D6AC3ED632A51
:1085880083F8F82190F82E10C48EB0F838E0D7EDB3
:10859800005AC1F1AF0206EE102AC1F1640207EEDB
:1085A800102A642202FB04F102FB0EF207EE902A65
:1085B80006EE901AB8EEC66AB8EEC77AF8EEE66A22
:1085C800F8EEE77A26EE046A90F8272083ED7F6AB2
:1085D80067EEA57A27EE057A66EEA56AB7EE006A19
:1085E800632A83ED807AC3ED726AC3ED717AC3EDB5
:1085F800707A83ED0A6A0BD807EE902AF8EEE77ACC
:10860800B0EE467AA7EEC57AC6EE077AC3ED0A7AC7
:1086180090F84F209FED727AB0F8404090F844707F
:10862800B0F842E090F8511007EE902A90F84520F3
:1086380005EE102A828F05EE902A428F06EE102A48
:10864800C28FF8EEE77A06EE902AB0F8482067EE77
:10865800877A07EE102AB0F84A20C3EDCC7A07EEE5
:10866800902A4FF47A7202FB04F4003102FB0EF2F6
:1086780007EB8707B8EE455AF8EE655AB8EE466A32
:10868800F8EE666AB8EE477AF8EE677AC3F81442ED
:1086980090F83040C3F810224FEA470718BF01216D
:1086A800828E83ED875AC3ED9D5AC3F8207283EDFD
:1086B8009C6AC3ED9E6A83ED867AC3ED967A83F849
:1086C80080111C779A84002C00F0CF80494A4FF023
:1086D8007E51116090F85420DFED476A83F8242317
:1086E80007EE902AF8EEE77A90F8552083F83C22B6
:1086F80086EEA77AB0F8622090F8531083F84412F7
:1087080083ED907AA2B190F82610002900F0CC8071
:10871800012940F0C580022183F834130AE007EEEE
:10872800903A9FED367AF8EEE77AC7EE274A89E65F
:1087380083F834233249A3F836230A6890F8661080
:1087480083F8081290F869109FED237AB0F8644016
:10875800A3F8384307EE901A12F00202F8EEE77A0F
:1087680018BF90F8682083F81A2367EE877A90F884
:108778006E20C3ED957A12B1AA42C0F08680DFED73
:10878800136A90F86F20C3ED9F6A002A42D0B24264
:1087980040D207EE902AB8EEE77A07EE906AF8EE34
:1087A800677A90F87020C7EE276AC3EDA06ACAB34B
:1087B800944537D907EE902AB8EEE77A07EE90CAC3
:1087C800F8EE677A87EE275A2EE000BF0000000017
:1087D8009D381039D730033D033F7A3E97AC0A3AAB
:1087E800CDCCCC3D946100206666E63FA8150020FC
:1087F8000AD7233CC4070020000048440000C842B0
:10880800C43000200000000095BF5633ACC5A73621
:108818006F1283395FED056A90F87020C3EDA06A86
:10882800002AC5D11FED095A90F87120D3ED9A7A24
:108838005FED0B5A1FED0B6A83EDA15A07EE102A64
:1088480090F87220B8EEC77A06EE902A67EEA57AFD
:10885800F8EEE66A67EE877A27EE067A67EEA67A7A
:1088680083EDBD7AC3EDBE7AF0BDA2F57A7207EE4C
:10887800902A5FED196A0E4AF8EEE77AB7EE007AA9
:10888800A7EEA67A82ED007A24E707EE902AB8EEE2
:10889800E77A07EE905AF8EE677AC7EE276A70E72C
:1088A800002183F8341345E7012183F8341341E7A5
:1088B800C407002038B5164A164B15781B689FED7B
:1088C800166ADFED166A164C164A174903FB05F3BC
:1088D80007EE903AF8EE677A236086EE277A044628
:1088E80067EEA67A82ED9A7AC1ED007A53B90F4BFA
:1088F800C2F89C30C2F80C31C2F850322046BDE8AC
:10890800384097E5FFF7C4F82046BDE8384091E5C0
:10891800AC3B00209C47002000247449BD378635B5
:10892800B8600020A8150020946100203D020008CE
:10893800334B1B78012B2BD1324B1B68B0F57A7F58
:1089480003F4805308DADFED307A9FED300A002B0C
:1089580008BFB0EE670A7047B0F5FA6F1DDCFBB9C7
:10896800B0F57A7F20D06FF47A7340F2CF72184452
:10897800274B02FB00F0A3FB0023C01A03EB5003B4
:108988005B0A30339BB200EE103AB8EE400A7047EB
:1089980007EE900AB8EE670A70479FED1E0A704707
:1089A80040F2DC53984202D19FED170A704740F21B
:1089B800DB53984211D9A0F2DD5040F2E73303FBB4
:1089C80000F340F2F31293FBF2F303F583639BB2D7
:1089D80000EE103AB8EE400A7047A0F57A70A3F698
:1089E800C21303FB00F340F2F31293FBF2F303F21A
:1089F80017439BB200EE103AB8EE400A704700BF2A
:108A080032530020344E00200000000000E0824471
:108A1800410A680600E0FF442DE9F84F414B1B78F6
:108A280083B3414A116809B100200860012B29D09D
:108A3800916909B100200860022B23D0116B09B19C
:108A480000200860032B1DD0916C09B1002008603C
:108A5800042B17D0116E09B100200860052B11D026
:108A6800916F09B100200860062B0BD0D2F8901046
:108A780009B100200860072B04D0D2F8A8300BB148
:108A880000221A6012F0B0FB284CDFF8AC80DFF847
:108A9800ACE0274DDFF8A890264E4FF0100A4FF4AF
:108AA8007A7740F2DB5CDEF80430C3F30803CBB915
:108AB800EFF31183B3B92368A96822689342FAD106
:108AC80032689142F7D8D8F8002007FB02FBABEBDD
:108AD8000101B1FBF2F107FB03131B1A6345E2D94D
:108AE800BDE8F88FEFF311818AF31288D5F808B042
:108AF8002B68DB0304D50123C9F80030D5F808B08A
:108B08002368D9F80020C9B281F31188D8F8001079
:108B1800134407FB01F2A2EB0B02B2FBF1F207FBD5
:108B28000323DAE79060002058520020984500207F
:108B380010E000E0A8450020A445002000ED00E07A
:108B4800A04500202DE9F04F6E4B6F4ED3EDCF7A44
:108B580030786E4B83B01A78002800F0CC80FDEE98
:108B6800E77A012817EE903A1BB207EE903A684B65
:108B7800F8EEE77AC3ED007A19D00228C3ED017A3E
:108B880015D00328C3ED027A11D00428C3ED037A67
:108B98000DD00528C3ED047A09D00628C3ED057A5F
:108BA80005D00728C3ED067A01D0C3ED077A002A5D
:108BB80040F0918032235748DFF86CE1DFF86CC150
:108BC800554CDFF86C81554E01934FF01009DCF8D5
:108BD8000430C3F30803002B5ED1EFF31183002B9D
:108BE8005AD10568A26803689D42FAD133689A424F
:108BF800F7D8DEF800704FF47A7101FB07F39B1A7F
:108C0800B3FBF7F301FB05354FF47A774FF0010A10
:108C1800DCF80430C3F30803FBB9EFF31183E3B9BD
:108C28000368A16802689342FAD132689142F7D882
:108C3800DEF8002007FB02FBABEB0101B1FBF2F110
:108C480007FB03135B1BB3F57A7FE1D3019B013B61
:108C58000193BCD103B0BDE8F08FEFF3118189F324
:108C68001288D4F808B02368DB0344BFC8F800A012
:108C7800D4F808B00368D8F80020C9B281F3118885
:108C8800DEF80010134407FB01F2A2EB0B02B2FB63
:108C9800F1F207FB0323D5E7EFF3118389F3128879
:108CA800A7682268D20303D50122C8F80020A76864
:108CB8000568D8F800A0DBB283F31188DEF800104D
:108CC8004FF47A72554402FB01F3DB1BB3FBF1F35B
:108CD80002FB053598E70E4D114F0024E0B23B68C2
:108CE800B5EC010A9847307801348442F6DB0D4B25
:108CF8001B6898475EE7002A3FF45CAF094B1B6886
:108D0800984757E7A81500209060002008600020C9
:108D1800502D00209845002010E000E0A8450020D4
:108D2800345300203C530020A445002000ED00E00F
:108D3800A0450020094BD3F83C23C3F84023C3F8CF
:108D48004423C3F84823C3F84C23C3F85023C3F87B
:108D58005423C3F85823C3F85C237047A815002090
:108D68002DE9F04FDA4CDFF894B394F86033A3F1AF
:108D780017020021022A8BF800105FD9D54A12F891
:108D880033508BF8005002EBC303082DD3F804C00E
:108D980040F2B88108258BF80050BCF1000F00F0B4
:108DA800DF809CE80F0004F5597686E80F000CF187
:108DB80010030FCB04F55D7787E80F00AB460CF185
:108DC80020030FCBC44DBBF1030F85E80F0000F063
:108DD800B5810CF130030FCB05F1100EBBF1040F78
:108DE8008EE80F0000F0B5810CF140030FCB05F1C0
:108DF8002008BBF1050F88E80F0000F0B3810CF1E3
:108E080050030FCB05F13009BBF1060F89E80F00BD
:108E180000F0AF810CF160030FCB05F1400ABBF104
:108E2800080F8AE80F0040F0A9810CF1700C9CE84B
:108E38000F0005F1500C8CE80F00A1E0DFF8C0C26C
:108E4800DCED007AF5EE407AF1EE10FA00F0888059
:108E58009CE80F00DCED047AF5EE407A04F55976CB
:108E68000125F1EE10FA86E80F008BF8005079D052
:108E78000CF110030FCBDCED087AF5EE407A04F51F
:108E88005D770225F1EE10FA87E80F008BF80050A5
:108E98006AD00CF120030FCBDCED0C7AF5EE407AAA
:108EA80004F561754FF0030EF1EE10FA85E80F0036
:108EB8008BF800E05AD00CF130030FCBDCED107AC0
:108EC800F5EE407A04F5657E4FF00408F1EE10FAED
:108ED8008EE80F008BF800804AD00CF140030FCBCE
:108EE800DCED147AF5EE407A04F569784FF005095F
:108EF800F1EE10FA88E80F008BF800903AD00CF1E8
:108F080050030FCBDCED187AF5EE407A04F56D7955
:108F18004FF0060AF1EE10FA89E80F008BF800A06E
:108F28002AD00CF160030FCBDCED1C7A04F5717AC2
:108F3800F5EE407A8AE80F00F1EE10FA4FF00703D9
:108F48008BF800301AD00CF1700C9CE80F0004F577
:108F5800757C8CE80F004FF008038BF800300FE0A9
:108F680004F5597604F55D7704F5617504F5657EB9
:108F780004F5697804F56D7904F5717A04F5757C62
:108F880096E80F00554E86E80F0097E80F00544EFC
:108F9800D4EDFB7A86E80F0095E80F00514D85E87F
:108FA8000F00F5EEC07AD4EDFF7AF1EE10FAF5EE87
:108FB800C07AD5ED027A2B464FF0000B44BFC4F8B7
:108FC800ECB3C4F8E4B30027F1EE10FA03F1080398
:108FD800F5EEC07A4FF0000644BFC4F8FC73C4F83D
:108FE800F473F1EE10FA44BF1E602E609EE80F0085
:108FF8003D4D85E80F00D5ED027A2B46F5EEC07A97
:109008000833F1EE10FA4FF0000648BF1E6098E8EA
:109018000F0048BF2E60354D85E80F00D5ED027A68
:109028002B46F5EEC07A0833F1EE10FA4FF0000641
:1090380048BF1E6099E80F0048BF2E602C4D85E898
:109048000F00D5ED027A2B46F5EEC07A0833F1EE23
:1090580010FA4FF0000644BF1E602E609AE80F0019
:10906800244D85E80F00D5ED027A2B46F5EEC07A3F
:109078000833F1EE10FA4FF0000648BF1E609CE876
:109088000F0048BF2E601C4D85E80F00D5ED027A11
:109098002B460833F5EEC07A0026F1EE10FA48BFE9
:1090A8001E60D4F83C3348BF2E60C4F84033C4F87F
:1090B8004433C4F84833C4F84C33C4F85033C4F8C4
:1090C8005433C4F85833C4F85C33BDE8F08F00BF9C
:1090D800A8150020904D03082C1900208C19002099
:1090E8009C190020AC190020BC190020CC190020C4
:1090F800DC190020EC190020FC19002090600020E9
:1091080010600020BCF1000F3FF42AAFAB46002DE1
:109118003FF426AF9CE80F0004F55976012D86E848
:109128000F003FF41FAF0CF110030FCB04F55D7770
:10913800022D87E80F007FF442AE15E705F1100E07
:1091480005F1200805F1300905F1400A05F1500C38
:1091580016E705F1200805F1300905F1400A05F187
:10916800500C0DE705F1300905F1400A05F1500CE6
:1091780006E705F1400A05F1500C01E705F1500C2E
:10918800FEE600BF6A4B1B6893F87330632B37D831
:1091980007EE903A9FED677AF8EEE77A67EE877AFE
:1091A8006549664B8A781B68053A042A03F480539C
:1091B80029D80A8ADFED626A6249B7EE007A77EE4B
:1091C800677A07EE102A0020B8EEC77A67EEA67A0B
:1091D800C1F83C03002B43D1DFED5B5A9FED5B6A7E
:1091E800DFED5B6A5B4A5C4BA7EE256A76EEE77AB1
:1091F80082ED006AC3ED007A584B594A1A607047ED
:10920800F7EE007ACCE730B4002B53D18B8A4A8A28
:10921800C98A51489C1A07EE103A06EE104AF7EE32
:10922800005A77EEE57AB8EEC66AB8EEC77A06EE67
:10923800901AA6EE277A4349464BF0EE477A07EE96
:10924800102AF8EE666AB8EE477AC0ED007AC1EDEA
:10925800CF6A83ED007A414B414A1A6030BC7047AF
:109268009FED3B5ADFED3F5ADFED386ADFED3E4AAE
:109278009FED3E6A374B3848F1EE677AB6EE004A02
:10928800A7EE845A01F58D6201F26441E7EE845A33
:10929800F0EE667AA7EE246AE7EE247AC2ED005A69
:1092A80080ED005A81ED006AC3ED007A2B4B2C4A01
:1092B8001A607047234B274DB3F87424B3F876141B
:1092C800B3F87004244C07EE102AF7EE006A8A1AE5
:1092D80076EEE76AB8EEC76A07EE901A07EE102A2C
:1092E80005EE900ABAEEEF7AB3F86E04B3F86C2480
:1092F800F8EEE77AA6EE876A03F26441E6EEC77AEB
:1093080007EE100AF8EE476A07EE102AF8EE655ADB
:10931800B8EE477A03F58D62C3EDCF5A85ED006A42
:10932800C4ED007AC1ED006A82ED007A93E700BFD0
:10933800C82C00200AD7233C18530020344E0020A4
:1093480000E0F944A815002095B24C3E00004042C8
:1093580000E0FF444C2D0020702D0020241A00202E
:1093680000007A4400E082445E98CC3D00008344CB
:109378002C4B187810F001004FD12B4B1B78002B89
:109388004DD02A4AD2EDD07A92EDCF7AF4EE477AD0
:10939800F1EE10FA41D1012B42D092EDD17AB4EE20
:1093A800677AF1EE10FA38D1022B39D092EDD27AE1
:1093B800F4EE477AF1EE10FA2FD1032B30D092ED6C
:1093C800D37AF4EE477AF1EE10FA26D1042B26D0A0
:1093D80092EDD47AF4EE477AF1EE10FA1DD1052B0E
:1093E8001DD092EDD57AF4EE477AF1EE10FA14D149
:1093F800062B14D092EDD67AF4EE477AF1EE10FAF5
:109408000BD1072B0BD092EDD77AF4EE477AF1EE19
:1094180010FA14BF01200020704701207047002077
:10942800704700BFB728002090600020A8150020D2
:109438004A4B9FED4B7A1A799FED4A5ADFED4A5A0B
:1094480007EE902AF8EEE77A1A885B8867EE877A43
:1094580006EE102A37EE857A06EE903AFDEEC74AF8
:10946800B8EEC66AF8EEE66A14EE903A3F4A66EE3F
:10947800A56A26EE256A2033402BC2ED006A82EDEC
:10948800016A06EE900A13D99FED397A9FED396A81
:10949800394BF8EEE67A03F28C42C6EE276A03F5FA
:1094A8009160C3F8901480ED007AC2ED006A7047AD
:1094B800F4EEC57AF1EE10FA4DDDDFED305A9FED8E
:1094C800306A01E0B0EE677AB4EEC67AF1EE10FACF
:1094D80077EE657AF6DC9FED2B7AF4EEC77AF1EE3B
:1094E80010FA35D5DFED255A9FED276A01E0F0EE39
:1094F800477AF4EEC67AF1EE10FA37EEA57AF6D48A
:10950800DFED187AB4EEE77AF1EE10FA1BDCDFED46
:109518001F7AB4EEE77AF1EE10FA44BFDFED197A5C
:1095280037EEC77A67EE075A9FED195A9FED196A09
:10953800DFED197AA5EE856A27EE255AE5EE867ADB
:10954800A5EE277AA2E7DFED157A37EEC77AE9E7C5
:10955800B0EE677AD4E7F0EE477ABCE7BC28002083
:1095680035FA8E3CDB0FC93F17B7D138281A0020CF
:1095780000000000C0C9FB48A8150020DB0FC94047
:10958800E4CB1641DB0F49C0E4CB16C1DB0FC9BFE2
:1095980092E741B99730083C15A82ABEDB0F49402D
:1095A8003D4B3E4AD3ED0F5A93ED116AD3ED107A35
:1095B800D3ED0E6A2DED048B25EEA59A26EE060A4C
:1095C80039EE097A30EE005A27EEA78A26EE861A77
:1095D80065EEA71A66EEA72A26EEA52A67EE867A12
:1095E80065EE865AB1EE477AF0EE004AF0EE470A89
:1095F800F0EE458AE8EE640AE8EE248A37EE457A0A
:1096080071EEC13A31EE214A72EEA54A35EEE25AC0
:1096180037EEC26A66EEA66A33EEA33A74EE043AEF
:1096280034EEA44A75EE054A36EE065A32EE276A3B
:10963800C3ED006AF7EE006A37EE267A70EEA60AE6
:1096480036EE066A76EEE86A83ED049A83ED078AB9
:1096580083ED090A82ED047AC2ED080AC2ED006AB8
:1096680083ED031AC3ED051A82ED013AC2ED033A00
:1096780083ED012AC3ED022AC3ED065AC3ED087A29
:1096880082ED024AC2ED064A82ED055A82ED076A6A
:10969800BDEC048B704700BF2C0000203C1A002052
:1096A800064B1B6813F0020F054B02D093F83820C5
:1096B80042B90022DA621A635A637047C430002044
:1096C800843200202DE9F041F04CD4F8B814D4F8D5
:1096D800BC24C4F8B804411A2DED088B06EE101A04
:1096E800002A00F0C08307EE902AB8EE677AF7EEFA
:1096F800007AC7EE876A04F598620021C4F8BC14A2
:109708000021D2ED010ADFEDE23AD2ED007A92EDC6
:10971800021A116066EEA00A66EEA77A60EEA32A26
:1097280027EEA33A22EEA24A26EE811AA3EE034AB6
:109738005160916061EE233AA3EEA34AD4F8CC2499
:10974800002A40F39F8307EE102AB8EEC77AF7EE97
:10975800006A86EE875ACF4ACF490025C4F8CC5410
:10976800D2ED016AD2ED004AD2ED021A93ED007AE9
:109778009FEDCA2A65EE266A65EE244A66EEA65A69
:1097880025EE215AE4EEA45A0023136027EE077A47
:10979800E5EE055A53609360C1ED004A27EE257A3D
:1097A800C1ED016AB4EEC27AF1EE10FA81ED025A07
:1097B80007DD9FEDBB2AB4EEC27AF1EE10FA48BF7E
:1097C8000125B84E9FEDB87A3378B8EEC66A13F023
:1097D800010326EE076A00F0DD81B44B012193ED09
:1097E800017A84F8DC14002D40F00E83DFEDB07AA6
:1097F800DFF8EC82F0EE676AF0EE674AF0EE671A7F
:10980800B0EE671AF0EE670A93ED007AB5EEC07A0B
:10981800F1EE10FA4FF0000340F34783A54B9FED9C
:10982800A60A93ED002A19461A46B4EEC04A043136
:109838000832F1EE10FA91ED005AD2ED005A00F11B
:109848003B8373EEA53A72EE852A33EE023AB6EE02
:10985800007A9A4926EE076A74EE834A77EEA37A6D
:1098680064EE864AD1ED113A91ED103A91ED0E7AF7
:1098780091ED0F4A76EEA26A67EE867A66EE866A00
:1098880064EEA35A27EE835AE6EE875AA4EE875A67
:1098980026EE846A75EE835AA7EE876AF1EE672A88
:1098A80035EE045AE2EE845AF0EE467AB0EE456A96
:1098B800A6EEE36A25EEA55A77EEA37AA6EE065A37
:1098C800E4EEC37A66EE836AA2EEA37AE4EE846AD3
:1098D800A7EEA75A37EE667AF0EE456AE7EE076A12
:1098E800B7EE00BAB1EEE65ACBEE056A27EE267A55
:1098F80026EE266A65EEA65A67EEA67A81ED0E7AFE
:1099080081ED0F6AC1ED105AC1ED117AFFF748FEDB
:109918006B4B1F887B0640F17D81D1ED144AD1ED58
:10992800135A91ED156A91ED127A64EEA49A24EE19
:10993800865AF0EE693AE5EEA53AA7EE255A73EE97
:10994800A33A35EE055A7BEE636AB0EEC54AF0EEEF
:10995800E66AF4EEC46AF1EE10FAB4BFF0EE447AA7
:10996800F0EE667AF5EE407AF1EE10FA67EE248AA8
:1099780027EE068A25EEA4AA25EE869A66EE06AAA2
:1099880040F0D9829FED5C7A9FED4E0A4E4DF4EE81
:10999800C46AF1EE10FA44BFDFED587A37EEC77AA1
:1099A800F7EE007AF4EEE73AF1EE10FAC8BFDFED11
:1099B800557AB5EEC05AC8BF37EEC77AF1EE10FA3D
:1099C80048BFB1EE477A27EE000A27F021F978EE72
:1099D800C97AB7EE005A77EEA77ADFED3C4ADFED99
:1099E8003C5A9FED3C6A9FED3C7A2880F0EEE76A8E
:1099F80035EE665AE6EEA45AB1EEC50AA6EEA56A99
:109A0800F5EEC07AA6EE867AF1EE10FA48BFDFEDE1
:109A18003D7A27EE007A9FED2B0A48BF37EEC77ACA
:109A2800DFED367A37EEC77A27EE000A27F0F0F82E
:109A380079EEAA7A38EE0A7A77EEA77AF7EE005A24
:109A480037EE077A75EEE76AB0EEC76AF0EEE66AB7
:109A5800F4EEC66AF1EE10FAB4BFB0EE465AB0EEB4
:109A6800665AB5EE405AF1EE10FA688000F0EE82C0
:109A7800F4EEC66AF1EE10FA8CBFB0EE464AB0EECC
:109A8800664AC4EE054A9FED152A3DE0A815002058
:109A980035FA8E3C781A002048330020295C4F3F65
:109AA80048E19A3FB7280020BD378635281A00209C
:109AB80000000000941A0020E68AF93D2C000020DE
:109AC800482D00204C3D0F44B0280020306E99BC32
:109AD8002716983D843459BEA40DC93F99FB243FED
:109AE8003C1A002069A2163E39094E3DE3B59E3E58
:109AF80088FA163E45FE7F3FA7DFA834DB0FC93F33
:109B08004C3D0FC4DB0F49401FED0A5A5FED0A1A9E
:109B18005FED0A2A1FED0A3A5FED0A3A1FED0A4A7D
:109B2800A4EE825AE4EEE12AE4EE855AA4EEA23AC3
:109B3800B0EE655AF0EE635AE4EE835AA4EEA54AF5
:109B4800C4EE055AF4EEC66AF1EE10FA48BF5FEDAE
:109B5800156A1FED150A48BF76EEE55AF7EE006A5A
:109B6800F4EEE67AF1EE10FAC8BF5FED1A7AB5EEB8
:109B7800C07AC8BF77EEE55AF1EE10FA48BFF1EEA9
:109B8800655A25EE800A27F043F800B2A88098EDC0
:109B9800088A0DE194F8DC14002940F0F681D4F825
:109BA800E414002900F0B182F0EEE77AB2EE0E7A02
:109BB800F4EEC77AF1EE10FA00F33082F0EEE07AB4
:109BC800F4EEC77AF1EE10FA00F32882F0EEC17ACB
:109BD800F4EEC77AF1EE10FA00F32082002D00F0BF
:109BE8001D82002900F08E8288424FF00003C0F0E9
:109BF80006810121C4F8E034C4F8E43484F8DC3484
:109C080084F8E814EB4B93ED017AF2EE047A27EE30
:109C1800277AE8E5D8ED075A98ED088AB0EEE57A94
:109C2800F0EEC86AF4EEC76AF1EE10FAB4BFF0EECF
:109C3800477AF0EE667AF5EE407AF1EE10FA40F0E7
:109C480050819FEDDD6A9FEDDD0ADD4DF4EEC76AB8
:109C5800F1EE10FA48BFDFEDDB7AB5EEC08A48BFF7
:109C680037EEC66AF1EE10FA48BFDFEDD77AF5EEA7
:109C7800C05A48BF37EEC66AF1EE10FA48BFB1EED7
:109C8800466A26EE000A26F0C3FF98ED065ADFED75
:109C9800DF4A9FEDDF6ADFEDE06ADFEDDE7A2880DC
:109CA800B0EEC57AF7EE005A75EEC75AA7EE246AE9
:109CB800B1EEE50AE7EE066AB5EEC05AE7EE267A97
:109CC800F1EE10FAC8BF9FEDC07A67EE807A9FED7B
:109CD800BB0AC8BF77EE677A9FEDBA7A77EE677AE4
:109CE80027EE800A26F094FF98ED036AD8ED005A13
:109CF8006880F0EEC67AB0EEE57AB4EEE77AF1EE77
:109D080010FAB4BFB0EE675AB0EE475AB5EE405AF3
:109D1800F1EE10FA00F09D81B4EEE77AF1EE10FA58
:109D28008CBFF0EE674AF0EE474AC4EE856A9FEDB5
:109D3800A72A9FEDA75A9FEDA73A9FEDA74ADFED07
:109D4800A72ADFEDA73ADFED9C4AA6EEC25AE6EE57
:109D5800A23AA6EE853AB7EE005AA6EE834AA6EED8
:109D6800A35AE6EE844AC4EE856AB4EEE77AF1EEC9
:109D780010FA48BFDFED937A9FED9A0AF5EEC05AC4
:109D880048BF77EEE66AF1EE10FA48BFDFED8E7A4B
:109D9800B5EEC06A48BF77EEE66AF1EE10FA48BF42
:109DA800F1EE666A26EE800A26F032FF00B2A8803D
:109DB8008D4B8E4AD3ED007A13780028B8BF00F592
:109DC8006160F4EEC87AB8BFA880F1EE10FAD4F852
:109DD80090544CBF43F0080303F0F703137045B1E8
:109DE80017F0030704D0337813F0010340F03681ED
:109DF8000025BDEC088BC4F8F854BDE8F08184F860
:109E0800DC346C4BB3EE097ADFED797AF4EEE75A7D
:109E1800F1EE10FA7FF7EAACB1EEE52ADFF8E0815F
:109E2800F7EE005AC5EE827A98ED080AD8ED075A7F
:109E380098ED062A67EEA44A67EEA66A27EE855AC9
:109E480020EE641A62EE661A65EEC50AE4EEA51AFB
:109E5800E6EE800AA5EE021A60EE874A61EE076A0E
:109E680061EE877AD0E49FED634AF0EE443AF0EE73
:109E7800442AB0EE443AB0EE441AF0EE440AF0EE4A
:109E8800447A5BE49FED5B7A5B4BF0EE475A83EDD7
:109E9800007AB0EE475AF0EE476AF0EE474A83ED93
:109EA800017A83ED027A00258BE454490A468B60D7
:109EB80042F8043B1360CAE426EE077AA0EE872A2C
:109EC800A1EE075AE1EE875A83ED002A33EE023AF3
:109ED80081ED005A72EE852AC2ED005A73EEA53A5A
:109EE800B5E4F4EEC76AF1EE10FA8CBFB0EE475A4B
:109EF800B0EE665A85EE276ADFED342ADFED343A94
:109F08009FED344ADFED344A9FED343ADFED347A81
:109F18009FED295AE6EE623AE6EE037AA6EE234A68
:109F2800A6EE27BAE6EE044AF0EE4B7AA6EE245ADD
:109F380085EE0B6A87E6F4EEC46AF1EE10FA8CBF80
:109F4800B0EE446AB0EE666A86EE277ADFED204A04
:109F5800DFED1E7A9FED1F6ADFED1F5A9FED1F3A56
:109F6800E7EE674ADFED1E7AA7EE246AE7EE037A8A
:109F7800E7EE065A9FED106AA7EE27BAA7EE256A04
:109F8800F0EE4B7A86EE0B7AFEE400F574319031F0
:109F9800C4F8E43484F8E834C4F8E01400295BD148
:109FA80094F8E834002B7FF4FFAD002384F8DC3408
:109FB80028E600BF281A0020A7DFA8344C3D0F442C
:109FC800B0280020DB0FC93FDB0F494039094E3D5F
:109FD800E3B59E3E88FA163E45FE7F3F99FB243F37
:109FE80069A2163E4C3D0FC4301A0020B828002044
:109FF8000AD7233C0000000048330020941A0020B0
:10A008003C1A0020A7DFA8348FC2753C306E99BC7B
:10A018002716983DA40DC93F843459BE00F5743302
:10A0280090330021C4F8E034C4F8E414002BBCD009
:10A038009842BAD300F5F420002300F59070C4F8D4
:10A04800E404C4F8E03484F8DC34DBE55FED135A4B
:10A0580078E55FED146A88E60021A5E55FED167ADC
:10A06800B4EEE78AF1EE10FA7FF6C2AEB0EEC87A27
:10A07800F7EE005A75EEC75A5FED1C4A1FED1C6AD1
:10A088005FED1B6A5FED1D7A214BB1EEE55AA7EE35
:10A09800246AB5EEC08AE7EE066AF1EE10FAE7EE3A
:10A0A800267A48BF9FED1B7A93ED000A67EE857A02
:10A0B80048BF77EE677A27EE800A26F0A9FDB0F54B
:10A0C800617F14DC07EE900AB8EEE70ADFED127A3A
:10A0D80020EE270AFDEEC07A17EE903A2033402B87
:10A0E80007D99FED0E0A26F093FD054681E69FED00
:10A0F8000C0AF9F769FF07EE905AF8EEE77A27EEAF
:10A10800800AF0E7D4F8E03490E7D4F8E01445E7A3
:10A11800341A0020DB0F4940D06D393A00000000A6
:10A1280084F9223FF0B51A4E1A4D83B00024ADF8D9
:10A1380004400094C6F8FC44C6F800450CE0D6F884
:10A148000035F218013382F80475C6F80035013479
:10A15800142C05F1060518D06B79284606226946A5
:10A16800E7B2002BEBD126F09FFD0028EFD0D6F800
:10A17800FC340134F218142C03F1010382F8187529
:10A18800C6F8FC3405F10605E6D103B0F0BD00BF02
:10A19800A8150020603F00202DE9F041284F00213C
:10A1A80007F1060E0A468C4601EB4104630017F8D6
:10A1B8001440844207EB03053CD05B1B2C464E1C25
:10A1C800CABB7344142E1D4407D014F8062F8242CC
:10A1D80005D00136142E1D44F7D1BDE8F0810122C7
:10A1E8009319132B15D803EB430407EB440117F815
:10A1F8001440844208BF013305D012E011F8068FDD
:10A2080080450ED12346132B02F1010203F101040C
:10A21800F4D9C5F800C0A5F804C0711C1429C3D12D
:10A22800DBE703EB430307EB4303196829609B88CB
:10A23800AB80F2E70AB10E46D2E70E460122CFE71D
:10A24800603F0020114B03F1780102E006338B4296
:10A258001AD01A788242F9D110B49C78DA789442EC
:10A268000ED35A7962B906338B4205D01A788242E6
:10A27800F3D006338B42F9D100205DF8044B7047C8
:10A2880001205DF8044B704700207047603F0020B4
:10A2980001460148FBF7B2B9703B00202DE9F041B7
:10A2A800274F284E82B00024ADF804400094C7F828
:10A2B800FC44C7F8004535460CE0D7F80035FA18D5
:10A2C800013382F80485C7F800350134142C05F1F0
:10A2D800060519D06B792846062269465FFA84F884
:10A2E800002BEAD126F0E0FC0028EED0D7F8FC34A9
:10A2F8000134FA18142C03F1010382F81885C7F801
:10A30800FC3405F10605E5D10F4A02E00636B242F3
:10A318000FD03378002BF9D1B078F178884202D386
:10A3280071790029F2D0094A82F8583002B0BDE8A4
:10A33800F081064A012382F8583002B0BDE8F08166
:10A34800A8150020603F0020D83F00202C000020E6
:10A35800144B154A1B68DB0410B5B2F9064006D445
:10A36800124B988AA042CCBF0020012010BD1521B5
:10A378000F48FBF743F90028F2D10E4B93F87824E5
:10A38800002AEDD1094AB3F87234508AC21A9442AD
:10A3980005DD18448442B4BF0020012010BD01200F
:10A3A80010BD00BF344E002024330020646100201B
:10A3B800703B0020A8150020054B93F8252022B9F2
:10A3C800187E003018BF012070470120704700BF79
:10A3D800646100202DE9F041DE4BDF481D68DF4C49
:10A3E8002F786A78BBB2594209B2002914BFBE4619
:10A3F8004FF0010E01FB01FCC2F164060EFB0EFEDC
:10A4080002FB0CFC9CFBFEFCB44401FB0CF103EBCF
:10A41800830C80FB010EC8174FEA4C01C0EBAE005D
:10A4280001F57A71C3F10A0E0844C7F1640CBEF154
:10A43800000FA4F82C055FFA8CFC40F37E81E046FF
:10A448000EFB0EF018FB08F802FB00F090FBF8F08A
:10A45800DFF8048330440EFB00FE88FB0E804FEAD1
:10A46800EE7ECEEBA00EC3F114008E440028A4F8B3
:10A478002EE540F35B81E64600FB00F81EFB0EFE6E
:10A4880002FB08F898FBFEF8DFF8CCE2B04400FBCA
:10A4980008F08EFB008EC017C0EBAE0EC3F11E0095
:10A4A8008E440028A4F830E540F33981E64600FBE5
:10A4B80000F81EFB0EFE02FB08F898FBFEF8DFF81A
:10A4C80098E2B04400FB08F08EFB008EC017C0EB8A
:10A4D800AE0EC3F128008E440028A4F832E540F3FC
:10A4E8001781E64600FB00F81EFB0EFE02FB08F88B
:10A4F80098FBFEF8DFF860E2B04400FB08F08EFB42
:10A50800008EC017C0EBAE0EC3F132008E44002897
:10A51800A4F834E540F3F580E64600FB00F81EFB9E
:10A528000EFE02FB08F898FBFEF8DFF82CE2B044B8
:10A5380000FB08F08EFB008EC017C0EBAE0EC3F117
:10A548003C008E440028A4F836E540F3D380E64664
:10A5580000FB00F81EFB0EFE02FB08F898FBFEF855
:10A56800DFF8F4E1B04400FB08F08EFB008EC01762
:10A57800C0EBAE0EC3F146008E440028A4F838E5BF
:10A5880040F3B180E64600FB00F81EFB0EFE02FB1E
:10A5980008F898FBFEF8DFF8C0E1B04400FB08F0CB
:10A5A8008EFB008EC017C0EBAE0EC3F150008E4478
:10A5B8000028A4F83AE540F38F80E64600FB00F84F
:10A5C8001EFB0EFE02FB08F898FBFEF8DFF888E198
:10A5D800B04400FB08F08EFB008EC017C0EBAE0E37
:10A5E800C3F15A008E440028A4F83CE56EDDE64627
:10A5F80000FB00F81EFB0EFE02FB08F898FBFEF8B5
:10A60800DFF854E1B04400FB08F08EFB008EC01761
:10A61800C0EBAE0EC3F164008E440028A4F83EE5FA
:10A628004EDDE04600FB00FE18FB08F802FB0EFEBC
:10A638009EFBF8FEDFF82081B64400FB0EF088FB95
:10A64800008EC017C0EBAE00C3F16E030844002BA8
:10A65800A4F8400503DC0CBF4FF0010CBC4603FB1B
:10A6680003F002FB00F21CFB0CFC3B4892FBFCF2E3
:10A67800324403FB02F380FB0302DB17C3EBA203A4
:10A688001944A4F84215AB78354A012B14BF354B51
:10A69800354BC4F84435354B5B7E00211170042BD3
:10A6A80006D8DFE803F00A54075103000B231370A0
:10A6B800BDE8F0810F231370FAE703231370F7E75F
:10A6C80018BFB846AED14FF00108ABE718BFBE4679
:10A6D8008ED14FF0010E8BE718BFBE467FF46EAFE8
:10A6E8004FF0010E6AE718BFBE467FF44CAF4FF03B
:10A6F800010E48E718BFBE467FF42AAF4FF0010E9F
:10A7080026E718BFBE467FF408AF4FF0010E04E7F6
:10A7180018BFBE467FF4E6AE4FF0010EE2E618BF62
:10A72800BE467FF4C4AE4FF0010EC0E618BFBE4669
:10A738007FF4A2AE4FF0010E9EE618BFB8467FF434
:10A748007FAE4FF001087BE608231370B0E70723BC
:10A758001370ADE7C432002067666666A81500204E
:10A7680090610020716600083D6700086461002060
:10A778002DE9F843974D2C68E00500F1CB80964A07
:10A78800964B92F85880964F00221A70B8F1000F35
:10A7980000F0B08006219348FAF730FF002800F057
:10A7A800A48044F01004904A904B16682C6016F46C
:10A7B8008056B3F9069060D18D4B9B8A4B4570DC6F
:10A7C80044F040048B4B2C601B78190706D41B21DE
:10A7D8008448FAF713FF002800F0BE8024F08004B4
:10A7E800B7F84A35642BB7F84C358CBF44F480640D
:10A7F80024F480641BB1804B1B689A0704D47F4BF8
:10A80800D3F8AC30002B4FD044F400647C4B2C6060
:10A8180003F1780102E006338B4216D01A781C2A1D
:10A82800F9D19878DA78904202D35A79002AF2D08E
:10A838001C216C48FAF7E2FE20B1724B1B785B07CB
:10A8480040F1918044F400742C601F216548FAF7A8
:10A85800D5FE60BBB8F1000F2FD0002C43D10023E8
:10A8680087F84E3510F0C0FCD7F85035C01A0028CC
:10A878003EDBBDE8F8430CF083BB15215948FAF7D5
:10A88800BDFE002898D197F87834002B94D1584B06
:10A89800B7F872245B8A991A494591DA13444B45F3
:10A8A8008EDD24F040048DE724F40064AEE744F420
:10A8B80080342C60B8F1000F15D1534B1B78002B56
:10A8C80036D19846002E3DD100214648FAF796FE2B
:10A8D800002851D0002CC2D0B8F1000F03D1002EAF
:10A8E80045D0002844D00223BAE724F010045AE7E0
:10A8F800BDE8F883454A97F8483516787BBB7EB3A0
:10A9080041463848FAF77AFE002850D124F0080466
:10A918002C6025E03E4A3F4B91791A684FF47A73D0
:10A9280003FB01F393429CBF24F480742C6026E758
:10A9380024F4801828F40068B8FA88F84FEA581800
:10A94800002EC1D015212748FAF758FE18BB97F8F2
:10A95800783483B30646B7E744F0800440E796BBF3
:10A9680087F8486516E724F400742C606DE7A0B9F1
:10A9780024F480142C6070E724F020040146194860
:10A988002C60FAF73BFE64B900287FF468AF24F422
:10A9980080142C6061E7002696E744F480142C604C
:10A9A800A1E7B8F1000F9CD1002E9AD1DFE744F05F
:10A9B80008042C60D4E724F4801626F04006B6FA82
:10A9C80086F6760980E741460648FAF717FE00281A
:10A9D800C6D19BE7AC3000202C000020B628002010
:10A9E800A8150020703B0020344E0020243300209E
:10A9F80064610020B8280020C4300020AC47002043
:10AA0800603F0020B7280020BC3B00205C390020B4
:10AA1800A4630020984500202DE9F047BD4E337807
:10AA2800002B40F08280BC4D2B78DB0723D4FFF746
:10AA38009FFEBA4B1A6852BB2B78DF0701D5BDE8D9
:10AA4800F08710F0D1FBB64BB64A1B68C31A934285
:10AA580080467FD8DFF8E092D9F80030002BEED19D
:10AA68001B21B148FAF7CAFD002800F0058102232E
:10AA7800C9F80030E3E7AD4AAD4B1178186801F02A
:10AA8800010111F033FCA54B1A68002AD4D0A94B58
:10AA9800A9491B780020086023B1A84BD3F8AC3033
:10AAA800002BCCD1A64C002A92FAA2F3B3FA83F376
:10AAB800D4F85C2508BF4FF0FF3301339A42BED06B
:10AAC800A04AC4F85C35DBB2A2FB0312920802EB81
:10AAD80082015B1A4FF0053043F20525DBB202F024
:10AAE800FF01C4F86C05C4F87005A4F87455002A71
:10AAF80000F091811920012984F8760579D08A1E01
:10AB0800D2B20732520084F877050C2104F26C5552
:10AB180068544E1C0231914205EB010700F0A580F4
:10AB2800402907F8010CF3D172E0824A1378002B10
:10AB38007FF479AF8449854B488B1C687F4942F282
:10AB4800107303FB00F30120B3FBF4F31070C1F89A
:10AB5800AC3068E77E4B1B78002B40F09680DFF81E
:10AB6800D8917C4FDFF80CA2754C9AF80030002B76
:10AB780000F0B68028787849784B40F003022A70B4
:10AB880000220A70C9F8002002E006339F420CD068
:10AB98001A781C2AF9D19978DA78914202D35A792D
:10ABA800002AF2D040F007032B70FBF7AFFB737855
:10ABB800DFED6B6A07EE103A07EE908AB8EEC77AB7
:10ABC800F8EE677A674BE7EE267A00251D800520A8
:10ABD800FCEEE77AC4F85C5517EE903AC4F858359D
:10ABE8000CF01EFCC4F86055C4F86455C4F86855E8
:10ABF80025E7322284F877250C22002B00F0878085
:10AC0800A1180526012B81F86C6502F1010108D114
:10AC18000C44FF2384F86C350E20BDE8F0470CF097
:10AC2800FFBB6018911C19253E2980F86C55EFD898
:10AC38006018022B02F1030180F86C65E8D06018F7
:10AC4800111D3E2980F86C55E2D86018032B02EBE1
:10AC5800060180F86C65DBD02144931D3E2B81F8FA
:10AC68006C5540F2E2801946D2E7264432203E294C
:10AC780086F86C05C1D9CBE73B4B1B78DD0640F164
:10AC880095800123C9F80030D9E6344B03F17807E1
:10AC980002E006339F4234D01A781B2AF9D19978FA
:10ACA800DA78914202D35A79002AF2D01B211E4841
:10ACB800DFF88490FAF7A2FC2C4B1B6803F480534E
:10ACC800002840F09580D9F80020022A00F09080F2
:10ACD800DFF8A0A08AF80000002B00F09E80184C36
:10ACE800214B1B78D90647D5D9F80030032B7FF4C0
:10ACF80041AF1F4B1A78002A7FF43CAF01221A702B
:10AD080038E7DFF83490DFF86CA00D4C2DE71146DA
:10AD18007EE700BFBC3B0020B7280020AC300020F5
:10AD2800BC3000207F4F1200703B00200C470020F1
:10AD380010470020753D0020B8300020AC470020A7
:10AD4800A8150020CDCCCCCC744700209C4700200F
:10AD580032530020D83F002013330020603F0020EA
:10AD68000024744920330020B8280020344E0020E5
:10AD7800C0300020B62800202E4B93F85830002B06
:10AD8800B2D127212C48FAF739FC0028ACD02B4B3C
:10AD98001B68DA0603D52A4A1278002AA4D0DB04F5
:10ADA800A2D4284B1B88002B9ED1A2E7214B93F8F5
:10ADB8005830002B7FF465AF27211F48FAF71EFC97
:10ADC80000283FF45EAF1D4B1B68DC0604D51C4A07
:10ADD8001278002A3FF455AFD8043FF552AF194B0B
:10ADE8001B88002B7FF44DAF0323C9F8003026E6FB
:10ADF800DFF85CA0144C012100228AF8001084F8C6
:10AE08005425002B7FF4B6AE104AFF201178152286
:10AE180008F090F9A9E60A22EFE60C4A0A4C1178E4
:10AE2800FF20142208F086F99FE62344D11D83F8F9
:10AE38006C65EDE62C000020703B0020344E0020AD
:10AE48004A2D0020482D0020A815002090600020E1
:10AE5800B6280020334A344B10B5B2F906401B68B7
:10AE6800B4F5FA6FA8BF4FF4FA64B4F57A7FB8BFA7
:10AE78004FF47A74DB0410D42C4B9B8A6420E41AB8
:10AE880000FB04F0C3F5FA6390FBF3F06428A8BF55
:10AE9800642020EAE07040B210BD15212448FAF77A
:10AEA800ADFBC8B9234B93F878040028E4D11F49B7
:10AEB800B3F872244B8A9918A14226DB9B1AA34245
:10AEC800EADD1C1B6FF06300A3F57A7300FB04F046
:10AED80090FBF3F040B210BD144A164B908A93F8D9
:10AEE8007824241A6423C0F5FA6003FB04F494FB65
:10AEF800F0F49C42A8BF1C4624EAE474E0B212B104
:10AF0800404240B210BD60B210BDE01A841AC3F5C9
:10AF1800FA6364209B1A00FB04F090FBF3F040B244
:10AF280010BD00BF24330020344E0020646100208F
:10AF3800703B0020A8150020874A1378D80700D452
:10AF480070472DE9F04123F00103844C137010F091
:10AF58004BF9834D2378C5F8B0051BBB814B1B7893
:10AF6800012B1FD0804B9A781ABB804B1B88002B73
:10AF780057D17F4A7F4B1178186881F0010111F091
:10AF8800B5F97D4E33782BB123781BB17B4B1B6809
:10AF9800D90467D57A4B1B68002222709A062FD5F0
:10AFA800BDE8F081774B01221A706F4B9A78002A1E
:10AFB800DBD01B79022BD8D0734E33780B2B18D8E3
:10AFC80001229A4040F6030112EA0107CDD112F49A
:10AFD800C06F0ED0093B012B0BD845201DF0C8F9D6
:10AFE800FF201DF0C5F969481DF0AEF938461DF07F
:10AFF800BFF9674A674B12685A600B233370B4E78E
:10B00800D5F808369B0300F19C80634900220B4663
:10B018001878042803F10C030CD00132192AF7D14F
:10B02800BEE75E4B5A69002AABD0196800220A6055
:10B038005A74A6E7D5F81446530044B158486478C2
:10B048009E1800EB860090F87900A042A8D21A4416
:10B0580001EB82010023C5F81416A5F81836C5F8C7
:10B068001C369DE74F4B1F7810F0BEF83378002B45
:10B0780090D095F8B48595F8B53508F1010202F03D
:10B0880003029A4286D04FEA880606EB080105EBD0
:10B09800810100F51C50103085F8B4250A234FF4BF
:10B0A8007A72C1F8B805C1F8BC2581F8C135002FFE
:10B0B80050D014213C4811FB083318443A4625F077
:10B0C80026FE3A4A1389012FB3FA83F34FEA531342
:10B0D8002ED0B2F86C10002918BF0023022F27D0F9
:10B0E800B2F8D010002918BF0023032F20D0B2F8DF
:10B0F8003411002918BF0023042F19D0B2F8981171
:10B10800002918BF0023052F12D0B2F8FC1100291E
:10B1180018BF0023062F0BD0B2F86012002918BF01
:10B128000023072F04D0B2F8C422002A18BF002336
:10B1380083F0010306EB080205EB820282F8C035B2
:10B1480028E71B4B1B78032B7FF45FAFBDE8F0416A
:10B158000CF04AB93B46EDE7B7280020B628002096
:10B16800A8150020C0300020042D00201C47002016
:10B178001E4700202047002032530020344E002074
:10B18800AC300020133300203C380020185403084A
:10B19800984500209C3B0020EC1003082447002021
:10B1A8007410030890600020601B002044530020A6
:10B1B800CC2C00202DE9F04FC24B2DED028B1B68E3
:10B1C800DB0495B0044600F12587BF4B1B78022BA2
:10B1D80000F02E87042B00F03483012B00F0CE8280
:10B1E800BA4B0493DFF834B3B94B0693B94BBA4A58
:10B1F8009C42927800F2F782002A40F0F782B74B1F
:10B208000793B74B0593AF4B1E68049BF704B3F93C
:10B21800065000F16182069B9B8AAB42CCBF002599
:10B228000125FFF717FEAF4B0A931A78059BAE4F1F
:10B238001B78397880EAE07CACEBE07CCDF804C080
:10B248005FFA8CF903F00103002A40F06F824FF097
:10B25800000C8BF828C6002D00F0FE8501254FF064
:10B26800000E4FF0010C8BF819E38BF818C3DFF8C8
:10B27800B0C29CF800C0002B00F04884DFF8A4821C
:10B2880098F801E0BEF1000F05D09BF854E5BEF137
:10B29800000F00F09187954A0B92BCF1210F07D15E
:10B2A800934A00205060002B02F0E980854B1E680D
:10B2B800012901F0CE818F4F9FED8F7A7B7807EEC1
:10B2C800903AF8EEE77AF20667EE877AFCEEE77ACC
:10B2D80004D58A4A1278D10641F17F80884B0293BF
:10B2E80017EE903A1C44CBF85845864B1B78002B38
:10B2F80040F0D582069B049A998AB2F90000DA8A4E
:10B308008142B4BF8023002382420498B0F902002E
:10B31800C8BF43F040039B088142BCBF63F07F0372
:10B32800DBB282420498B0F90400C8BF43F040037E
:10B338009B088142BCBF63F07F03DBB28242049862
:10B34800B0F90600C8BF43F040039B088142BCBF68
:10B3580063F07F03DBB282429BF82B26C8BF43F021
:10B3680040039A4201F0B481079A8BF82B3692F881
:10B3780058100022ABF82C268BF83426002901F04F
:10B388005A815F2B00F08B826F2B00F088825E4B16
:10B3980000221A60059A4B4B12781B68D40703F0F9
:10B3A800040307D49BF8342622B9BBF92C26322A89
:10B3B80001F34582002B40F07982DBF8FC240192EE
:10B3C8000DF1340900230D93CDE90F331293C9F819
:10B3D8000430002A4FF0004311934CDD11AB4B4E63
:10B3E8009FED4B8ADFF82CA10393CDF820B01AF813
:10B3F800015B03984FEA450808EB050416F814B0FA
:10B4080006EB440459462746FAF7F8F8002840F0B6
:10B418007082BBF1270F26D8A378E1788B421CD223
:10B428006278049C043240F6330534F91220AA42AB
:10B43800A8BF2A46B2F5617F4FF0190440F2833560
:10B44800B8BF4FF4617214FB0353934205DA14FB3F
:10B4580001509042B4BF00200120034638464A46B6
:10B468000FA9FCF785FA2B4B019AAAEB0303934229
:10B47800BDDBDDF820B0DBF80075002F54DD264D6C
:10B48800224E2F4415F8014B04EB440306EB43030B
:10B498000FA893F805A05146FAF7B0F85146804630
:10B4A8004846FAF7ABF804EB440488EA0003DBB239
:10B4B80006EB44004A460FA9FCF75AFAAF42E1D11D
:10B4C80032E000BF344E0020B23800202433002080
:10B4D80064610020404B4C00E02C00202C00002030
:10B4E800B72800204A2D0020C0300020B6280020B0
:10B4F80008270020BC3B002000247449B8280020FD
:10B50800482D0020C0330020B8300020603F0020C4
:10B518008096984AC01A0020AC1A0020A81500206E
:10B5280004270020AC3B00200DA80FC842404B4028
:10B53800CDE90D23854A864B126899E8030083E814
:10B548000300530240F1FD820B9B0A9A1B780120ED
:10B558001070002B40F0FE827E4B1C78002C00F00F
:10B56800018301217A48FAF749F8029B1C880028D0
:10B5780040F00A82784BDB78002B40F00582774D4B
:10B58800029E24F001039BB2A34233800AD041F209
:10B598000242FF230E20ABF86C258BF86E350BF0BA
:10B5A8003FFF34886A480221FAF728F823B20028B6
:10B5B80000F0F38123F001039BB2029EA342338083
:10B5C8000AD041F20242FF23ABF86C250E208BF81B
:10B5D8006E350BF025FF3488A30740F1DD86604AFD
:10B5E800604B11785868A70701F0020100F0F68156
:10B5F800003118BF012110F079FE079A4FF4FA6361
:10B60800C2F870311C215248F9F7F8FF30B9059A91
:10B6180013785E0744BF23F0040313702B68029A63
:10B6280013F00A0F148812D004214948F9F7E6FFED
:10B63800002800F05985650641F12B80092144480E
:10B64800F9F7DCFF002840F02A85029B1C88404857
:10B658000521F9F7D3FF002800F01E8244F4807317
:10B66800029AA342138009D041F20242FF230E201E
:10B67800ABF86C258BF86E350BF0D2FE3A4B1B7885
:10B68800082B00F016820E2B00F013822F4B1B683C
:10B69800580500F12682059B1B78D90700F1B38174
:10B6A800324B1D78002D00F0008708212848F9F753
:10B6B800A5FF002800F0BF819BF81D30834203D00E
:10B6C8002B4B4FF07E521A608BF81D00012015B0ED
:10B6D800BDEC028BBDE8F08F15211D48F9F78EFFF0
:10B6E80000287FF498AD9BF87834002B7FF493AD55
:10B6F800069BBBF872245B8A991AA942C1F298800A
:10B70800FFF7A8FB1B4B0A931A78059B1A4F1B7867
:10B71800397880EAE075A5EBE07501955FFA85F95F
:10B7280003F00103002A01F0E6840125002B00F054
:10B73800B384012900F02D86069A127F4A4501F24A
:10B74800398001228BF8282689E500BF344E002075
:10B75800703B0020912D0020E02C0020C4300020F8
:10B768000C47002010470020603D002000300020DA
:10B77800C00700204A2D0020C0300020DFF810B399
:10B78800DBF82036E31A002B66DBAD4AAD49527C64
:10B79800AD4B069133F81230497C04F59C422032B7
:10B7A8009B08CBF8202619B1C3F57F7303339BB2EE
:10B7B800A648A7490278A74D31F8126021F812303F
:10B7C80029689B1B0B44A4492B601B0901320B8081
:10B7D800A24B049302F00F02A14B0270A14A9C42B3
:10B7E80092787FF609AD002A00F0CE859E4B9D4ADF
:10B7F8001E780593062092F82150FEF749FD06F0C1
:10B808000107824620B19BF80A30022B00F0FA8229
:10B81800012D40F0F7824FF00008924B934A93F8BD
:10B828002030934EDFF86C920792062B00F22F849B
:10B83800DFE813F0B60237064D0260026D0282029D
:10B84800D802DFF84CB20FF0CFFCDBF82436894A77
:10B85800C01A904200F3A784804B0493794B069357
:10B86800C4E49E2903D10021012025F041F99BF869
:10B878002B369D2B03D10021FF2025F039F99BF8A9
:10B888002B36AE2B03D10121002025F031F99BF88E
:10B898002B36AD2B03D1FF21002025F029F9764B5B
:10B8A8001B6803F00403002B3FF487AD9BF8383680
:10B8B8005BB1059B1B78DA0707D5049BB3F9062013
:10B8C800069B9B8A9A4200F3FB870D216B48F9F788
:10B8D80095FE002800F03C849BF83C362BB99BF879
:10B8E800363613B93223ABF83A3601238BF83C3697
:10B8F80063E559466148F9F781FE0346002860D19F
:10B90800A17894F803C061451CD26078049A043089
:10B9180040F6330E32F910007045A8BF7046B0F5F6
:10B92800617F4FF0190440F2833EB8BF4FF4617055
:10B9380014FB01E1814205DA14FB0CE38342B4BF36
:10B948000023012359464E480993F9F757FE099BEE
:10B9580000287FF483AD01930FF046FC07EE900AB0
:10B96800F8EE677A019BF4EEC87AF1EE10FA06DB7E
:10B978002BB94544424816F81510F9F72FFE089BD5
:10B98800D3F8FC3401936EE53E4D2B6899077FF59B
:10B99800F7ADE20740F1868623B223F002039BB29B
:10B9A800029EA34233803FF41AAE41F20242FF23C3
:10B9B8000E20ABF86C258BF86E350BF031FD348812
:10B9C8000DE659460FA8F9F7F9FD21784846F9F729
:10B9D80005FE089BD3F8FC34019344E5B1FA81F1E4
:10B9E800490910F083FC079A42F21073C2F87031CB
:10B9F80008E6059B1B78DB0740F14D829BF8283849
:10BA0800002B00F03585069B1F4A93F8253001214D
:10BA18008B4211707FF449AE1C4B1B78002B7FF4CE
:10BA280044AE17200BF0FCFC08211448F9F7E6FD9A
:10BA380000287FF441AE104B1868C0F300703BE655
:10BA4800DC4600206461002004470020B338002051
:10BA5800B4380020D4380020D838002024330020FF
:10BA6800404B4C00E02C0020B72800202C00002080
:10BA78009845002060E31600344E0020703B0020FB
:10BA8800E81B0020C430002000300020BC600020EB
:10BA9800A8150020AC30002024F480739BB2029AD1
:10BAA800A34213807FF4E0ADAD4B1B78082B7FF4E5
:10BAB800EAAD02990A8822F040039BB29A420B80B1
:10BAC8003FF4E4ADFF2341F202420E208BF86E35BD
:10BAD800ABF86C250BF0A4FCA24B1B6858057FF54E
:10BAE800DAADA14A02F17800134603E00633834237
:10BAF8003FF47FAF19780F29F8D19C78D9788C4218
:10BB0800C0F0C98159790029F0D0C4E1BCF1210FF6
:10BB180001F0DD84954B0B93022900F0AA850023E0
:10BB28003B70934F9FED937A7B7807EE903AF8EE4F
:10BB3800E77A914B029367EE877AFCEEE77AFFF794
:10BB4800CFBB0B9B0A9A1B78C0F300501070002BD8
:10BB58003FF402AD14200BF063FC884B1C78002CDA
:10BB68007FF4FFAC07988649864BC56D864A0968FD
:10BB78001B7808916F1CD2F80090019300F0298679
:10BB8800002D3EDDDFF810A20A275544AAF5967865
:10BB980001261AF8011B01EB81040BEB440417FB87
:10BBA8000161414494F84C06FAF734FD38B3B4F80F
:10BBB80052C6BCF1000F22D194F8510694F84F36C2
:10BBC80000EB40010BEB8101013BD1F8BC2703924C
:10BBD8006E4A03EB43031344039A93420FD09BF836
:10BBE800E82794F8504681F8B84706FA00F022EAA8
:10BBF8000000C1F8BC37C1F8C0C78BF8E807AA45F0
:10BC0800C7D1634CDFF894A100256368002B00F0CE
:10BC180077811F78002F00F07381A268A9EB0202D8
:10BC2800002A0ADB9BF8E8270121A94022EA010241
:10BC380009F5FA718BF8E827A160019A002A00F04B
:10BC48005F81227859780432D2B2002940F03981D4
:10BC580006990498498A30F912009BF8E82701F1FF
:10BC6800C80C604540F382832A41D60793F80280C6
:10BC780000F14681B8F1000F0CBF012002200BF043
:10BC8800BFFC7B1E1F2B00F2B086DFE813F0D30643
:10BC9800B1062307F506A3067E062F081D08090826
:10BCA800F507E107AE06F506DF077E062F081D0833
:10BCB800DB07C507AF079A0786076F07AE06D306E7
:10BCC8006D07B1066B07AE06860753073D07002DC3
:10BCD80040F01E82002F40F022822E4A33685269BB
:10BCE8009A4280F026822B4947F230520323CA61D8
:10BCF80081F8203002200DF005FBFFF71DF92549DA
:10BD08003268CB69134404228B6181F82020002D0E
:10BD180001F06F821F4A336892699A4280F0B781B6
:10BD2800079B93F85800002800F03382D9F80030B8
:10BD380023F00203C9F800303268BBF806306421EA
:10BD480001FB0323134900224FF480600B6181F843
:10BD58002020CA700DF0A6FA0E4991F8203064E54B
:10BD6800603D0020344E0020603F0020B6280020AF
:10BD7800BC3B002000247449482D0020912D002050
:10BD8800C43200205C3900209845002018120308AE
:10BD9800601D0020E02C0020201D00205C330020C6
:10BDA800002F00F06981FEF7D3FA012800F008831C
:10BDB800BAF1000F40F0DE81002D40F06881BD4AE5
:10BDC800336812699A4225D29BF80B30022B21D096
:10BDD800FAF7FCFCB749032240F6B83381F8202073
:10BDE800CB6187E765B3B34A052382F82030002F7B
:10BDF8003FF479AFFAF7D2FCAE4B4FF0030893F853
:10BE0800203012E516F002053FF405AD00254FF08D
:10BE1800020802E5A74A012382F820309BF80B307C
:10BE2800012BD5D0C1F00881022BF7D1FAF7CEFC4F
:10BE3800A04A40F6B8334FF0060182F82010D361CB
:10BE4800002F3FF450AFFAF7A9FC4FF00308404623
:10BE58000BF0E6FAFFF7D7B901293FF400AA964D8F
:10BE68002D6895F82C504FF0010C8BF819C3002D54
:10BE780000F0AB848BF818C30025FFF7F8B9917868
:10BE8800D3789942C0F0E8825379002B40F0E482DD
:10BE98000632824205D013780F2BF0D00632824248
:10BEA800F9D19BF82838002B3FF4F5AB16F090FF3A
:10BEB80016F078FC0BF024FA00238BF82838FFF7EB
:10BEC800EABB012915D19978049B0C2F33F912305C
:10BED80001F0E880B3F5617F80F21C85182F01F02E
:10BEE8004F81222F05D19AF8033013B100238AF825
:10BEF80003309BF8E8270123AB4013438BF8E8375E
:10BF08000135042D04F10C047FF47FAE019B002B56
:10BF18003FF427ABDBF84886B8F1000F7FF721AB79
:10BF2800664FDDF8109004E0644BFB1A4345BFF6FA
:10BF380018AB17F8011B01EB81040BEB44040BEB66
:10BF4800410694F85036B6F9EC270433DBB239F9D8
:10BF580013A05245E8D0B4F85236002BE4D094F838
:10BF68004F56574A013D05EB4505154495F8A5215F
:10BF7800002AD9D10193534B94F84C060A2202FBAC
:10BF880001310131FAF746FB019B0028CCD0DFF8DC
:10BF980028810899B4F85426A6F8ECA7D8F8000028
:10BFA800002900F0DA86002800F0D786AAF2DC5AC9
:10BFB80002FB0AFA444A95F8A45182FB0A124FEA96
:10BFC800EA74C4EB62146A1E1C441F2A00F2C58678
:10BFD800DFE812F0A406E206C9062108B407110832
:10BFE8000307A507930781076F07C30621086007A2
:10BFF80011080307A5074C074A073607FD07D707A7
:10C00800C507C306A406C307E2063008C306D70758
:10C018002E08230700212D48F9F7F0FA00287FF4AD
:10C02800D4A8FEF789FF2A4B1B78022B7FF4D2A8ED
:10C03800284A2949D37B0692013B527C049131F965
:10C0480013301AB1C3F53B6308331BB2A3F57A73F7
:10C0580007EE903A9FED217A214ADFF888B0F8EE92
:10C06800E77A67EE877AFDEEE77A17EE903A83F380
:10C078000A031380FFF7BAB84FF48060BAF1000FD3
:10C0880001F0E9800DF026F90A4A00231361B8F19E
:10C09800000F3FF4B8A8DAE60122FFF7D8B8FAF79C
:10C0A80035F900283FF4D1AA0A200BF0B9F9FFF7B7
:10C0B800CCBA00BFE02C0020C82C0020401D002076
:10C0C80074100308F41B0020D34D6210703B00204D
:10C0D800B23800206461002024330020AAF1823F96
:10C0E800D8380020A815002024F040039BB2029AFB
:10C0F800A34213803FF4A2AA41F20242FF230E207A
:10C10800ABF86C258BF86E350BF08AF9FFF796BA09
:10C11800C54A052382F82030002F3FF4DEADFAF738
:10C128003DFBC14A336852699A424FF00308FFF455
:10C13800DAAD9BF80932002B7FF4D5AD002F3FF420
:10C14800D2AD002DA3D0B84B93F82030FFF76DBBCC
:10C158009BF83636002B3FF430A9059B1B7813F06B
:10C1680001037FF42AA901228BF836368BF837268B
:10C17800FFF723B99BF80A30012B7FF41DAEFAF7BD
:10C1880025FBA94903224FF47A7381F82020CB615B
:10C19800B0E5FEF77DF800283FF4C8ADB8F1000F10
:10C1A8003FF431A853E6A14AA14B0492A14A069252
:10C1B80000221A80FFF71AB89F480B9090F800E009
:10C1C800BEF1000F7FF469A89BF829E6BEF1000FC5
:10C1D8007FF463A8DFF87CE29EF800E01EF0100F01
:10C1E8007FF45BA8DBF860350393F00600F1CC8799
:10C1F80098F8042053004B2BA8BF4B23DBB24A45C9
:10C20800089363D8049B069AB3F900608B4BB2F885
:10C2180012E093F800A05B7802936FF47A72B31877
:10C228009BB240F2E6329342CEF5FA6052D80EEB5A
:10C238000A03B342099381F25B80A6EB0E036422E2
:10C24800A3EB0A0302FB03F3A0EB0A0293FBF2F34E
:10C25800DBB20E2B3ED8049BB3F902606FF47A73FD
:10C26800F3189BB240F2E632934233D8099B9E42C0
:10C2780041F35E80A6EB0E03A3EB0A066423A0EB52
:10C288000A0203FB06F393FBF2F3DBB20E2B21D871
:10C29800049BB3F904606FF47A7A06EB0A039BB245
:10C2A80040F2E632934215D8029A0EEB02039E4200
:10C2B80041F32E80A6EB0E039E1A6423821A03FB19
:10C2C80006F393FBF2F3DBB20E2B03D8089B4B4526
:10C2D80000F260875A4BDFED5B7A93ED097AB0EE96
:10C2E800C77AB4EEE77AF1EE10FA40F1538793ED8E
:10C2F800047AB0EEC77AB4EEE77AF1EE10FA40F1BC
:10C30800498793ED0E7AB0EEC77AB4EEE77AF1EE8C
:10C3180010FA40F13F87039B0BB9CBF86045019BAE
:10C32800B8F80260DBF860054A2BDBF86435C8BF53
:10C3380076084FF47A721B1A03EB040E02FB06F21E
:10C34800964502D901238BF85435002800F02D8733
:10C35800BCF1210F7EF4AAAF3B4B3C48A3FB0E2354
:10C368009B090122C3808280FEF7A0BFC83988429A
:10C3780080F269862A41D00793F802803FF5C0AD64
:10C38800C8F1000801207AE4274A01239370FFF7D7
:10C398002DBA0A46FEF75BBF44F00203029EA34291
:10C3A80033803FF41CA941F20242FF23ABF86C250D
:10C3B8000E208BF86E350BF033F83488FFF70FB981
:10C3C8003268BBF80630642101FB0323164A136167
:10C3D800BAF1000F3FF4F0ACCCE6F2043EF57EAFC4
:10C3E8000A9B1A781A4B0293002A7EF479AF1A88AE
:10C3F80013053EF575AF079B93F85820002A00F007
:10C408004E87002D40F0D88717EE903A23B1DBF81D
:10C4180058359C4201F22D8010200BF001F80123C1
:10C428008BF82A36FEF761BFE02C00202433002069
:10C43800D838002064610020B6280020B43B0020D2
:10C44800C43E00200000C842D34D621008270020D7
:10C45800482D0020B82800200F21C348F9F7CEF84E
:10C4680000283FF41EAD9BF82838002B7FF413A951
:10C47800BE4C94F8DA30002B40F07E8294F8B63146
:10C48800002B40F06F8294F89232002B40F06082CB
:10C4980016F09EFC16F086F901238BF82838FFF772
:10C4A800FAB8002D7FF448ACB8E4B14B1B68002BF8
:10C4B8003FF4FBA8079BAF499BF82C0893F860450D
:10C4C800FAF7A8F8002862D0002C50D1AA499BF8A6
:10C4D8003108FAF79FF8002840F0A586A7499BF88D
:10C4E8003608FAF797F8002863D0022C40F09F86A8
:10C4F800A3499BF83B08FAF78DF8002840F0A3867B
:10C50800A0499BF84008FAF785F8002863D0042C66
:10C5180040F095869C499BF84508FAF77BF8002877
:10C5280040F0898699499BF84A08FAF773F8002879
:10C5380063D0062C40F08B8695499BF84F08FAF794
:10C5480069F8002840F0E48392499BF85408FAF708
:10C5580061F8002863D0082C40F0DD838E499BF8F1
:10C568005908FAF757F800283FF49FA809252B46E1
:10C5780003EB83035B440799884A81F8605593F875
:10C588002D1893F82E3811705370FFF78EB87A492A
:10C598009BF83108FAF73EF800289FD0012C40F0AC
:10C5A800428676499BF83608FAF734F8002840F0B6
:10C5B8003E8673499BF83B08FAF72CF800289FD071
:10C5C800032C40F040866F499BF84008FAF722F8A0
:10C5D800002840F034866C499BF84508FAF71AF8A9
:10C5E80000289FD0052C40F0268668499BF84A0809
:10C5F800FAF710F8002840F02A8665499BF84F089A
:10C60800FAF708F800289FD0072C40F08183614989
:10C618009BF85408F9F7FEFF002840F07C835E4938
:10C628009BF85908F9F7F6FF00283FF43EA8092CB3
:10C638003FF43BA89AE700214B48F8F7DFFF0028B2
:10C6480000F0838000238BF83536FEF7E5F9FEF716
:10C65800A1BE534B1B6893F867304B45BEF42BAE15
:10C66800504B002202215A609A61DA623970FEF753
:10C6780022BE4B4B1B6893F86A30002B3FF451AA3B
:10C6880027213948F8F7BAFF00287FF44AAAFFF7AC
:10C6980046BA44F04003029AA34213807FF42CADBB
:10C6A800FEF7CCBF44F00103029AA34213803FF483
:10C6B80073A9FF2341F202428BF86E350E20ABF8C6
:10C6C8006C250AF0ADFE029B1C8823B2FFF765B902
:10C6D800DBF830063449C469BBF92C5681FB0401E8
:10C6E8008911E417601A00F5FF407F30854240F356
:10C6F800B584079991F8581000299CD05F2A00F05A
:10C70800ED806F2B7EF443AEB5F5FA7FFFF6C7A830
:10C718009BF83426002A7FF4C2A8059B1B780121C8
:10C72800DD078BF8341600F1EA84FEF775F91F4B24
:10C738001B68002B00F04D851D4B1B6803F004039C
:10C7480000228BF83426FEF735BE059B174A1B7866
:10C75800CBF85C05DE07106000F18784144B1B687A
:10C7680003F00403FEF71EBE703B0020EC4E0020D1
:10C7780004300020D71D0020DC1D0020E11D002012
:10C78800E61D0020EB1D0020F01D0020F51D0020F7
:10C79800FA1D0020FF1D0020041E0020D42C0020BC
:10C7A800C82C0020C43E0020D34D6210B8300020B1
:10C7B800344E0020002D40F07E869BF82826002A63
:10C7C8007EF44DAD0122FFF74ABB8BF81853FEF7F4
:10C7D8004EBD11AE1194B64DC4650746CBF8484618
:10C7E800746034810BE0FB6D0BEB0301013381F8BE
:10C7F8007827FB6501341E2C05F10A0514D00A229E
:10C808003146284624F050FA0028F3D0EB88E2B2EB
:10C81800002BE8D0DBF848360BEB0301013381F835
:10C828009827CBF84836E5E7079BDD6DFFF7A8B9F1
:10C838001344AB42CCBF00250125FEF7F2BC9D4A4C
:10C84800126812F020027EF4B5AD9BF82B16012079
:10C8580057298BF8340600F0D78413B15A2900F011
:10C8680089855D2900F012855E2900F006855B291F
:10C8780000F0FA84562900F0C785972900F0EF8563
:10C88800A72900F0E185029B1B88980740F0C28524
:10C89800A1F1B703072B3EF6E4AF01A252F823F04B
:10C8A8001DD500086BB800086BB800086BB8000805
:10C8B8000BD500086BB80008F9D40008E7D40008C5
:10C8C80000217D48F8F79AFE00287EF4FEAF322357
:10C8D8008BF83806ABF83A36FEF7F7BFB5F5FA7FAE
:10C8E800FEF6DDAF9BF83436002B7EF4D8AF059A00
:10C8F800724912780B60012312EA03048BF834366C
:10C9080000F00A84FEF718FB6D4B1B6803F0040364
:10C91800FEF750BD40F633029342A8BF1346182FC6
:10C92800A3F561734FF4966292FBF1F193FBF1F377
:10C93800DBB200F00684222F7FF4DBAA9AF80320EA
:10C948009A423FF4D6AA012B3FF6D3AAFFF7CFBAF3
:10C95800D4F8B8010AF040FBDC220021594824F041
:10C96800D6F995E5D4F8DC000AF036FBDC22002184
:10C97800554824F0CCF986E520680AF02DFBDC2226
:10C988000021204624F0C3F978E5504A504E10683B
:10C99800B378817B4144C829A8BFC82121EAE17145
:10C9A8008173002B40F0D4840F2F0FD0017AB37815
:10C9B8004144C829A8BFC82121EAE17101722BB1FD
:10C9C80012200392FBF706F8039A1068FBF732FD72
:10C9D800FFF78FBA089A3E4ED17AB378414481F373
:10C9E8000801D172002B40F07C84384B1868EDE7C1
:10C9F800089B374E9979B27841446429A8BF6421CD
:10CA080021EAE1719971002A40F05F841B2FECD074
:10CA1800089AB378D17941446429A8BF642121EAEE
:10CA2800E171D171002BE0D01C20FAF7D3FF274B1E
:10CA38001868CBE7089B264ED978B2784144FF297D
:10CA4800A8BFFF210129B8BF0121D970002A40F0F1
:10CA58008784192FC9D0089AB37811794144FF29DE
:10CA6800A8BFFF210129B8BF01211171002BBCD03B
:10CA78001A20FAF7AFFFB8E7089B154E997AB278F3
:10CA8800414481F308019972002A40F06E840D2F09
:10CA9800ABD0089AB378517A414481F308015172B6
:10CAA800002BA2D00E20FAF795FF084B18688DE7E7
:10CAB800F41B0020AC300020703B0020B830002070
:10CAC800344E0020A4500020C84F0020C82C00205D
:10CAD800042D0020089BAE4E5A789044B8F1640F9C
:10CAE800A8BF4FF0640828EAE87883F80180FDF7CA
:10CAF80071FCB378002B3FF478AF03204146FAF776
:10CB080069FFA44B186861E7A24FA14E3868B37853
:10CB1800018B4144B1F5FA6FA8BF4FF4FA6121EADD
:10CB2800E1710183002B3FF451AF2020FAF752FF47
:10CB380038684BE7974A964E10688189B378414424
:10CB4800B1F5FA6FA8BF4FF4FA6121EAE17181816A
:10CB5800002B3FF43BAF1F200392FAF73BFF039AE9
:10CB6800106833E78A4E53E7894E74E7894F884E39
:10CB78003868B37890F8471041446429A8BF642105
:10CB88000129B8BF012180F84710002B3FF41EAFE0
:10CB98001720FAF71FFF386818E77E4A7C4E10689E
:10CBA800B378418A4144B1F5FA6FA8BF4FF4FA61EE
:10CBB80021EAE1714182002B40F08C831E2FBCD109
:10CBC80004E7089A724E5179B3784144FF29A8BF07
:10CBD800FF210129B8BF01215171002B3FF405AF96
:10CBE8001520FAF7F7FE6B4B1868EFE6694A684EAE
:10CBF8001068817AB3784144C829A8BFC82121EABE
:10CC0800E1718172002B3FF4E1AE14200392FAF730
:10CC1800E1FE039A1068D9E65E4A5D4E1068417AD3
:10CC2800B3784144C829A8BFC82121EAE1714172FB
:10CC3800002B3FF4CBAE13200392FAF7CBFE039AF6
:10CC48001068C3E6534A524E1068AFE6504E20E7CC
:10CC5800504F4F4E3868B378817D4144C829A8BFEA
:10CC6800C82121EAE1718175002B3FF4AFAE0B209A
:10CC7800FAF7B0FE3868A9E6464F454E3868B378EB
:10CC8800417D4144C829A8BFC82121EAE171417505
:10CC9800002B3FF49BAE0A20FAF79CFE386895E615
:10CCA8003C4F3B4E3868B378017D4144C829A8BF42
:10CCB800C82121EAE1710175002B3FF487AE0920F4
:10CCC800FAF788FE386881E6324A314E1068B37840
:10CCD800017C4144C829A8BFC82121EAE171017437
:10CCE800002B40F05C83112F83D16FE6294A284E30
:10CCF8001068B378C17B4144C829A8BFC82121EA7C
:10CD0800E171C173002B40F0D982102F87D15DE605
:10CD180007252B462CE408252B4629E4FF2C1C4E1E
:10CD2800089AB3782146A8BFFF210129B8BF01217D
:10CD3800D170002B40F0AF83192D0CD0FF2C214669
:10CD4800A8BFFF210129089AB378B8BF0121117142
:10CD5800002B40F02B83D8F80000FBF76BFBDBF8C7
:10CD68004886FFF7E1B8642C089B094EA8BF6424E5
:10CD780024EAE4745C70FDF72DFBB378002BEAD04D
:10CD880003202146FAF726FED8F80000E5E700BFA1
:10CD9800042D0020C82C0020642CBF4E089AB378BC
:10CDA8002146A8BF64210129B8BF01219171002B38
:10CDB80040F079831B2DCED0642C2146089AB37895
:10CDC800A8BF642121EAE171D171002BC3D01C20D6
:10CDD800FAF700FED8F80000BFE7AF4EC82C21468E
:10CDE800B378A8BFC82121EAE171C173002B40F0D4
:10CDF8007283102DAFD0C82C2146D8F80000B37824
:10CE0800A8BFC82121EAE1714172002BA5D01320E7
:10CE1800FAF7E0FDD8F800009FE79F4EB4F5FA6FE7
:10CE28002146B378A8BF4FF4FA6121EAE171018382
:10CE3800002B92D02020FAF7CDFDD8F800008CE71F
:10CE4800954ED8F80000B378C82C2146A8BFC82151
:10CE580021EAE1718172002B3FF47FAF1420FAF7C9
:10CE6800B9FDD8F8000078E78B4EC4E78A4ED8F8A9
:10CE78000000B378C82C2146A8BFC82121EAE17177
:10CE88000172002B3FF469AF1220FAF7A3FDD8F81E
:10CE9800000062E7804E089AB37884F30801517263
:10CEA800002B3FF458AF0E20FAF794FDD8F8000095
:10CEB80053E7794EC82C2146B378A8BFC82121EA88
:10CEC800E1718175002B3FF448AF0B20FAF782FD22
:10CED800D8F8000041E7704EC82C2146B378A8BFA7
:10CEE800C82121EAE1714175002B3FF436AF0A20D1
:10CEF800FAF770FDD8F800002FE7674EC82C2146D6
:10CF0800B378A8BFC82121EAE1710175002B3FF46D
:10CF180024AF0920FAF75EFDD8F800001DE75E4E41
:10CF2800C82C2146B378A8BFC82121EAE171017451
:10CF3800002B40F0C482112D83D10CE7564E089A7D
:10CF4800B37884F30801D172002B3FF406AF0520B3
:10CF5800FAF740FDD8F80000FFE64F4EEEE6642CE5
:10CF68004D4E2146A8BF64210129B378B8BF0121DD
:10CF780080F84710002B3FF4F0AE1720FAF72AFD8F
:10CF8800E9E6454EB4F5FA6F2146B378A8BF4FF4E9
:10CF9800FA6121EAE1714182002B40F080821E2D66
:10CFA8003FF4D9AEB4F5FA6F2146D8F80000B3784B
:10CFB800A8BF4FF4FA6121EAE1718181002B3FF4A7
:10CFC800CCAE1F20FAF706FDD8F80000C5E6FF2C06
:10CFD800314E089AB3782146A8BFFF210129B8BF6E
:10CFE80001215171002B3FF4B8AE1520FAF7F2FC7D
:10CFF800D8F80000B1E6284EC82C2146B378A8BF5F
:10D00800C82121EAE1718173002B40F05C820F2D69
:10D018007FF42DAF9FE6204E089AB37884F3080179
:10D028009172002B40F043820D2D7FF434AF92E6CD
:10D03800194EB7E7184EBFE6F9F7C8FB174B93F838
:10D048002030FEF7F2BB0123AB4022EA030209F5C8
:10D05800FA738BF8E827A360FEF752BF091B0D444B
:10D068002DB2ABF82C56FFF744BB0D4B1B78002BA9
:10D078003EF415AC094BDB78002B7EF410AC9BF822
:10D0880035360133DBB2032B8BF835367EF607AC29
:10D09800FDF752FFFEF77EB9042D0020E02C00209A
:10D0A8005C390020CA4A107988B3C821B3F5617F7A
:10D0B80062DB40F63307BB42A8BF3B46A3F5617766
:10D0C80097FBF1F75FFA87F8537843453EF411AFC1
:10D0D800C04E404606F03AFCB378002B40F0BF80C3
:10D0E80008F10107FFB2002F3EF403AF38460AF0FB
:10D0F80087FAFEF7FEBE8BF82826FEF7AFB8B64BC8
:10D10800CBF85C251B6803F00403FEF753B94FF412
:10D11800966797FBF1F1C9E70F200AF081F9AF494B
:10D12800BBF82C260B688BF8344623F020030B60E1
:10D13800A94B1B68FA3AABF82C2603F00403FEF758
:10D1480039B9C82B1A46A8BFC8221946D0B2A44B71
:10D158001F683B7F83423EF4CCAED21A9D4E38778F
:10D1680048BF0732D210B378571CFFB2002BBAD091
:10D178001820FAF72FFCB6E74FF000084746A3E758
:10D18800002001460246E2E7002A7FF431A8002D7C
:10D198007FF42EA8039A2AB1DBF864359B1A23443E
:10D1A800CBF864350023CBF86035BCF1210F7EF451
:10D1B8007DA88C4ADBF864358B48A2FB0323059ACB
:10D1C8009B091278C3800023838002F00103FEF7D5
:10D1D8006AB8824A804B12681B68B2F5006F03F088
:10D1E80004037EF4E7A83A78002A3EF4E3A8FFF7A0
:10D1F800A7BA7E493268CB6913448B61B8F1000F36
:10D208003EF401A8FEF723BE79497A4A4C8B7A4945
:10D21800106842F2107202FB04F2B2FBF0F2C1F89D
:10D22800AC20FEF7C7B801252B46FFF7A1B90225A8
:10D238002B46FFF79DB905252B46FFF799B904251D
:10D248002B46FFF795B903252B46FFF791B906251D
:10D258002B46FFF78DB90CF025F8FEF715BFF9B28C
:10D268000C20FAF7B7FB3BE701200CF031F95A4BD9
:10D278001B6803F00403FEF79DB802200CF028F9A0
:10D28800554B1B6803F00403FEF794B800200CF01C
:10D298001FF9514B1B6803F00403FEF78BB8002DF0
:10D2A8003FF4BAA89BF82A36002B3EF41EA80AF0D1
:10D2B8009BF800238BF82A36FEF717B81020039244
:10D2C800FAF788FB039A10681FE51B20FAF782FB20
:10D2D800FFF79CBB1E200392FAF77CFB039A1068A9
:10D2E8006CE40520FAF776FB3D4B1868FFF76EBB38
:10D2F800AEEB0A02B2427EF7AEAF961B6423A2F5EC
:10D308007A7203FB06F393FBF2F3DBB2FEF7A1BFDD
:10D31800AEEB02029642BEF6D9AF961B6423A2F585
:10D328007A7203FB06F393FBF2F3DBB2FEF7CCBF92
:10D33800AEEB0A02B2427EF7ABAF961B6423A2F5AE
:10D348007A7203FB06F393FBF2F3DBB2FEF79EBFA0
:10D358000F200392FAF73EFB039A1068FFF724BBED
:10D368001920FAF737FBFFF774BB0D20FAF732FBE9
:10D37800FFF78DBB9BF83636002B3FD19BF838362C
:10D3880083F001038BF83836002B7BD10C200AF090
:10D3980047F8114B1B6803F00403FEF70BB8112084
:10D3A8000392FAF717FB039A10689CE41A20FAF71D
:10D3B80011FBD8F80000D0E417EE903A9BF82A2623
:10D3C8001C44CBF85845002A3DF48FAF6FE700BFE7
:10D3D800A4630020042D0020344E0020AC3000202F
:10D3E800C82C0020D34D621008270020E02C002014
:10D3F800744700209C470020AC4700208BF8362655
:10D408008BF83706FEF752BA0DF05EFB9BF82B1629
:10D41800FFF733BA0022A1F1B7031192072B3EF6AA
:10D4280020AA01A252F823F07DD500086BB80008A5
:10D438006BB800086BB8000875D500086BB8000811
:10D448006BD500082FD500084D494E4B0A781B684C
:10D4580042F004020A7003F00403FDF7ABBF494B26
:10D468001B684FF4C87203F00403ABF84C25FDF7B2
:10D47800A1BFFDF761FD8BF82A56FDF736BF397855
:10D48800FEF74ABB0B2009F0CBFF3E4B1B6803F0AD
:10D498000403FDF78FBF1920FAF79CFA4CE41E200D
:10D4A800FAF798FA7BE51B20FAF794FA82E40D2044
:10D4B800FAF790FAB8E501252A46FDF7D0BE112003
:10D4C800FAF788FA37E50F20FAF784FA9FE52E4A2B
:10D4D8000B92FDF7E5BE1020FAF77CFA89E40220EA
:10D4E80006F034FA274B1B6803F00403FDF762BF0C
:10D4F800032006F02BFA234B1B6803F00403FDF707
:10D5080059BF002006F022FA1E4B1B6803F00403E3
:10D51800FDF750BF012006F019FA1A4B1B6803F0FB
:10D528000403FDF747BF0223ADF84430174BBDF89D
:10D53800444059899A89BDF84600214402445981DA
:10D548009A810DF0C1FA0F4BBBF82C261B68FA3AEA
:10D558000021ABF82C2603F004038BF83416FDF7F2
:10D5680029BF4FF6FE73ADF84430DFE70223ADF86C
:10D578004630DBE74FF6FE73ADF84630D6E700BF1E
:10D58800B8280020344E0020B6280020C8300020DB
:10D598002DE9F04FDFF820A3B949DAF86028DAF866
:10D5A800BC34CAF860082DED0E8BA0EB02080D788C
:10D5B80043449DB08146CAF8BC34002D53D0DFF8EF
:10D5C800FCB29BF800509AF86C328BBBAD4BAE4A5C
:10D5D800D3EDE95AD2ED017AD2ED023AC3EDE97AF8
:10D5E80077EEA57A05EE908A92ED034AD3EDEA4AE2
:10D5F80093EDEB5A93ED006A93ED027AD3ED016A4D
:10D60800C3EDEA3AFAEEEF5A73EEA44A34EE055A3D
:10D61800A5EEA76AF0EE477AE5EEA46AE5EE257A6C
:10D6280083ED006AC3ED016A83EDEB4AC3ED027A2C
:10D63800052D00F0F480954ADAF870381178B3FBBC
:10D64800F1F201FB12320133CAF87038002A00F0F7
:10D65800BB809BF80030012B00F0D4801DB0BDECDE
:10D668000E8BBDE8F08F8A4C63682046984704907B
:10D67800002800F0DB80D4F8AC6084F85C50002E01
:10D6880041F0FE80B4F9503094ED085AD4ED095AAF
:10D6980094ED0A6A94F85A1006EE903AB4F95230AA
:10D6A80007EE103AB4F9543007EE903AF8EEE66A0D
:10D6B800B8EEC77AF8EEE77A76EEC56A37EE657A9D
:10D6C80077EEC67A04F12C00C4ED0B6A84ED0C7A6F
:10D6D800C4ED0D7A1CF074FB6E4B1D78002D01F023
:10D6E800DE85DFF8D8B16C4B9BF80050CDF8208070
:10D6F800374604F12C02B8460793174604F5CA7654
:10D708002A461D46B7EC018AD4ED077A142A28EE7A
:10D71800278A02F04382062A08D1B0EE480A069208
:10D7280023F076FA5D4B069A23F8180029688900D9
:10D7380004D594F88416414503F00182B0EE480AF6
:10D74800D4F8902130469047D4F8002206F17000B2
:10D758009047D4F8B020A6F1E0009047D4F82021F3
:10D76800A6F1700090472A689300B0EE408A18D559
:10D7780094F88426424503F0F081D7EDCC7AD4F8AA
:10D78800702277EE887AB0EE480AC7EDCC7A06F1B7
:10D79800E4009047D4F8742206F5A8709047B0EEDC
:10D7A800408A9BF80020032A02F0E38108F101086F
:10D7B800B8F1030F87ED028A06F12406A2D1DDF83D
:10D7C8002080154601F09DBD354B93F85830002B4D
:10D7D80076D0344B3449B3F906208B8A04919A42A7
:10D7E80000F38081314B1B780E2B00F07B81082BD6
:10D7F8002F4B01F069861A46069300239360CAF8F6
:10D80800BC3161E0DAF83026244BD169BAF84A25F0
:10D8180019805A801DB0BDEC0E8BBDE8F08F0DF05D
:10D82800E3FC1E4BA0EB0900188004E7DFF88CB07E
:10D83800D4F8AC309BF8005053B9134BA16BE26B92
:10D8480059609A60216C94F85423D9608AF86C2244
:10D85800184B1B78002B3FF4B6AE162D01F035821D
:10D86800152D41F0A68294ED0E0A0C4E23F0D0F946
:10D8780094ED0F0A308023F0CBF97080A3E600BF47
:10D88800773D0020681A00209C470020AC3B002010
:10D89800AC470020733D0020344E002008270020AC
:10D8A8002C0000202433002064610020603D00200B
:10D8B800E8320020743D0020A8150020042700202D
:10D8C800B44B0493B44B06939AF87428002A40F09A
:10D8D8001081B24B0793B24B0893049E96F825101B
:10D8E800012950D19AF8A438AE4C002B40F06A8137
:10D8F800002096F82A508AF8A418C4F89C004FF61D
:10D90800FF7196F826002370C4F89830C4F8A03048
:10D91800C4F8A410A4F89400002D01F05A8596F8D4
:10D928002710A4F89610002843F0C582002942F079
:10D93800B1879D4E012135788AF8A518002A40F054
:10D94800478105EA01030A9345FA01F30B934FEA6D
:10D95800A508EF10049B93F829100A9B002B01F0EF
:10D96800A385924A92ED007A069B83ED007A0B9B81
:10D97800D80702F1988118F0010300F0938192ED25
:10D98800027A01F083BD357E002D00F0AF81022DB3
:10D9980002F09287032D41F0AB85B37EC3EB4311B0
:10D9A80003EB8103DB009BB2002A01F0BC87002B4C
:10D9B80001F0B9877E4A7C4E1268B3FBF2F319B2C4
:10D9C80007EE901A3478AAF8BC18B8EEE77AF7EEA2
:10D9D800006A14F00108C6EE877A0BD0754B069AD8
:10D9E800D3ED046A92ED007A37EE667A27EE277A4D
:10D9F80083ED007A6710F8070BD56E4B069AD3EDC6
:10DA0800056A92ED017A37EE667A27EE277A83ED7A
:10DA1800017AA510EA070BD5664B069AD3ED066A7C
:10DA280092ED027A37EE667A27EE277A83ED027A4C
:10DA3800E410E3070BD55F4B069AD3ED076A92ED26
:10DA4800037A37EE667A67EE277AC3ED037A9BF896
:10DA58000030072B03F0BA84002940F3C4813478DE
:10DA680004F001086710A510E410B8F1000F0BD0FE
:10DA7800504BD3ED007A93ED047A77EE877AC3EDB5
:10DA8800047A069BC3ED007AF8070BD5494A069B32
:10DA980092ED057AD2ED017A77EE877AC2ED057AB2
:10DAA800C3ED017AE9070BD5424A069B92ED067A47
:10DAB800D2ED027A77EE877AC2ED067AC3ED027A62
:10DAC800E2070BD53C4BD3ED037A13ED017A77EEE1
:10DAD800877AC3ED037A069BC3ED037A9AF8742814
:10DAE800042505E19AF874282B4B0693002A3FF485
:10DAF800F0AE9AF81D30002B3FF4EBAE2F4DBAF87C
:10DB080076382749254C08680891A5FB03539B09DB
:10DB1800642595FBF3F5069B2168D3ED037ADAF8C3
:10DB280078380794BDEEE77A142D448EA8BF1425E3
:10DB3800CE040AEB430117EE106A03F101034CBF50
:10DB4800640824B2A1F87C689D4290F83010CAF8A5
:10DB58007838DCBF0023CAF8783801297FF4BDAED5
:10DB68000AEB4303B3F97C3807EE103AB8EEC77AEC
:10DB780077EEC77AFDEEE77A17EE903A1BB2002BE4
:10DB8800B8BF5B42A34203F37C840D4B4FF07E5138
:10DB98001960A2E664610020E8320020344E0020BB
:10DBA800C82C0020BC60002090610020501E00207E
:10DBB800B8600020681E0020781E0020D34D621037
:10DBC800C0070020B84E23783578002A00F08580F9
:10DBD8009AF8A52815F001010A9103D00698B349CF
:10DBE800006808606910C8070B9103D50698AF490B
:10DBF800406848604FEAA50818F0010F03D006985E
:10DC0800AA4980688860EF10F90703D50698A749E4
:10DC1800C068C860002A41F06F84002B3FF49AAEB8
:10DC28009BF80030292B01F05284049B93F82910AB
:10DC38000A9B002B01F01B849C4A92ED007AD4EDDC
:10DC4800016AD4ED027A002903F06A81D4ED065AFC
:10DC580094ED073AD4ED033A94ED086A94ED044A3A
:10DC6800D4ED094A94ED055A069B84ED067A65EED3
:10DC7800A77AC4ED075AE7EE267A84ED096AE3EE3F
:10DC8800237AE6EE447AE4EEC57AC4ED087AC3ED69
:10DC9800007A0B9BDB0701F1A38718F0010F41F015
:10DCA800CE870123FE0741F1FB83804A92ED037A78
:10DCB800002B01F0F283D4ED1C6AD4ED1D7A002903
:10DCC80043F0FE8037EE667A069BE7EE276AC4EDDE
:10DCD8001C6AC3ED036A01F0E3BB05F001020A9276
:10DCE8006A100B924FEAA508EF1096E7AAF8BC58FD
:10DCF8009BF80030072B70D0002A74D1002D40F01B
:10DD0800B0859BF80070052F00F0E0860024089B82
:10DD180049461868F8F768FE9BF80030052B00F0B4
:10DD2800CE86634B1B7813F0010800F0D980614B55
:10DD38001B78DE0600F1D4805F4B5B78002B00F087
:10DD4800CF809AF854355D4C002B40F0CA80237878
:10DD5800002B40F0C6809AF82936002B40F0C1808D
:10DD6800079B1B68DD0603F17C87554BDFED557A71
:10DD780093ED097AB0EEC77AB4EEE77AF1EE10FACD
:10DD880083F20D8693ED047AB0EEC77AB4EEE77AA3
:10DD9800F1EE10FA83F2038693ED0E7AB0EEC77AAD
:10DDA800B4EEE77AF1EE10FA83F2F9850023CAF8A7
:10DDB80068359BF80030212B40F09B80DAF86835F5
:10DDC8003B49414A0978003318BF01235380012396
:10DDD800138001EA030800F04CBD3B4BBAF8BC18AD
:10DDE8009980002A8AD00223384E394A394D9FED4E
:10DDF8003A8ACDF8289006F1100800241F4691466B
:10DE0800B9EC010ADAF8443520EE080A2046F0EEAB
:10DE1800C00AA6EC010AE8EC010A98472B682F4AC9
:10DE280003EB440302EB84015B8A07EE903AF8EEB9
:10DE3800E77AB1EE677AB4EEC70AF1EE10FA08D4C1
:10DE4800B4EEE70AF1EE10FA8CBFB0EE677AB0EEE6
:10DE5800407A9BF8003081ED007A082B06D1BDEEA0
:10DE6800C00A194A10EE101A22F814100134BC42E4
:10DE7800C6DD072B1F46DDF8289007D1DAED6D7A4D
:10DE8800114BFDEEE77A17EE902ADA80049BDC7ED0
:10DE9800002C40F0B3859AF87438002B3FF433AF68
:10DEA80000238AF874382EE790610020501E002065
:10DEB800B7280020B8280020AC3B0020B628002056
:10DEC800C43E0020000016440827002080170020C8
:10DED800E8320020C43200206F12033B5C17002098
:10DEE800D44C9BF800300022212BCAF8682500F09A
:10DEF800BE84012B00F0EF85052B00F05187CE4B37
:10DF08001B7800220E9203F00108089B1A68079BF1
:10DF180092F846201B680B92069AD80492ED038A61
:10DF280040F14E84049B5D8AB8F1000F01D1AAF834
:10DF3800EC581521C148F7F761FB20B99AF87834F5
:10DF4800002B01F03E82049B9B8AA3F57A7303EBB6
:10DF5800D373C3F34F03EA1A1D4492B2ADB207EE6E
:10DF6800902AF8EEE77AA2F57A73C5F5FA6107EE1A
:10DF7800103A06EE901AF4EEC87AF1EE10FAB8EEFE
:10DF8800C77AF8EEE66A9AF9EE3803DA21780029BA
:10DF980001F0D381AA48AB49AB4AD1ED006A0C9095
:10DFA800A0F5916191ED006AC0ED006A16EE101AB5
:10DFB800127840F8041F0D90002A00F0ED8576EEE7
:10DFC800665AA24906910A46C1ED005A16EE901A01
:10DFD80077EEC87A42F8041FBCEEC88A01330A9269
:10DFE8009B4F0CBFDAF80029CAF8009918EE101AEE
:10DFF8004FF0FF030CBFA9EB02020022C7ED007A25
:10E00800AAF8EC188AF8EE38924B9A4240F2BB868E
:10E0180087EE878A2378904E3478F7EE007AB4EE4C
:10E02800E78AF1EE10FA88BFB0EE678AB5EEC08ACB
:10E038009FED927AF1EE10FAB8BFB0EE478A87EDFD
:10E04800008A002B40F0EE83844B089A93F800C0B6
:10E058001068834DBCF1010F06D190F8661005F1E8
:10E068008003012908BF1D46038D7E495A4207EEE9
:10E07800902A91ED046AF8EEE77A07EE103AB4EECA
:10E08800E76AF1EE10FAB8EE477A00F1F683B4EEDB
:10E09800C76AF1EE10FA88BFB0EE476AD1ED096A97
:10E0A800DFED715AF4EEE67AF1EE10FA26EE256A03
:10E0B80008DCB4EEE67AF1EE10FA8CBFF0EE667A80
:10E0C800F0EE477A438D91ED0E7ADFED675A5A42AA
:10E0D80006EE902AF8EEE66A67EEA57AB4EEE67ADE
:10E0E800F1EE10FA0AD406EE903AF8EE666AF4EE0B
:10E0F800C76AF1EE10FA88BFF0EE476A5B4B9FEDF6
:10E108005A7A5B7866EE876A0BB9F1EE666A0B9B02
:10E11800002B40F0A985F7EE005A554B1B68197C77
:10E12800C1B15B7C632B13D807EE103A9FED515AAF
:10E13800B8EEC77A012927EE057A02F07E87022910
:10E1480006D1B4EEC78AF1EE10FA88BFB0EE478A5E
:10E1580087ED008A484B1B78002B40F01583BCF1F3
:10E16800010F40F016839FED458A0123089387ED40
:10E17800008A002C02F0A783D5ED028AD5ED014A6A
:10E1880095ED035A9FED3D7A67EEA88AE6EE248A5C
:10E19800E6EE858A65EEA88AF4EEC78AF1EE10FAF3
:10E1A8008CBFB0EE479AB0EE689ACDED148AD8BF0E
:10E1B800F0EE478A012C00F0018195ED067AD5ED45
:10E1C800054A95ED075A27EE877AA6EE247AA6EE39
:10E1D800857A25EE877AB4EEE87AF1EE10FA00F344
:10E1E8008F84B4EEC79AF1EE10FA88BFB0EE479A62
:10E1F800022C8DED157A00F0E18095ED0A7AD5EDC7
:10E20800094A95ED0B5A27EE877AA6EE247AA6EEF0
:10E21800857A25EE877AB4EEE87AF1EE10FA00F303
:10E228005985B4EEC79AF1EE10FA88BFB0EE479A56
:10E2380026E000BFB6280020B7280020703B002049
:10E24800981E00204C2D002032530020A01E0020D4
:10E25800AC1E00208FD0030090600020C03000204A
:10E268000C190020C43E00206F12833A603D002044
:10E27800C43200200AD7233C4A2D002000000000A9
:10E28800032C8DED167A00F0998095ED0E7AD5ED78
:10E298000D4A95ED0F5A27EE877AA6EE247AA6EE58
:10E2A800857A25EE877AB4EEE87AF1EE10FA01F372
:10E2B8003980B4EEC79AF1EE10FA88BFB0EE479AEB
:10E2C800042C8DED177A79D095ED127AD5ED114A97
:10E2D80095ED135A27EE877AA6EE247AA6EE857A6C
:10E2E80025EE877AB4EEE87AF1EE10FA01F3E984C4
:10E2F800B4EEC79AF1EE10FA88BFB0EE479A052C33
:10E308008DED187A5AD095ED167AD5ED154A95ED1A
:10E31800175A27EE877AA6EE247AA6EE857A25EE96
:10E32800877AB4EEE87AF1EE10FA02F3AF82B4EE2F
:10E33800C79AF1EE10FA88BFB0EE479A062C8DED19
:10E34800197A3BD095ED1A7AD5ED194A95ED1B5AF5
:10E3580027EE877AA6EE247AA6EE857A25EE877AC6
:10E36800B4EEE87AF1EE10FA02F3A282B4EEC79A9C
:10E37800F1EE10FA88BFB0EE479A072C8DED1A7AA5
:10E388001CD0D5ED1E4A95ED1D5A95ED1F7A67EE06
:10E39800A47AE6EE057AE6EE877A65EEA77AF4EED9
:10E3A800E78AF1EE10FA02F1E683B4EEE79AF1EEAD
:10E3B80010FA88BFB0EE679ACDED1B7A78EEC99A4D
:10E3C8009AF81C306BB9DAEDCA7ADAEDCB6A38EE16
:10E3D800677AE6EE877A38EE677ACAEDCA7A8AED06
:10E3E800087ADAF80C3941F28732A9EB0303934231
:10E3F80000F3D8839AEDCC7A5FED606AB4EEE67AE2
:10E40800F1EE10FA1FDDDAEDC77A9AEDC85A78EE08
:10E41800675AB7EE006AE5EE257A78EE675ACAEDD4
:10E42800C77AA7EE258AB4EEC68AF1EE10FA88BF3D
:10E43800B0EE468AB4EEE68AF1EE10FAB8BFB0EE56
:10E44800668A87ED008AB7EE007AD34BCAED0B9A3D
:10E45800F4EEC79AF1EE10FA83ED008A40F3548384
:10E46800FCB3C7EE297A012C9DED147A27EE277AA2
:10E478008DED147A35D09DED157A27EE277A022C8A
:10E488008DED157A2DD09DED167A27EE277A032C7F
:10E498008DED167A25D09DED177A27EE277A042C74
:10E4A8008DED177A1DD09DED187A27EE277A052C69
:10E4B8008DED187A15D09DED197A27EE277A062C5E
:10E4C8008DED197A0DD09DED1A7A27EE277A072C53
:10E4D8008DED1A7A05D09DED1B7A67EE277ACDED82
:10E4E8001B7A089B1BB1B6EE008A87ED008A079B52
:10E4F8001B68DA0603D5B8F1000F40F07F87002CBF
:10E5080000F01C81A54B9AF9EE280699DAEDCF5A4E
:10E5180091ED006A0A9906EE902ADA780C9BD1ED03
:10E52800007A93ED007A0D9B93ED005A9C4BFDEE1B
:10E53800C74ABDEEC55AFDEEE55A1B78F8EEE66A05
:10E5480014EE901A15EE107A15EE900A002A41F092
:10E55800178295ED007ADDED145A28EE077AA6EEBB
:10E56800A57AF0EE675AE6EE075ABDEEE57A17EEA1
:10E57800103A994200F32E84BB42A8BF3B4607EEEF
:10E58800103AB8EEC77A874A012C82ED007A00F07B
:10E59800CD8095ED047ADDED155A28EE077AA6EEC2
:10E5A800A57AF0EE675AE6EE075ABDEEE57A17EE61
:10E5B800103A994240F3BA8607EE101AB8EEC77AB5
:10E5C800022C82ED017A00F0B18095ED087ADDED3C
:10E5D800165A28EE077AA6EEA57AF0EE675AE6EE06
:10E5E800075ABDEEE57A17EE103A994201F36D83AA
:10E5F800BB42A8BF3B4607EE103AB8EEC77A032CD9
:10E6080082ED027A00F0928095ED0C7ADDED175AD2
:10E6180028EE077AA6EEA57AF0EE675AE6EE075AD4
:10E62800BDEEE57A17EE103A994202F33D81BB42FE
:10E63800A8BF3B4607EE103AB8EEC77A042C82ED25
:10E64800037A73D095ED107ADDED185A28EE077A23
:10E65800A6EEA57AF0EE675AE6EE075ABDEEE57A21
:10E6680017EE103A994202F35381BB42A8BF3B46CA
:10E6780007EE103AB8EEC77A052C82ED047A55D029
:10E6880095ED147ADDED195A28EE077AA6EEA57AEB
:10E69800F0EE675AE6EE075ABDEEE57A17EE103A45
:10E6A800994202F36C82BB42A8BF3B4607EE103A80
:10E6B800B8EEC77A062C82ED057A37D095ED187A30
:10E6C800DDED1A5A28EE077AA6EEA57AF0EE675A1B
:10E6D800E6EE075ABDEEE57A17EE103A994202F3D4
:10E6E8002A84BB42A8BF3B4607EE103AB8EEC77A69
:10E6F800072C82ED067A19D095ED1C7ADDED1B5AB0
:10E7080028EE078AA6EEA58AE6EE087AFDEEE77AF5
:10E7180017EE903A994203DC9F423946A8BF194642
:10E7280007EE901AF8EEE77AC2ED077AB8F1000F13
:10E7380004D1A2001C491B4822F0C5FA1B4B1B78C8
:10E748002BB1002C7ED11A4B20461B6898479BF8AA
:10E758000030052B00F09F81164A1478002C7EF4B7
:10E768007AAF154DAA78002A40F0C2829BF8003093
:10E77800052B7EF470AF0CF037FD104A9BF8003083
:10E78800001BD080FEF767BFBCF1010F3FF4EBAC74
:10E7980001230893EDE400BF0C3F0020E02C00208B
:10E7A80032530020502D0020E81800200860002077
:10E7B8003C530020912D0020042D00200827002024
:10E7C800DF4BE04A93ED006ADAF8F834D2ED006ADC
:10E7D8009FEDDD7ADD4F07EE903A38EE478AF8EE86
:10E7E800E77A76EE665A07F27C4307F58F6107F2FF
:10E7F800744007F59065012297ED007A06930D9114
:10E808000C900A9577EE887AC3ED005A81ED006A7C
:10E81800C0ED006AC5ED006A07F591678AF8EE2831
:10E82800FFF7F6BBB8F1000F40F0FE82002C00F0B5
:10E838008287A200C649C74822F045FAC64B1B7812
:10E84800002B84D0C34FDFF844830025E8B2D8F802
:10E858000030B7EC010A984734780135A542F5DB5A
:10E8680071E7022DA8BF02252B46FFF7BDBABB4BA7
:10E878001A6000230E93FFF748BBB0EE676A0DE4F9
:10E88800B74BB849588B1D78049542F210750A6841
:10E89800DFF8FCB2B14F9BF800C005FB00F5B5FBF3
:10E8A800F2F5B4F95020B7F90600AE4207EE902A07
:10E8B80002F0508394ED197AD4F880E0F8EEE77A04
:10E8C8000EF1010237EE277A012AC4F8802084ED80
:10E8D800197A02F07686D4ED1C5AD4ED1E6A07EE3A
:10E8E800102A37EEE56AB8EEC75A012E86EE057A89
:10E8F80037EE257A77EEC77A84ED1D7AE7EE866AD9
:10E9080084ED1C7AF0EE667AC4ED1F6AC4ED1E6AC7
:10E9180000F04886B4F9522094ED1A7A07EE902A4E
:10E92800D4F89420F8EEE77A02F1010C37EE277A52
:10E93800BCF1010FC4F894C084ED1A7A02F04B863A
:10E94800D4ED215AD4ED236A07EE10CA37EEE56AF2
:10E95800B8EEC75A012E86EE057A37EE257A77EE9D
:10E96800C77A84ED227AE7EE866A84ED217AF0EEA2
:10E97800667AC4ED246AC4ED236A00F09286B4F97D
:10E98800542094ED1B7A07EE902AD4F8A820F8EECC
:10E99800E77A02F1010C37EE277ABCF1010FC4F8CF
:10E9A800A8C084ED1B7A00F04886D4ED265AD4ED31
:10E9B800286A07EE10CA37EEE56AB8EEC75A012E84
:10E9C80086EE057A37EE257A77EEC77A84ED277AD0
:10E9D800E6EE276A84ED267AF0EE667AC4ED296AB7
:10E9E800C4ED286A00F08186F880D4F8AC309BF832
:10E9F8000050013BC4F8AC30FEF71EBF16215A4840
:10EA0800F6F7FCFD00283FF446AA584B1B885B0626
:10EA18003FF541AA9AF8E038A34242F00685544AE5
:10EA2800544B92ED008A93ED000A9AED6F7ADAED75
:10EA38006D5A9FED516ADFED516A60EE477A25EE17
:10EA4800800AE5EE887AA7EE080AF4EEC67AF1EEB7
:10EA580010FA88BFF0EE467AF4EEE67AF1EE10FA94
:10EA6800B4EEC60AB4BFB0EE667AB0EE677AF1EEDD
:10EA780010FA8CBFF0EE467AF0EE407AF4EEE67AC1
:10EA8800F1EE10FAB8BFF0EE667A8AED6D7ACAED4B
:10EA98006F7AFFF700BA0CF0A7FB9BF800300E99CD
:10EAA8002E4A401A052B908040F018810CF09CFBF0
:10EAB800334B1B780446002B7FF458AE51E60CF01C
:10EAC80093FB264B001B5880FFF72BB90CF08CFBEF
:10EAD8000446FFF71CB90CF087FB2A4ADAF8E83835
:10EAE800294E12681D490E900546EB1A3078CAF86F
:10EAF800E8589A1ACA808B8000F00108FFF705BA17
:10EB0800F0EE478AFFF774BB089B002B00F0D28415
:10EB1800B1EE499AB4EEC89AF1EE10FA0ADCB7EEF3
:10EB2800009A39EE689AB4EEC89AF1EE10FA88BFE6
:10EB3800B0EE489AB0EE498A87ED009AD7E400BF54
:10EB4800702D00204C2D002000007A44241A00204B
:10EB5800E8180020502D0020086000200827002019
:10EB6800744700209C470020703B0020482D00205F
:10EB7800900500208C1E002000C0F94400C0F9C494
:10EB8800912D0020B8600020B728002034530020C1
:10EB9800042700200000C84276EEC65AF0EE466A06
:10EBA800FFF70FBA1FED050A28EE000A22F030F829
:10EBB8008A4B0B90D3F8683598423FF41BAC884BCE
:10EBC800DFED887A1B780F9307EE100AB8EEC7AA14
:10EBD8002AEE27AA002B39D0834BDFED846A1B88E5
:10EBE80007EE903A2AEE4A6AF8EEE77AF7EE085A04
:10EBF800B7EE007A67EEA57AA6EE267A67EE8A7AED
:10EC080067EE877A17EE900A21F00EFB784B0A46DA
:10EC180001461888CDE9101221F0E4FA02460B46A5
:10EC2800DDE91001CDE9122321F0CAFB18B99DEDE9
:10EC3800127B8DED107BDDE9100121F0D5FB0F9BD8
:10EC4800012B02F02C84022B02F05E859AF83433F3
:10EC58000F93002B42F07982604B0B9AC3F868251A
:10EC6800CAF80C99FFF7C6BB624B597A00293FF4E2
:10EC780052AA6149097800293FF44DAA1B889FEDE3
:10EC88005F4A07EE103A5E4BF8EE475A1B8807EECC
:10EC9800101A05EE103AB8EEC77AB8EE455A25EEC6
:10ECA800877AF7EE004AC7EE055AF4EEC45AF1EE39
:10ECB80010FA88BFF0EE445AF4EEE45AF1EE10FA76
:10ECC800B8BFF0EE645AFFF728BA4E4B226D1A60AF
:10ECD800FEF779BCF0EE478AFFF7D2BA4A4A1478B1
:10ECE800002C7EF4B8AC494DAA78002A3EF4B3ACA7
:10ECF800474E3378013B0A2B00F28F85DFE813F08B
:10ED08006C050806810522058D058D05F405C205EB
:10ED1800D305AD059805BAF8EC18914204D89AF8CD
:10ED28007824002A02F08D819AF80829002A42F0F6
:10ED38008881384F384AD7ED007A92ED007A37EE5D
:10ED4800676A07F2944207F5926107F28C4007F56B
:10ED58009365012B06920D910C900A9582ED006A3D
:10ED680081ED007AC0ED007AC5ED007A02F0638685
:10ED780007F5946700220123CAF80099B0EE667A75
:10ED88003A608AF8EE382549254B0978D7ED007A9C
:10ED980000225A609A61DA6201F00108FFF738B977
:10EDA8000CF022FA1D4B0E901B7803F00108FFF7B8
:10EDB800ACB8172D7EF407AC1A4E124C96ED010A2A
:10EDC80021F026FF96ED020A208021F021FF6080C5
:10EDD800FEF7F9BBB0EE647AFFF7D3BB2C00002036
:10EDE800384E00200AD7233C3C4E0020ABAAAA3E4E
:10EDF8003A4E0020D4270020CD2C0020713DAA3F98
:10EE0800C02C002008270020912D0020042D002070
:10EE18003C3800200C1A0020702D0020B728002054
:10EE2800C43E00209C470020DAED7A5A9AED775AC2
:10EE38009AED7B6ADAED764ADAED786AF24B9AED6A
:10EE48007C3A5A7865EEA53AB5EEC05AF1EE10FA5A
:10EE5800BFEE005AF5EEC04AE6EE063A54BFB0EEF1
:10EE6800454AB0EE674AF1EE10FAF5EEC06A54BFB3
:10EE7800F0EE454AF0EE674AF1EE10FA54BFF0EEB4
:10EE8800456AF0EE676A58BFB0EE675A002A18BFA5
:10EE9800B0EE665AF1EEE36AF4EEC65AF1EE10FAF5
:10EEA800B4BFF0EE467AF0EE657AF4EEC37AF1EE8E
:10EEB80010FADFEDD67A48BFF0EE436A66EEA77A1D
:10EEC80035EE863A48BFF0EE474AC3EE273A58BFB8
:10EED800B0EE475A9FEDCE7AF4EEC73A48BFB0EE8F
:10EEE800644AF1EE10FA0BD5DFEDCA7AF4EEC65A91
:10EEF800F1EE10FAD8BFF0EE674A88BFB0EE674A65
:10EF08009FEDC57A9FEDC36ADFEDC47A36EEC77A06
:10EF1800B4EEC67AF1EE10FAB8BFB0EE467A27EE34
:10EF2800277A002C00F007849B780A9ADFEDBC7AD8
:10EF380092ED006A069ADAEDCF5AD2ED003A06EE63
:10EF4800903AB8EE663AF3EE046A23EE273A76EE84
:10EF5800266ADAEDDA7A002B41F01C86DAEDDB2A34
:10EF68009AEDDC3A64EEA77AE4EE227AE5EE037ACB
:10EF7800F5EEC07AF1EE10FA02F1EA8167EE277A2F
:10EF8800B7EE003AF4EEC37AF1EE10FA88BFF0EE6D
:10EF9800437AB0EE463AA3EEA73AF0EE437AF4EE9F
:10EFA800E76AF1EE10FA9CBFB3EE043A77EEC37A43
:10EFB8009C4A88BFF0EE657A012CC2ED007A3FF4D6
:10EFC8003DACDAEDDE7ADAEDDF2A9AEDE03A64EE6E
:10EFD800A77AE4EE227AE5EE037AF5EEC07AF1EE4E
:10EFE80010FA02F1128267EE277AB7EE003AF4EED1
:10EFF800C37AF1EE10FA88BFF0EE437AB0EE463AE3
:10F00800A3EEA73AF0EE437AF4EEE76AF1EE10FACF
:10F018009ABFB3EE043A77EEC37AF0EE657A022C23
:10F02800C2ED017A3FF40AACDAEDE27ADAEDE32ACE
:10F038009AEDE43A64EEA77AE4EE227AE5EE037AF2
:10F04800F5EEC07AF1EE10FA02F1558267EE277AF2
:10F05800B7EE003AF4EEC37AF1EE10FA88BFF0EE9C
:10F06800437AB0EE463AA3EEA73AF0EE437AF4EECE
:10F07800E76AF1EE10FA9ABFB3EE043A77EEC37A74
:10F08800F0EE657A032CC2ED027A3FF4D7ABDAEDE5
:10F09800E67ADAEDE72A9AEDE83A64EEA77AE4EE42
:10F0A800227AE5EE037AF5EEC07AF1EE10FA02F173
:10F0B800848267EE277AB7EE003AF4EEC37AF1EE6F
:10F0C80010FA88BFF0EE437AB0EE463AA3EEA73ABC
:10F0D800F0EE437AF4EEE76AF1EE10FA9ABFB3EE77
:10F0E800043A77EEC37AF0EE657A042CC2ED037A1F
:10F0F8003FF4A4ABDAEDEA7ADAEDEB2A9AEDEC3AD2
:10F1080064EEA77AE4EE227AE5EE037AF5EEC07AA9
:10F11800F1EE10FA02F1848367EE277AB7EE003A2F
:10F12800F4EEC37AF1EE10FA88BFF0EE437AB0EE4F
:10F13800463AA3EEA73AF0EE437AF4EEE76AF1EE28
:10F1480010FA9ABFB3EE043A77EEC37AF0EE657A16
:10F15800052CC2ED047A3FF471ABDAEDEE7ADAED04
:10F16800EF2A9AEDF03A64EEA77AE4EE227AE5EE19
:10F17800037AF5EEC07AF1EE10FA02F1868367EEB3
:10F18800277AB7EE003AF4EEC37AF1EE10FA88BFA8
:10F19800F0EE437AB0EE463AA3EEA73AF0EE437AA1
:10F1A800F4EEE76AF1EE10FA9ABFB3EE043A77EE9E
:10F1B800C37AF0EE657A062CC2ED057A3FF43EABD1
:10F1C800DAEDF27ADAEDF32A9AEDF43A64EEA77AF8
:10F1D800E4EE227AE3EE057AF5EEC07AF1EE10FA63
:10F1E80002F1C48367EE277AB7EE003AF4EEC37AE9
:10F1F800F1EE10FA88BFF0EE437AB0EE463AA3EE8D
:10F20800A73AF0EE437A0FE0603D0020F304B53FE3
:10F21800D7B35D3F000000009A99193E9696963F35
:10F228000AD723BC502D0020F4EEE76AF1EE10FA5D
:10F238009ABFB3EE043A77EEC37AF0EE657A072CFC
:10F24800C2ED067A3FF4FAAADAEDF67ADAEDF72A91
:10F258009AEDF83A64EEA77AE4EE227AE5EE037ABC
:10F26800F5EEC07AF1EE10FA0CD427EE277AF7EE15
:10F27800007AB4EEE77AF1EE10FA88BFB0EE677A5A
:10F28800A7EE236AF4EEC66AF1EE10FA9CBFF3EE1D
:10F29800045A76EE655AC2ED075AFFF7CFBAAE4B5D
:10F2A800079304F5397304F12C0604F5017B04F186
:10F2B800B4070693D4ED077AA84BB6EC010AD4F844
:10F2C8009021581920EE270A9047D4F800220BEB1A
:10F2D80005009047D4F8B02078199047A04BD4F88F
:10F2E800202158199047079B1A68900000F15F8405
:10F2F80024356C2D86ED020ADCD1DFF8A0B29BF82C
:10F308000050984B1B7D23B1974B1B78002B01F0C5
:10F318004186079B1B689F0000F1DB84D4F8AC3062
:10F32800FEF78ABAF0EE478AFEF7CABFBB42A8BF0B
:10F338003B4607EE103AFFF741B907EE905AF8EE50
:10F34800E77AF4EEC87AF1EE10FA3FF6E4AC874AB1
:10F35800874892ED007A90ED006A864F78EE677ADA
:10F36800BCEEC88A012B02F2944002F5926502F2C3
:10F378008C4602F5936282ED007A0A9276EE475A3D
:10F3880008BFDAF8002986ED007A18BF0A4618EE99
:10F39800101A4FF0010306900D950C96C0ED005A17
:10F3A80085ED006A0CBFA9EB0202CAF80099B0EE1D
:10F3B800667AC7ED007AAAF8EC188AF8EE38FEF7F4
:10F3C80023BEBAF87234EA1A1D4492B2ADB2FEF7FF
:10F3D800C6BD002801F05E8200238AF8A5381FF018
:10F3E80077FF9AF8743801222270002B01F05B86AF
:10F3F800614E9AF8A5283578FEF7ECBBDF043FF597
:10F408007EA8089B002B7FF47AA85C4B1B88180504
:10F418003FF575A85A4A049BB2F906209B8A9A427E
:10F42800BFF66DA8002C3FF489A9564ADAF83C3398
:10F438001360012C3FF482A9022C53603FF47EA98B
:10F44800032C93603FF47AA9042CD3603FF476A987
:10F45800052C13613FF472A9062C53613FF46EA981
:10F46800072C93613FF46AA9D361FFF767B90B9B37
:10F47800DE0700F1B483012318F0010F3EF412AC4B
:10F48800414A92ED027A002B40F0DB83069BFF078E
:10F4980083ED027A04D592ED037A069B83ED037A15
:10F4A8009AF87428FEF728BC0B9BD80700F1FA835A
:10F4B8000A9BE1E7F6EE007AB4EEE78AF1EE10FA7D
:10F4C8007FF715A8FFF724BB0693FEF7FDB9049A4A
:10F4D8002D4B92F8282003EB820393ED000A21F0CC
:10F4E80097FB2A4AD4F898301080D380FEF79DBB4A
:10F4F800274B5B88FEF758BA264F386841F28832A6
:10F50800904241F2CD85244A1168002942F06F806B
:10F518009BF8002035782B2A7EF4DFAB1B4ABAF81B
:10F528007608D1801080D4F8A010D4F898005180C3
:10F538009080049AEE0792F8291042F1A380124AAB
:10F5480092ED007A002B42F086826B100B934FEA03
:10F55800A508EF10FEF708BA344E002040490020F5
:10F56800D048002074470020D80800200C1A00203A
:10F57800702D0020AC1E002090610020482D002036
:10F5880024330020502D0020501E00200827002082
:10F598007839002098450020B86000200427002012
:10F5A8000AD7233C012A41F3E98407EE10EAB8EEB2
:10F5B800C77AC7EE876AB1EEE68ABCF1140F02F08B
:10F5C800A185049A4AB107EE902AF8EEE77AF4EE9C
:10F5D800C87AF1EE10FA00F19F8007EE905AD4ED48
:10F5E800196AF8EEE77AAE4286EEA77A84ED087AD1
:10F5F8007FF490A9B4F9522007EE902A4FF0010C3D
:10F60800F8EEE77A00226645C4ED1A7AC4ED227A4C
:10F61800C4ED217A6262C4F88C20C4F894C056D034
:10F62800B4F9542007EE902AF8EEE77A0021012277
:10F63800C4ED1B7AA162C4F8A8200022012EC4EDF3
:10F64800277AC4ED267AC4F8A0207FF4CDA907EE66
:10F65800905AD4ED1B5AB3F912305FED2F6AF88037
:10F66800B8EEE76A07EE103AC5EE867AB44B197819
:10F67800DAF8303600225A63C3E90E22B8EEC77AA8
:10F68800E7EE667AC4ED0A7A1A6329B1AD4B1B68B6
:10F6980033F400637FF4A9A9012007F0C1FEFFF746
:10F6A800A4B9BCF1010F12DD07EE102AB8EEC77A33
:10F6B800049AC7EE876AF1EEE67A42B107EE102A9D
:10F6C800B8EEC77AF4EEC77AF1EE10FA24DC07EE4A
:10F6D800905AD4ED1A6AF8EEE77AAE4286EEA77A27
:10F6E80084ED097A7FF44BA99AE7BCF1010FAEDDEE
:10F6F80007EE102AB8EEC77A049AC7EE876AF1EEC9
:10F70800E67A002AA3D007EE102AB8EEC77AB4EE3C
:10F71800E77AF1EE10FA9AD55D8B0A68F88042F222
:10F72800107303FB05F39BF80050B3FBF2F3C4F826
:10F73800AC30FEF781B8844B1B78002B7FF403A80C
:10F74800FFF705B818F0D0FD804A0292A2F10C0329
:10F758002C2101930091A2F10A035021163A492065
:10F7680019F01EFE002858D1794B4FF0FF310722BF
:10F778001860596032702B79012B7EF4F7AF754F02
:10F78800754B1B78DA0741F186873A68DAF8101961
:10F798003378914248D8012B3EF4E8AF6F4D2A7870
:10F7A800002A3EF4E3AF0B2B0DD801229A4040F615
:10F7B800030112EA01080BD112F4C06F03D0093B10
:10F7C800012B42F2D984624B3A685A600B2333709A
:10F7D80000232B70FEF7CABF5F4B1B78D90702F1D5
:10F7E800B7812B79012B01F05587022B7EF4BEAF30
:10F7F8005A4B1B78002B7EF4B9AF19F0D3FFFEF7F4
:10F80800B5BFDFF84C81534F18F06EFDD8F80430BF
:10F818003A6864339342C2F0B4812B79012BAED09D
:10F82800022B7EF4A3AF3378012B7EF49FAFDFE782
:10F83800474B484F5B683968C8338B4204D318F08C
:10F8480075FD0028E9D0AA78032A02F0FD832B79F8
:10F85800012293423270C8D192E7414B1B78002BAA
:10F8680001F0A6861320FAF713FD002841F0A086C0
:10F878003A4B1B78002B41F09B860923337018F014
:10F88800B5FFCAE718F030FD18F0E6FF0028C4D02D
:10F8980018F04CFD0028C0D0324A334B12681A6069
:10F8A8000A23337067E71320FAF7F2FC0028E6D042
:10F8B8002E4B1B88002BE2D12D4B45201F6818F0DA
:10F8C80057FD0E2018F054FD384618F0A9FE48469A
:10F8D80018F0A6FE234A244B12681A6048460A23E9
:10F8E80033701AF055FECAE718F0FEFC214B0520CC
:10F8F80000210090A3F10802CDE90111532019F06D
:10F908004FFD002889D1124A08231060337032E76E
:10F91800104F0F4A3B6853601749002313600322B6
:10F928000B60327027E7BAF8BC38013B1BB2002BDA
:10F93800AAF8BC3841F32781104EFEF790B800BFF3
:10F94800753D0020AC30002008600020E612030856
:10F958009C3B002098450020B7280020713D0020DE
:10F96800633D0020803B00207C3B0020903B002032
:10F978008C3B0020E81403085C3B002090610020C9
:10F98800002B40F0C98795ED007ADDED145A28EE7A
:10F99800077AA6EEA57AF0EE675AE6EE075ABDEEAC
:10F9A800E57A17EE103A984201F39083BB42A8BF5C
:10F9B8003B4607EE103AB8EEC77AD74A012C82EDDB
:10F9C800007A3EF4B3AE95ED047ADDED155A28EED3
:10F9D800077AA6EEA57AF0EE675AE6EE075ABDEE6C
:10F9E800E57A17EE103A984201F38784BB42A8BF24
:10F9F8003B4607EE103AB8EEC77A022C82ED017A40
:10FA08003EF494AE95ED087ADDED165A28EE077AA5
:10FA1800A6EEA57AF0EE675AE6EE075ABDEEE57A4D
:10FA280017EE103A984201F37C84BB42A8BF3B46CC
:10FA380007EE103AB8EEC77A032C82ED027A3EF44C
:10FA480075AE95ED0C7ADDED175A28EE077AA6EE1D
:10FA5800A57AF0EE675AE6EE075ABDEEE57A17EE9C
:10FA6800103A984201F37084BB42A8BF3B4607EEA8
:10FA7800103AB8EEC77A042C82ED037A3EF456AEFB
:10FA880095ED107ADDED185A28EE077AA6EEA57ADC
:10FA9800F0EE675AE6EE075ABDEEE57A17EE103A31
:10FAA800984201F3B684BB42A8BF3B4607EE103A22
:10FAB800B8EEC77A052C82ED047A3EF437AE95EDA0
:10FAC800147ADDED195A28EE077AA6EEA57AF0EE3B
:10FAD800675AE6EE075ABDEEE57A17EE103A9842F5
:10FAE80001F30D85BB42A8BF3B4607EE103AB8EEBE
:10FAF800C77A062C82ED057A3EF418AE95ED187A91
:10FB0800DDED1A5A28EE077AA6EEA57AF0EE675AC6
:10FB1800E6EE075ABDEEE57A17EE103A984201F381
:10FB28004385BB42A8BF3B4607EE103AB8EEC77AFA
:10FB3800072C82ED067A3EF4F9AD95ED1C7ADDEDE1
:10FB48001B5A28EE078AA6EEA58AE6EE087AFDEE8D
:10FB5800E77A17EE903A984203DC9F423846A8BFEE
:10FB6800184607EE900AF8EEE77AC2ED077AFEF734
:10FB7800DDBDB0EE480A069221F04AF8674B87EDE2
:10FB8800028A23F8180008F10108B8F1030F06F1FA
:10FB98002406069A7DF4B6ADFDF711BE04EB4801C4
:10FBA8005E4BB1F8501023F81810FDF7BFBD96ED65
:10FBB800CC7A5B4BD4F8702277EE007A5819C6EDF0
:10FBC800CC7A9047069BD4F874225819904724356C
:10FBD8006C2D86ED020A7FF46DABFFF78EBB514AA0
:10FBE80092ED017AD4ED0A6AD4ED0B7A002901F07E
:10FBF8005781D4ED0F5A94ED103AD4ED0C3A94EDA8
:10FC0800116A94ED0D4AD4ED124A94ED0E5A069BF2
:10FC180084ED0F7A65EEA77AC4ED105AE7EE267ADE
:10FC280084ED126AE3EE237AE6EE447AE4EEC57ACE
:10FC3800C4ED117AC3ED017A18F0010F2BD092EDC3
:10FC4800027AD4ED136AD4ED147A002901F05D81AB
:10FC5800D4ED185A94ED193AD4ED153A94ED1A6A80
:10FC680094ED164AD4ED1B4A94ED175A069B84ED81
:10FC7800187A65EEA77AC4ED195AE7EE267A84ED6C
:10FC88001B6AE3EE237AE6EE447AE4EEC57AC4ED25
:10FC98001A7AC3ED027AFB077FF502AC92ED037A7C
:10FCA800FEF709B81F4A92ED017A069B18F0010F7A
:10FCB80083ED017A7DF463AEF9073FF5ECABFFF70E
:10FCC800EFBBF0EE478AFEF71ABB07EE101AFEF7F5
:10FCD80094BC94F8583394F859230133DBB29A4210
:10FCE80084F8583301F0F68194F8F034002B3FF48F
:10FCF80015AB102D01F06C86002394F8F16406937F
:10FD0800062E00F2E283DFE816F0F3047A038B0391
:10FD18000F00DA007C040504502D0020082700207D
:10FD2800244A0020501E0020834B1A46B2EC011AC8
:10FD380093ED033AD2ED002AD3ED094AD3ED021A26
:10FD480093ED082AD3ED053A93ED074A93ED0B5A44
:10FD5800D3ED0D5A93ED0F6AD3ED116A93ED137A33
:10FD6800D3ED157A93ED049AD3ED068A93ED0A0A3A
:10FD7800D3ED0C0A93ED0E8A62EEA22A23EE033A23
:10FD880064EEA44AE1EE012A102DA1EEA13AE2EEBA
:10FD9800024A93ED101A93ED142AD3ED121A63EE6A
:10FDA800A33A24EE044A25EE055A65EEA55A26EE36
:10FDB800066A66EEA66A27EE077A67EEA77AE9EE84
:10FDC800093AE2EE027AA8EEA84AA0EE005AE0EE5E
:10FDD800A05AA8EE086AE1EE016AA1EEA17AB1EE96
:10FDE800E22AF1EEC32AB1EEE33AF1EEC43AB1EEFB
:10FDF800E44AF1EEC54AB1EEE55AF1EEC65AB1EE63
:10FE0800E66AF1EEC76AB1EEE77A03ED1E3A43ED12
:10FE18001D3A03ED1C4A43ED1B4A03ED1A5A43ED04
:10FE2800195A03ED186A43ED176A03ED202A43EDCA
:10FE38001F2A03ED167AD3ED175A93ED196AD3EDFD
:10FE48001B6A93ED1D7AD3ED1F7A93ED1E5A93ED3D
:10FE5800163AD3ED183A93ED1A4AD3ED1C4A65EEDB
:10FE6800A55A26EE066A66EEA66A27EE077A67EEB8
:10FE7800A77AE3EE035AA3EEA36AE4EE046AA4EEBB
:10FE8800A47AE5EE057AB1EEE55AF1EEC65AB1EE7E
:10FE9800E66AF1EEC76AB1EEE77A03ED155A43ED6B
:10FEA800145A03ED136A43ED126A03ED117A02F056
:10FEB800B78094F8F1640136F6B284F8F1641F4B08
:10FEC80019780F2902F3D280002301F243129FED23
:10FED8001C7ADDF810C004EB820218461F46F2ECCB
:10FEE800017A3FB952ED026AF4EEE76AF1EE10FAD0
:10FEF80009D5C8B2B4EEE77AF1EE10FA44BFB0EE15
:10FF0800677ACBB2674601311029E8D11A466C33BB
:10FF180004EB8303D3EDD75A531C25EEA56A07EEED
:10FF2800103A66EE257AB8EEC77A0F2A27EE277AB6
:10FF380000F0A38106E000BF384D0020983D002066
:10FF48000000000003F16C0104EB810191EDD75A28
:10FF5800F4EEC55AF1EE10FA40F38F8104EE903AB0
:10FF680066EE256AF8EEE44A0E2B77EEA67AA4EE42
:10FF7800A67A00F3828103F16D0104EB8101D1EDD2
:10FF8800D76AB4EEE65AF1EE10FA03F1010140F334
:10FF9800748165EE054A04EE101A24EE855AB8EE0F
:10FFA800C44A0F2977EE857AA4EE057A00F06581B8
:10FFB80003F16E0104EB810191EDD75AB4EEE65AD4
:10FFC800F1EE10FA03F1020140F1578166EEA64AFC
:10FFD80004EE101A64EEA66AB8EEC44A0F2977EE4A
:10FFE800A67AA4EE267A00F0488103F16F0104EBAB
:08FFF8008101D1EDD76AF4EE9E
:020000040801F1
:10000000C56AF1EE10FA03F1030140F13A8165EEA1
:10001000054A04EE101A24EE855AB8EEC44A0F2998
:1000200077EE857AA4EE057A00F02B8103F170015A
:1000300004EB810191EDD75AB4EEE65AF1EE10FAD5
:1000400003F1040140F11D8166EEA64A04EE101A88
:1000500064EEA66AB8EEC44A0F2977EEA67AA4EE3B
:10006000267A00F00E8103F1710104EB8101D1EDDC
:10007000D76AF4EEC56AF1EE10FA03F1050140F11A
:10008000008165EE054A04EE101A24EE855AB8EE9A
:10009000C44A0F2977EE857AA4EE057A00F0F18044
:1000A00003F1720104EB810191EDD75AB4EEE65AE7
:1000B000F1EE10FA03F1060140F1E38066EEA64A84
:1000C00004EE101A64EEA66AB8EEC44A0F2977EE61
:1000D000A67AA4EE267A00F0D48003F1730104EB33
:1000E0008101D1EDD76AF4EEC56AF1EE10FA03F1A1
:1000F000070140F1C68065EE054A04EE101A24EEB1
:10010000855AB8EEC44A0F2977EE857AA4EE057AAF
:1001100000F0B78003F1740104EB810191EDD75A2F
:10012000B4EEE65AF1EE10FA03F1080140F1A980AD
:1001300066EEA64A04EE101A64EEA66AB8EEC44A49
:100140000F2977EEA67AA4EE267A00F09A8003F1C2
:10015000750104EB8101D1EDD76AF4EEC56AF1EEC9
:1001600010FA03F1090140F18C8065EE054A04EEB6
:10017000101A24EE855AB8EEC44A0F2977EE857A14
:10018000A4EE057A7DD003F1760104EB810191EDB7
:10019000D75AB4EEE65AF1EE10FA03F10A0170D51F
:1001A00066EEA64A04EE101A64EEA66AB8EEC44AD9
:1001B0000F2977EEA67AA4EE267A62D003F17701B2
:1001C00004EB8101D1EDD76AF4EEC56AF1EE10FAC5
:1001D00003F10B0155D565EE054A04EE101A24EE25
:1001E000855AB8EEC44A0F2977EE857AA4EE057ACF
:1001F00047D003F1780104EB810191EDD75AB4EEB9
:10020000E65AF1EE10FA03F10C013AD566EEA64A71
:1002100004EE101A64EEA66AB8EEC44A0F2977EE0F
:10022000A67AA4EE267A2CD003F1790104EB8101A1
:10023000D1EDD76AF4EEC56AF1EE10FA03F10D03C1
:100240001FD565EE054A04EE103A24EE855AB8EE45
:10025000C44A0E2B77EE857AA4EE057A11D1A84B0D
:1002600093ED005AB4EEE65AF1EE10FA09D526EEF7
:10027000A65AF2EE0E4A65EE266AA6EEA47A77EE4C
:10028000A67A431C9A422CDD02F16B0304EB830334
:10029000D3EDD76AF4EEE56AF1EE10FA21D504EB5E
:1002A0008201033001F5A161531C0AE031ED016ABE
:1002B000B4EEE66AF1EE10FA13D5F0EE466A25EEDA
:1002C000A56A26EE256A05EE903AB8EEE55A984200
:1002D000F0EE665A77EE867AA5EE067A03F1FF33E2
:1002E000E4D1F5EEC07AF1EE10FA94F8F27441F32D
:1002F000C884C7EE278A834B07F5C8720792F7EECA
:10030000007A78EEE78A93ED008A28EE888A7E4BA1
:1003100018881FF06BFF02460B4618EE100ACDE955
:1003200004231FF085FF02460B46DDE90401CDE9F9
:10033000082320F049F818B99DED087B8DED047B6A
:10034000DDE9040120F074F807EBC70304EB830335
:1003500006EE100A03F20C6203F5C46092ED007A17
:10036000D0ED007AE6EE077A03F2246103F5C2626B
:10037000D1ED006AD2ED005A079AB0EE677AF0EE3E
:10038000667AE6EE257A03F5C36C04EB4202DCEDF7
:10039000006AB2F858E3A2F85EE3E7EE667A03F289
:1003A0001C6C03F21463FCEEC75AC0ED007ADCED5E
:1003B000007AD3ED006A67EEC77A15EE903AE6EE62
:1003C000267A9BB2A2F858330493C1ED007AFAF76B
:1003D00045FD0028B8BF4042142806DD4B4A049969
:1003E00013888B4238BF0B461380002F41F0F983EE
:1003F0000F2D01F0BD85112D41F07F86444BB4F8DF
:1004000078261A8065E0D4F8FC24B4F80015414839
:100410001FF042FD9BF80050102D01F00F8694F85C
:10042000F134013384F8F1343A4BB4F8F404D4F8DD
:1004300008251946B1EC016AD1ED007A77EEA77A6A
:10044000F0EE006AB0EE677AA6EE267A013803EB8A
:10045000C001D6EE267A08391032F6EE003A27EEC1
:10046000237A67EEA37A83ED207AC3ED217A1033E5
:1004700091ED027A91ED036A53ED016A53ED027A30
:1004800052ED014A12ED025A37EE674A76EEC65A2D
:1004900077EE277AE4EE845A0138A1F10801E5EEFF
:1004A000047A02F1080203F1080336EE267AE4EE3C
:1004B000877AE5EE475A67EEA37A25EEA37AC3ED75
:1004C0001C7A83ED1D7AD3D1102D00F0D88194F8D9
:1004D000F164114B94F8F0240136A3FB0613F11AD2
:1004E00003EB51039B08C3EBC303F61A013AD4F89C
:1004F000AC3084F8F16484F8F024FDF7A1B900BFB2
:10050000F44C0020943D0020903D0020203300203A
:1005100008270020B84C00202549922494F8F23492
:1005200094F86C2302F1DC0CC2F12002D0B20CEB87
:100530004313870804EB830C01F0AA853F0107F100
:100540001006E749E74A66440CF1100313ED024A2E
:1005500013ED035A13ED017A13ED046A51ED024ACB
:1005600051ED035A51ED046A51ED017A64EE244ACB
:1005700065EE255A66EE266A67EE277A10339E42AC
:1005800042ED024A42ED035A42ED046A42ED017A1D
:1005900001F1100102F11002D8D1D34ED34ABC446C
:1005A000F319174410F003021BD09CED007AD3ED31
:1005B000007A67EE877A012AC7ED007A11D09CEDA8
:1005C000017AD3ED017A67EE877A022AC7ED017AC4
:1005D00007D09CED027AD3ED027A67EE877AC7EDF9
:1005E000027A94F86C330493002B41F05983102D58
:1005F0007FF46DAF0AF0FCFD069ABD4B94F8F164F0
:100600009BF80050801A588063E794F8F25405F57F
:10061000C87304EB4303B3F85823B3F85E33934233
:1006200000EE102A50D0B34BB34EB44FB44A1B78EF
:100630001168D7ED000A05EBC50506EB8505D5ED7C
:10064000058A95ED068AD5ED079A95ED089A002B57
:1006500001F02985AB4BB8EEC00AD3ED007A2846ED
:1006600020EE270A1CF05AFAC5ED058A85ED068AA8
:10067000C5ED079A85ED089A94F8F234A24AA0498C
:1006800092ED000AD7ED000A096804EB430206F177
:100690006C05B2F8782607EE902A03EBC30305EB4E
:1006A0008305F8EEE77AD5ED058A95ED068AEF69C0
:1006B0002E6A27EE800A28461CF030FAC5ED058A1E
:1006C00085ED068AEF612E629BF80050102D01F037
:1006D000F98494F8F2348D4A94F8F1140133A2FBB2
:1006E0000302520802EB42029B1ADBB2013184F88A
:1006F000F23484F8F11413E7B4F8F4147B48D4F816
:10070000F8244FEA510E4FEA8E065FEAD10C06EB51
:10071000000300EB810500F0A18006F1100103EB5E
:100720000C1C29440CF1100C1030103302F110078E
:1007300005F1100656ED032A56ED043A10ED043A81
:1007400010ED032A56ED026A16ED016A10ED021A49
:1007500050ED010A11ED044A11ED035A53ED044A1C
:1007600053ED035A13ED027A53ED017A51ED021A5B
:1007700011ED010A73EE238A32EE228A40ED048ADB
:1007800000ED038A71EE268A30EE868A40ED028AF9
:1007900000ED018A74EE848A35EE858A43ED048A81
:1007A00003ED038A77EE218A37EE808A43ED028AD1
:1007B00003ED018A73EE633A75EE655A17ED035A3D
:1007C00032EE623A74EE644A25EE638A17ED044A0B
:1007D00023EE052A64EE652AA3EE048A10336345EE
:1007E00024EE843AA3EE842A00F1100007F11007EA
:1007F000A5EE853A06F1100601F11001E4EE852A16
:1008000006ED078A06ED082A01ED073A41ED082AB0
:1008100057ED055A17ED065A71EE666A30EEC66A54
:1008200031EEC77A70EE677A26EE253A65EEE63A43
:1008300025EE674A67EE054AE6EE053AA6EE853AEA
:10084000A7EE254AE7EEA54A06ED063A46ED053A3B
:1008500001ED064A41ED054A7FF46CAF1FFA8EF6B2
:10086000314622481DF0FCF928463146D4F8F824D8
:100870001DF0F6F99BF80050102D7FF428AE0AF019
:10088000B7FC069A1A4B94F8F1649BF80050801A52
:1008900058801EE6F0EE478AFDF754BD1C4E01213C
:1008A00035788AF8A518002A3DF44FA8FDF796B9C7
:1008B00007EE101AFDF7C4BEF0EE478AFDF761BDE2
:1008C000BAF8763803F57A739BB2FDF771B8DFEDAD
:1008D000119AB0EE699AF0EE698AFDF775BD00BF16
:1008E000AC3D0020C84C00209C3D0020B84C0020AE
:1008F00008270020D7080020244A00208C3D002033
:100900009C470020843D0020883D0020ABAAAAAA75
:10091000906100200000000007EE101AFDF7AEBE47
:10092000D5ED005A9DED145A68EE255AE6EE855A2B
:10093000B0EE675AA6EE255AB4EEC57AF1EE10FA7B
:1009400000F3C183FDEEC55A15EE903A9842C8BF38
:1009500005EE900A40F3B883F8EEE55A8D4A012C73
:10096000C2ED005A3DF4E6AED5ED045A9DED155AA0
:1009700068EE255AE6EE855AB0EE675AA6EE255A7D
:10098000B4EEC57AF1EE10FA00F3BF84FDEEC55A5D
:1009900015EE903A9842C8BF05EE900A40F3B6842F
:1009A000F8EEE55A022CC2ED015A3DF4C3AED5ED86
:1009B000085A9DED165A68EE255AE6EE855AB0EEB5
:1009C000675AA6EE255AB4EEC57AF1EE10FA00F396
:1009D000A484FDEEC55A15EE903A9842C8BF05EEC4
:1009E000900A40F39B84F8EEE55A032CC2ED025ABC
:1009F0003DF4A0AED5ED0C5A9DED175A68EE255A80
:100A0000E6EE855AB0EE675AA6EE255AB4EEC57AE0
:100A1000F1EE10FA00F3A484FDEEC55A15EE903AFB
:100A20009842C8BF05EE900A40F39B84F8EEE55A61
:100A3000042CC2ED035A3DF47DAED5ED105A9DED68
:100A4000185A68EE255AE6EE855AB0EE675AA6EEB9
:100A5000255AB4EEC57AF1EE10FA00F3E284FDEE09
:100A6000C55A15EE903A9842C8BF05EE900A40F379
:100A7000D984F8EEE55A052CC2ED045A3DF45AAE7D
:100A8000D5ED145A9DED195A68EE255AE6EE855AB1
:100A9000B0EE675AA6EE255AB4EEC57AF1EE10FA1A
:100AA00000F32585FDEEC55A15EE903A9842C8BF71
:100AB00005EE900A40F31C85F8EEE55A062CC2EDCF
:100AC000055A3DF437AED5ED185A9DED1A5A68EE29
:100AD000255AE6EE855AB0EE675AA6EE255AB4EED0
:100AE000C57AF1EE10FA00F31285FDEEC55A15EE47
:100AF000903A9842C8BF05EE900A40F30985F8EE97
:100B0000E55A072CC2ED065A3DF414AED5ED1C5A39
:100B10009DED1B5A28EE258AA6EE858AE6EE087A18
:100B2000B4EEE77AF1EE10FA08DCFDEEE77A17EEA4
:100B3000903A98423FF719A817EE900AB842A8BF1A
:100B40003846FFF712B80F2A00F00082112A40F051
:100B5000FA81B0EE480A20F05FF80F4BD880FCF71E
:100B6000F1BD9BF800200F2A00F0E383112A40F02A
:100B7000E68320F051F8084B9880FCF702BEF0EEB7
:100B8000678AFDF71DBC07EE101AFDF795BD00251D
:100B9000FDF7B2B8502D0020082700209AEDDB2A7F
:100BA000DAEDDC2A64EEA77AE4EE027AE5EE227A48
:100BB000F5EEC07AF1EE10FA00F13F8667EE277A83
:100BC000F7EE002AF4EEE27AF1EE10FA88BFF0EECA
:100BD000627AF0EE462AE3EEA72AF0EE627AF4EEAD
:100BE000E76AF1EE10FA9CBFF3EE042A77EEE27AA0
:100BF000E64A88BFF0EE657A012CC2ED007A3DF43A
:100C000021AEDAEDDE7A9AEDDF2ADAEDE02A64EE43
:100C1000A77AE4EE027AE5EE227AF5EEC07AF1EEFA
:100C200010FA00F1448667EE277AF7EE002AF4EE18
:100C3000E27AF1EE10FA88BFF0EE627AF0EE462A20
:100C4000E3EEA72AF0EE627AF4EEE76AF1EE10FA2C
:100C50009ABFF3EE042A77EEE27AF0EE657A022C80
:100C6000C2ED017A3DF4EEADDAEDE27A9AEDE32AD7
:100C7000DAEDE42A64EEA77AE4EE027AE5EE227A6F
:100C8000F5EEC07AF1EE10FA00F1788667EE277A79
:100C9000F7EE002AF4EEE27AF1EE10FA88BFF0EEF9
:100CA000627AF0EE462AE3EEA72AF0EE627AF4EEDC
:100CB000E76AF1EE10FA9ABFF3EE042A77EEE27AD1
:100CC000F0EE657A032CC2ED027A3DF4BBADDAEDAD
:100CD000E67A9AEDE72ADAEDE82A64EEA77AE4EEFE
:100CE000027AE5EE227AF5EEC07AF1EE10FA00F122
:100CF000918667EE277AF7EE002AF4EEE27AF1EEBB
:100D000010FA88BFF0EE627AF0EE462AE3EEA72AE8
:100D1000F0EE627AF4EEE76AF1EE10FA9ABFF3EEC3
:100D2000042A77EEE27AF0EE657A042CC2ED037ABB
:100D30003DF488ADDAEDEA7A9AEDEB2ADAEDEC2AA9
:100D400064EEA77AE4EE027AE5EE227AF5EEC07A56
:100D5000F1EE10FA00F1958667EE277AF7EE002A99
:100D6000F4EEE27AF1EE10FA88BFF0EE627AF0EE7D
:100D7000462AE3EEA72AF0EE627AF4EEE76AF1EE95
:100D800010FA9ABFF3EE042A77EEE27AF0EE657A73
:100D9000052CC2ED047A3DF455ADDAEDEE7A9AED0C
:100DA000EF2ADAEDF02A64EEA77AE4EE027AE5EEB5
:100DB000227AF5EEC07AF1EE10FA00F1B88667EE0D
:100DC000277AF7EE002AF4EEE27AF1EE10FA88BF05
:100DD000F0EE627AF0EE462AE3EEA72AF0EE627AAF
:100DE000F4EEE76AF1EE10FA9ABFF3EE042A77EE1A
:100DF000E27AF0EE657A062CC2ED057A3DF422AD7A
:100E0000DAEDF27A9AEDF32ADAEDF42A64EEA77AB3
:100E1000E4EE027AE5EE227AF5EEC07AF1EE10FA0F
:100E200000F1F38667EE277AF7EE002AF4EEE27A15
:100E3000F1EE10FA88BFF0EE627AF0EE462AE3EEA9
:100E4000A72AF0EE627AF4EEE76AF1EE10FA9ABFA2
:100E5000F3EE042A77EEE27AF0EE657A072CC2ED23
:100E6000067A3DF4EFACDAEDF67A9AEDF72ADAED90
:100E7000F82A64EEA77AE4EE027AE5EE227AF5EE3D
:100E8000C07AF1EE10FA00F1D58667EE277AB7EE58
:100E9000007AF4EEC77AF1EE10FA88BFF0EE477AE6
:100EA000A3EEA76AFEF7F2B937EE667A069BE7EE85
:100EB000276AC4ED0A6AC3ED016AFEF7C1BE0029C4
:100EC0003CF43BADFEF78CBAD4ED215AD4ED223A76
:100ED00094ED1E3A94ED236A94ED1F4A94ED245A42
:100EE000D4ED204A069B84ED217A65EEA77AC4ED05
:100EF000225AE7EE267A84ED246AE3EE237AE4EEC2
:100F0000467AE4EEC57AC4ED237AC3ED037AFEF7A0
:100F1000CBBA37EE667A069BE7EE276AC4ED136A12
:100F2000C3ED026AFEF7BBBE37EE667A069BE7EEBC
:100F3000276AC4ED016AC3ED006AFCF7AEBE07EE96
:100F4000101AFDF7D7BB2D2A7CF4FCABB0EE480A93
:100F50001FF062FE0E4B1880FCF7F4BBF8EEE77A48
:100F600001224FF0000E9642C4ED197AC4ED1D7AAD
:100F7000C4ED1C7AC4F820E0C4F878E0C4F88020FE
:100F80007EF43CAB9FED038AFEF71BBB502D002087
:100F9000082700200000000000D8F946D4ED0E7AA2
:100FA00094F8542394ED077AFDEEE77A17EE901A41
:100FB0000029B8BF494207EE901AF8EEE77A002AF6
:100FC00040F0AD821FED0C6AD4ED0F6A27EE067A71
:100FD000FDEEE66AB4EEE77A16EE902AF1EE10FA2C
:100FE0004CBF01230023002AB8BF524207EE902ACB
:100FF000F8EEE77AB4EEE77AD4ED107AFDEEE77A10
:10100000F1EE10FA17EE902A48BF43F00203002ACF
:10101000B8BF524207EE902AF8EEE77AD74AB4EE0C
:10102000E77AF1EE10FA127848BF43F00403134256
:101030003EF473A90123C4F8509384F85433FEF7A7
:101040006CB928EE078AFDF787B8CD48CD49CE4A5E
:10105000D1ED007A0C90A0F59161D1ED006AC0ED60
:10106000007A16EE901A127840F8041F0D90002AAC
:1010700000F07E8136EEE76AC44906910A4681EDAA
:10108000006A17EE901A42F8041F591C0A9200F0E9
:101090008082069FCAF800990022FF2347F80C2F90
:1010A0008AF8EE38FDF773BE0021FEF735BAB84B6B
:1010B0001D7805F001030A936B100B934FEAA50806
:1010C000EF10FCF7B1BD0346BB42A8BF3B4605EE9F
:1010D000903A41E407EE100AFEF771BC94EDD78A0E
:1010E00094EDD80A94F86C63AA4F28EE000A04EB3A
:1010F000860200230F2D82EDDC0AB7F9040084F884
:10110000583301F04B80D4EDD97AB88067EE887AF5
:1011100004EB8603C3EDFC7AD4EDDA7A9BF8005039
:1011200027EE888A06F1460104EB8101721C002338
:1011300081EDD68A02F01F020C21C4F8603384F8D6
:101140006C23C4F86433C4F8683384F8F014FEF7F1
:10115000D4BDBAF83833DFED906A07EE903A2AEE44
:101160004A6AF8EEE77AF7EE085AB7EE007A67EEC9
:10117000A57AA6EE267A27EE8AAA6AEE077A17EEF5
:10118000900A1FF055F802460B46BAF83603CDE92F
:1011900010231FF02BF802460B46DDE91001CDE9C4
:1011A00012231FF011F918B99DED127B8DED107B04
:1011B000DDE910011FF01CF90F9B1090012B00F0CE
:1011C0005183022B7DF44CAD744B9FED757A93EDFA
:1011D000006ADFED744A744BDFED742A9FED744AA8
:1011E0009FED741ADFED741A9FED742A9FED743A27
:1011F00007EE900AB8EE466AF8EE677A26EE076ABE
:10120000F0EE643A26EE276A03F16C00FDEEC67A32
:1012100076EE244A17EE901AFDEEE47A203117EEAE
:10122000902AB7EE005A2032402900F20183B4EE32
:10123000E26AF1EE10FA40F34A86B0EE467ADFED4C
:10124000615ADFED616A01E0B0EE677AB4EEE67AEA
:10125000F1EE10FA77EE657AF6DCF4EEC47AF1EE90
:1012600010FA40F18F86DFED575ADFED586A01E042
:10127000F0EE477AF4EEE67AF1EE10FA37EEA57A60
:10128000F6D4B4EEE37AF1EE10FA40F3B48332EE22
:10129000C77A67EE077AF0EE615AE7EE815AF0EE10
:1012A000420AE5EEA70A67EE276AF0EE457AA6EE57
:1012B000A07AF0EE450AE7EE030AE7EE437A87EEFE
:1012C000A00A402A40F20B839FED417AF6EE006AB5
:1012D000F7EE005AC5EE207A243303ED050A67EED7
:1012E000A66A67EEA55A67EE877A43ED096A43ED71
:1012F000076A43ED085A43ED067A834294D1FDF71D
:10130000AFBC07EE100AFEF77ABB0346BB42A8BF8C
:101310003B4605EE903AFFF743BB0346BB42A8BFEE
:101320003B4605EE903AFFF75EBB07EE100AFEF76C
:1013300085BB1FF071FC174B5880FCF722BA2D2A91
:101340007CF41FAA1FF068FC124BD880FCF719BA76
:1013500007EE100AFEF791BBF0EE467AFDF723BECA
:101360000346BB42A8BF3B4605EE903AFFF75EBB83
:1013700037EEE66AF0EE667A7EE600BF723D002048
:10138000981E00204C2D002032530020A01E00206B
:101390009061002008270020ABAAAA3EB860002078
:1013A00027D4D236DB0FC93F48160020DB0F494057
:1013B000DB0F49C092E741B99730083C15A82ABE17
:1013C000F304353FDB0FC940E4CB1641E4CB16C133
:1013D00000000000069B0A9193ED000AB94E1FF031
:1013E0001BFCBAF87638B84AA6FB03139B0907EE34
:1013F000903AF8EEE77A0A991080FDEEE77A002934
:1014000017EE903A53803CF734AB91800223FCF7FF
:10141000EFBCF0EE467AFDF7FBBD07EE100AFEF7D3
:101420004BBB0346BB42A8BF3B4605EE903AFFF7D5
:1014300020BB07EE904AF8EEE78ADFEDA47A9FED35
:10144000B30A8AF8E04868EEA78A38EE800AFDEE13
:10145000C07A17EE903A2033402B40F2D6829FEDAF
:101460009C8A9C4BFDEEE87A83ED008A17EE903A59
:101470002033402B00F23082B0EE680AF2F7A8FD6C
:10148000954B83ED000AFDF7D4BA838E9FED937AD6
:1014900007EE903AF8EEE77A914B67EE877AC3ED64
:1014A000007AFCF71EBA07EE900ADFED8E5A9BF821
:1014B00000309FED8D7AB8EE676A2D2BC5EE866AF7
:1014C00004BF814B9880894BD3ED007A884BF8EEAE
:1014D000677A67EE877A76EEA76A87EEA67A83ED5B
:1014E0002E7A83ED377A83ED407AFDF7B3BB03465E
:1014F000BB42A8BF3B4605EE903AFFF7DDBAF0EEDF
:10150000467AFDF7B8BD07EE100AFEF7F4BA0346B7
:10151000BB42A8BF3B4605EE903AFFF7F0BADFEDBD
:10152000756A27EE267AB4EEE77AF1EE10FA40F308
:10153000C480D4ED0F7AFDEEE77A17EE902A002AE8
:10154000B8BF524207EE902AF8EEE77AB4EEE77A97
:10155000F1EE10FA40F3B180D4ED107AFDEEE77AA7
:1015600017EE902A002AB8BF524207EE902AF8EEF2
:10157000E77AB4EEE77AF1EE10FA40F39E80D4F801
:1015800050234CF25031A9EB02028A427DF7C5AEDE
:1015900053E5DFED4F7ADAF800298AF8EE38564F36
:1015A00017EE903AA9EB020247F80C3FFCF730BD6A
:1015B00007EE100AFEF7BEBA484618F0EDFFFEF738
:1015C00062B9F0EE467AFDF789BD0022012EC4ED26
:1015D0001D7AC4ED1C7AA2677DF4A0A9D2E4002292
:1015E000012EC4ED227AC4ED217AC4F88C207DF45A
:1015F000CAA9FEF770B8414A92F80080B8F1000F0E
:1016000000F04B81BAF876584BF66872A5F57A71FE
:10161000914200F24281DAF8B818002940F05B8468
:10162000002B14BF4FF4FA624FF47A720244CAF8E6
:10163000B8288242BDF470AF002B00F0A784D4F824
:10164000982094ED267ADFED2E5AAA1A002AB8BF08
:10165000524207EE902AB8EEC77AF8EEE77AB3EE78
:10166000046AC7EE876A66EEA57AF4EEC67AF1EEF2
:1016700010FA40F18B8400220021C4F89C204FF620
:10168000FF72C4E928120221FDF746BFAA0700F144
:10169000ED814FEAA508EF10FDF7F2BE194FF7F7FD
:1016A0006BFE00283EF475A83A68337802F59C5228
:1016B0000832CAF81029FEF7BBB8C4F85093FDF7FA
:1016C0002CBE00BFD34D62100827002035FA8E3C97
:1016D00000000000900500208C1E00206F12833A4D
:1016E000C007002083F9223EBD3786359C47002085
:1016F000AC4700200008ED46A01E00205C39002009
:101700000000C8429845002027D4D236DB0FC93FDD
:101710009BF800305FED046A1FED047A2D2B04BFA7
:10172000E24B9880E24BD3ED00AA07EE900AF8EE68
:101730006AAAF8EE677A6AEEA6AA6AEEA7AAFDEE92
:10174000EA7A3AEE87CA17EE902AFDEECC7A20327A
:1017500017EE903A402A03F1200300F2BF81402B9C
:10176000B0EE6A0A40F22E83F2F732FCB7EE00BA0E
:101770009FEDD0CAD04BDFEDD1CA0F93F0EE4B6A8C
:10178000E0EE0C6AB0EE4B7ACBEE267AA0EE4C7A05
:10179000F6EE00BA67EEAB6A27EE277AC3ED2E7A33
:1017A00083ED317AC3ED2D6AC3ED2F6AC3ED30CAE4
:1017B000B0EE6A0AF2F70CFCF0EE4B6AE0EE0C6A4F
:1017C0000F9BB0EE4B7ACBEE267AA0EE4C7A67EE0A
:1017D000AB6A27EE277AC3ED377A83ED3A7AC3ED09
:1017E000366AC3ED386AC3ED39CAB0EE6A0AF2F759
:1017F000EFFBF0EE4B6AE0EE0C6A0F9BB0EE4B7A1B
:10180000CBEE267AA0EE4C7A67EEABBA27EE277ABB
:10181000C3ED42CA83ED437AC3ED3FBAC3ED41BA8B
:10182000C3ED407AFDF716BAF0EE467AFDF789BCB3
:10183000B7EE000AF0EE400A43E567EE032AB7EE82
:10184000002A62EEA77AF0EE462AF4EEC27AF1EEB2
:1018500010FA88BFF0EE427AE3EEA72AF0EE627A41
:10186000FFF7BDB907EE900ADFED956A954BF8EEEC
:10187000677A86EEA77AD3ED006A37EE267AC6EE4F
:10188000877ACAED297ACAED327ACAED3B7AFDF73A
:10189000E7B9F0EE467AFDF787BC002000214FF64D
:1018A000FF72C4F89C00C4E92812FDF735BE67EE4C
:1018B000032AB7EE002A62EEA77AF0EE462AF4EE8B
:1018C000C27AF1EE10FA88BFF0EE427AE3EEA72A70
:1018D000F0EE627AFFF7B8B99FED780AD0E5B4EE82
:1018E000E36AF1EE10FA40F3FA83F0EE647ADFED8A
:1018F000765ADFED766A01E0F0EE477AF4EEE67AAA
:10190000F1EE10FA37EEE57AF6DCB4EEC47AF1EED9
:1019100010FA40F1E183DFED6C5ADFED6D6A01E012
:10192000B0EE677AB4EEE67AF1EE10FA77EE257A49
:10193000F6D4F4EEE37AF1EE10FA40F35C8172EE45
:10194000E77A67EEA76AF0EE615AE6EE815AB0EEEA
:1019500042AAA6EEA5AA66EEA76AB8EE007AE6EE5F
:101960008A7AF6EE006A75EE675A27EE877A65EE98
:10197000A66AAFE4F0EE467AFDF75ABC67EE032A9A
:10198000B7EE002A62EEA77AF0EE462AF4EEC27AAB
:10199000F1EE10FA88BFF0EE427AE3EEA72AF0EEFD
:1019A000627AFFF784B9424AD2ED027AF0EEE77A22
:1019B000FCEEE77A17EE903A9BB20F2B40F2D981FA
:1019C000DAF86835002B40F0468109F59233F83398
:1019D000CAF86835FCF7F1B909F00AFC9BF8005029
:1019E0000690102D05BF314B94F8F16494F8F16422
:1019F0001E80FEF789B9DFED377AB4EEE77AF1EEB3
:101A000010FA48BF34EE477A43E4F2F7E1FAB0EE59
:101A1000408A26E567EE032AB7EE002A62EEA77A2F
:101A2000F0EE462AF4EEC27AF1EE10FA88BFF0EE3C
:101A3000427AE3EEA72AF0EE627AFFF76BB9DFEDA8
:101A40001F7ADAF800298AF8EE3807F59467B0EEC5
:101A5000667AC7ED007AA9EB0202FCF7D9BA6B10DF
:101A60000B934FEAA508EF10FCF7EDB81A4A4FEABE
:101A7000A50892ED017AEF10002B3EF41AA9FEF7AB
:101A8000B5B867EE032AB7EE002A62EEA77AF0EE49
:101A9000462AF4EEC27AF1EE10FA88BFF0EE427AEE
:101AA000E3EEA72AF0EE627AFFF767B90827002075
:101AB0009C470020F304353FAC47002000000000A5
:101AC00083F9223E94610020DB0FC940E4CB16412C
:101AD000E4CB16C1DB0FC9BF501E0020402B40F2E3
:101AE000FF81B04B4FF07C520021C3F8B420C3F803
:101AF000BC20C3F8D820C3F8E020C3F8FC20C3F80A
:101B000004214FF07E52C3F8B820C3F8C420C3F8B4
:101B1000DC20C3F8E820C3F80021C3F80C21C3F887
:101B2000C010C3F8E410C3F80811FDF793B867EECE
:101B3000032AB7EE002A62EEA77AF0EE462AF4EE08
:101B4000C27AF1EE10FA88BFF0EE427AE3EEA72AED
:101B5000F0EE627AFFF744B91DF07EFB074680B1D4
:101B6000DFF85882D8F80030984200F0EC82D8F8BC
:101B7000DC30BB4200F0DE82D8F8B8319F4200F082
:101B8000D08217F0D7FCFDF74CBE402016F092FB38
:101B900000287DF446AED8F80030834F4FF040095E
:101BA0000DE016F0E9FB3A68D8F80030013A01334D
:101BB000B9F101093A60C8F8003000F096827B4A1A
:101BC000134493F80C321846002BEAD100234FF04F
:101BD000FF32C8F800300423C8F804203370FDF742
:101BE000CEBD012F02D1112D00F05782102D3EF4F1
:101BF00046AEFEF76EBC9FED6E7AF4EEC77AF1EE5C
